
F103_multitest.elf:     file format elf32-littlearm

Sections:
Idx Name          Size      VMA       LMA       File off  Algn
  0 .isr_vector   0000010c  08000000  08000000  00010000  2**0
                  CONTENTS, ALLOC, LOAD, READONLY, DATA
  1 .text         00004d00  0800010c  0800010c  0001010c  2**2
                  CONTENTS, ALLOC, LOAD, READONLY, CODE
  2 .rodata       000002cc  08004e0c  08004e0c  00014e0c  2**2
                  CONTENTS, ALLOC, LOAD, READONLY, DATA
  3 .ARM.extab    00000000  080050d8  080050d8  0002007c  2**0
                  CONTENTS
  4 .ARM          00000000  080050d8  080050d8  0002007c  2**0
                  CONTENTS
  5 .preinit_array 00000000  080050d8  080050d8  0002007c  2**0
                  CONTENTS, ALLOC, LOAD, DATA
  6 .init_array   00000004  080050d8  080050d8  000150d8  2**2
                  CONTENTS, ALLOC, LOAD, DATA
  7 .fini_array   00000004  080050dc  080050dc  000150dc  2**2
                  CONTENTS, ALLOC, LOAD, DATA
  8 .data         0000007c  20000000  080050e0  00020000  2**2
                  CONTENTS, ALLOC, LOAD, DATA
  9 .bss          00000100  2000007c  0800515c  0002007c  2**2
                  ALLOC
 10 ._user_heap_stack 00000604  2000017c  0800515c  0002017c  2**0
                  ALLOC
 11 .ARM.attributes 00000029  00000000  00000000  0002007c  2**0
                  CONTENTS, READONLY
 12 .debug_info   000069f5  00000000  00000000  000200a5  2**0
                  CONTENTS, READONLY, DEBUGGING, OCTETS
 13 .debug_abbrev 000018b4  00000000  00000000  00026a9a  2**0
                  CONTENTS, READONLY, DEBUGGING, OCTETS
 14 .debug_aranges 00000798  00000000  00000000  00028350  2**3
                  CONTENTS, READONLY, DEBUGGING, OCTETS
 15 .debug_ranges 000006f0  00000000  00000000  00028ae8  2**3
                  CONTENTS, READONLY, DEBUGGING, OCTETS
 16 .debug_macro  00017986  00000000  00000000  000291d8  2**0
                  CONTENTS, READONLY, DEBUGGING, OCTETS
 17 .debug_line   00007f3b  00000000  00000000  00040b5e  2**0
                  CONTENTS, READONLY, DEBUGGING, OCTETS
 18 .debug_str    00083942  00000000  00000000  00048a99  2**0
                  CONTENTS, READONLY, DEBUGGING, OCTETS
 19 .comment      00000050  00000000  00000000  000cc3db  2**0
                  CONTENTS, READONLY
 20 .debug_frame  00002ad4  00000000  00000000  000cc42c  2**2
                  CONTENTS, READONLY, DEBUGGING, OCTETS

Disassembly of section .text:

0800010c <__do_global_dtors_aux>:
 800010c:	b510      	push	{r4, lr}
 800010e:	4c05      	ldr	r4, [pc, #20]	; (8000124 <__do_global_dtors_aux+0x18>)
 8000110:	7823      	ldrb	r3, [r4, #0]
 8000112:	b933      	cbnz	r3, 8000122 <__do_global_dtors_aux+0x16>
 8000114:	4b04      	ldr	r3, [pc, #16]	; (8000128 <__do_global_dtors_aux+0x1c>)
 8000116:	b113      	cbz	r3, 800011e <__do_global_dtors_aux+0x12>
 8000118:	4804      	ldr	r0, [pc, #16]	; (800012c <__do_global_dtors_aux+0x20>)
 800011a:	f3af 8000 	nop.w
 800011e:	2301      	movs	r3, #1
 8000120:	7023      	strb	r3, [r4, #0]
 8000122:	bd10      	pop	{r4, pc}
 8000124:	2000007c 	.word	0x2000007c
 8000128:	00000000 	.word	0x00000000
 800012c:	08004df4 	.word	0x08004df4

08000130 <frame_dummy>:
 8000130:	b508      	push	{r3, lr}
 8000132:	4b03      	ldr	r3, [pc, #12]	; (8000140 <frame_dummy+0x10>)
 8000134:	b11b      	cbz	r3, 800013e <frame_dummy+0xe>
 8000136:	4903      	ldr	r1, [pc, #12]	; (8000144 <frame_dummy+0x14>)
 8000138:	4803      	ldr	r0, [pc, #12]	; (8000148 <frame_dummy+0x18>)
 800013a:	f3af 8000 	nop.w
 800013e:	bd08      	pop	{r3, pc}
 8000140:	00000000 	.word	0x00000000
 8000144:	20000080 	.word	0x20000080
 8000148:	08004df4 	.word	0x08004df4

0800014c <__aeabi_fmul>:
 800014c:	f04f 0cff 	mov.w	ip, #255	; 0xff
 8000150:	ea1c 52d0 	ands.w	r2, ip, r0, lsr #23
 8000154:	bf1e      	ittt	ne
 8000156:	ea1c 53d1 	andsne.w	r3, ip, r1, lsr #23
 800015a:	ea92 0f0c 	teqne	r2, ip
 800015e:	ea93 0f0c 	teqne	r3, ip
 8000162:	d06f      	beq.n	8000244 <__aeabi_fmul+0xf8>
 8000164:	441a      	add	r2, r3
 8000166:	ea80 0c01 	eor.w	ip, r0, r1
 800016a:	0240      	lsls	r0, r0, #9
 800016c:	bf18      	it	ne
 800016e:	ea5f 2141 	movsne.w	r1, r1, lsl #9
 8000172:	d01e      	beq.n	80001b2 <__aeabi_fmul+0x66>
 8000174:	f04f 6300 	mov.w	r3, #134217728	; 0x8000000
 8000178:	ea43 1050 	orr.w	r0, r3, r0, lsr #5
 800017c:	ea43 1151 	orr.w	r1, r3, r1, lsr #5
 8000180:	fba0 3101 	umull	r3, r1, r0, r1
 8000184:	f00c 4000 	and.w	r0, ip, #2147483648	; 0x80000000
 8000188:	f5b1 0f00 	cmp.w	r1, #8388608	; 0x800000
 800018c:	bf3e      	ittt	cc
 800018e:	0049      	lslcc	r1, r1, #1
 8000190:	ea41 71d3 	orrcc.w	r1, r1, r3, lsr #31
 8000194:	005b      	lslcc	r3, r3, #1
 8000196:	ea40 0001 	orr.w	r0, r0, r1
 800019a:	f162 027f 	sbc.w	r2, r2, #127	; 0x7f
 800019e:	2afd      	cmp	r2, #253	; 0xfd
 80001a0:	d81d      	bhi.n	80001de <__aeabi_fmul+0x92>
 80001a2:	f1b3 4f00 	cmp.w	r3, #2147483648	; 0x80000000
 80001a6:	eb40 50c2 	adc.w	r0, r0, r2, lsl #23
 80001aa:	bf08      	it	eq
 80001ac:	f020 0001 	biceq.w	r0, r0, #1
 80001b0:	4770      	bx	lr
 80001b2:	f090 0f00 	teq	r0, #0
 80001b6:	f00c 4c00 	and.w	ip, ip, #2147483648	; 0x80000000
 80001ba:	bf08      	it	eq
 80001bc:	0249      	lsleq	r1, r1, #9
 80001be:	ea4c 2050 	orr.w	r0, ip, r0, lsr #9
 80001c2:	ea40 2051 	orr.w	r0, r0, r1, lsr #9
 80001c6:	3a7f      	subs	r2, #127	; 0x7f
 80001c8:	bfc2      	ittt	gt
 80001ca:	f1d2 03ff 	rsbsgt	r3, r2, #255	; 0xff
 80001ce:	ea40 50c2 	orrgt.w	r0, r0, r2, lsl #23
 80001d2:	4770      	bxgt	lr
 80001d4:	f440 0000 	orr.w	r0, r0, #8388608	; 0x800000
 80001d8:	f04f 0300 	mov.w	r3, #0
 80001dc:	3a01      	subs	r2, #1
 80001de:	dc5d      	bgt.n	800029c <__aeabi_fmul+0x150>
 80001e0:	f112 0f19 	cmn.w	r2, #25
 80001e4:	bfdc      	itt	le
 80001e6:	f000 4000 	andle.w	r0, r0, #2147483648	; 0x80000000
 80001ea:	4770      	bxle	lr
 80001ec:	f1c2 0200 	rsb	r2, r2, #0
 80001f0:	0041      	lsls	r1, r0, #1
 80001f2:	fa21 f102 	lsr.w	r1, r1, r2
 80001f6:	f1c2 0220 	rsb	r2, r2, #32
 80001fa:	fa00 fc02 	lsl.w	ip, r0, r2
 80001fe:	ea5f 0031 	movs.w	r0, r1, rrx
 8000202:	f140 0000 	adc.w	r0, r0, #0
 8000206:	ea53 034c 	orrs.w	r3, r3, ip, lsl #1
 800020a:	bf08      	it	eq
 800020c:	ea20 70dc 	biceq.w	r0, r0, ip, lsr #31
 8000210:	4770      	bx	lr
 8000212:	f092 0f00 	teq	r2, #0
 8000216:	f000 4c00 	and.w	ip, r0, #2147483648	; 0x80000000
 800021a:	bf02      	ittt	eq
 800021c:	0040      	lsleq	r0, r0, #1
 800021e:	f410 0f00 	tsteq.w	r0, #8388608	; 0x800000
 8000222:	3a01      	subeq	r2, #1
 8000224:	d0f9      	beq.n	800021a <__aeabi_fmul+0xce>
 8000226:	ea40 000c 	orr.w	r0, r0, ip
 800022a:	f093 0f00 	teq	r3, #0
 800022e:	f001 4c00 	and.w	ip, r1, #2147483648	; 0x80000000
 8000232:	bf02      	ittt	eq
 8000234:	0049      	lsleq	r1, r1, #1
 8000236:	f411 0f00 	tsteq.w	r1, #8388608	; 0x800000
 800023a:	3b01      	subeq	r3, #1
 800023c:	d0f9      	beq.n	8000232 <__aeabi_fmul+0xe6>
 800023e:	ea41 010c 	orr.w	r1, r1, ip
 8000242:	e78f      	b.n	8000164 <__aeabi_fmul+0x18>
 8000244:	ea0c 53d1 	and.w	r3, ip, r1, lsr #23
 8000248:	ea92 0f0c 	teq	r2, ip
 800024c:	bf18      	it	ne
 800024e:	ea93 0f0c 	teqne	r3, ip
 8000252:	d00a      	beq.n	800026a <__aeabi_fmul+0x11e>
 8000254:	f030 4c00 	bics.w	ip, r0, #2147483648	; 0x80000000
 8000258:	bf18      	it	ne
 800025a:	f031 4c00 	bicsne.w	ip, r1, #2147483648	; 0x80000000
 800025e:	d1d8      	bne.n	8000212 <__aeabi_fmul+0xc6>
 8000260:	ea80 0001 	eor.w	r0, r0, r1
 8000264:	f000 4000 	and.w	r0, r0, #2147483648	; 0x80000000
 8000268:	4770      	bx	lr
 800026a:	f090 0f00 	teq	r0, #0
 800026e:	bf17      	itett	ne
 8000270:	f090 4f00 	teqne	r0, #2147483648	; 0x80000000
 8000274:	4608      	moveq	r0, r1
 8000276:	f091 0f00 	teqne	r1, #0
 800027a:	f091 4f00 	teqne	r1, #2147483648	; 0x80000000
 800027e:	d014      	beq.n	80002aa <__aeabi_fmul+0x15e>
 8000280:	ea92 0f0c 	teq	r2, ip
 8000284:	d101      	bne.n	800028a <__aeabi_fmul+0x13e>
 8000286:	0242      	lsls	r2, r0, #9
 8000288:	d10f      	bne.n	80002aa <__aeabi_fmul+0x15e>
 800028a:	ea93 0f0c 	teq	r3, ip
 800028e:	d103      	bne.n	8000298 <__aeabi_fmul+0x14c>
 8000290:	024b      	lsls	r3, r1, #9
 8000292:	bf18      	it	ne
 8000294:	4608      	movne	r0, r1
 8000296:	d108      	bne.n	80002aa <__aeabi_fmul+0x15e>
 8000298:	ea80 0001 	eor.w	r0, r0, r1
 800029c:	f000 4000 	and.w	r0, r0, #2147483648	; 0x80000000
 80002a0:	f040 40fe 	orr.w	r0, r0, #2130706432	; 0x7f000000
 80002a4:	f440 0000 	orr.w	r0, r0, #8388608	; 0x800000
 80002a8:	4770      	bx	lr
 80002aa:	f040 40fe 	orr.w	r0, r0, #2130706432	; 0x7f000000
 80002ae:	f440 0040 	orr.w	r0, r0, #12582912	; 0xc00000
 80002b2:	4770      	bx	lr

080002b4 <__aeabi_drsub>:
 80002b4:	f081 4100 	eor.w	r1, r1, #2147483648	; 0x80000000
 80002b8:	e002      	b.n	80002c0 <__adddf3>
 80002ba:	bf00      	nop

080002bc <__aeabi_dsub>:
 80002bc:	f083 4300 	eor.w	r3, r3, #2147483648	; 0x80000000

080002c0 <__adddf3>:
 80002c0:	b530      	push	{r4, r5, lr}
 80002c2:	ea4f 0441 	mov.w	r4, r1, lsl #1
 80002c6:	ea4f 0543 	mov.w	r5, r3, lsl #1
 80002ca:	ea94 0f05 	teq	r4, r5
 80002ce:	bf08      	it	eq
 80002d0:	ea90 0f02 	teqeq	r0, r2
 80002d4:	bf1f      	itttt	ne
 80002d6:	ea54 0c00 	orrsne.w	ip, r4, r0
 80002da:	ea55 0c02 	orrsne.w	ip, r5, r2
 80002de:	ea7f 5c64 	mvnsne.w	ip, r4, asr #21
 80002e2:	ea7f 5c65 	mvnsne.w	ip, r5, asr #21
 80002e6:	f000 80e2 	beq.w	80004ae <__adddf3+0x1ee>
 80002ea:	ea4f 5454 	mov.w	r4, r4, lsr #21
 80002ee:	ebd4 5555 	rsbs	r5, r4, r5, lsr #21
 80002f2:	bfb8      	it	lt
 80002f4:	426d      	neglt	r5, r5
 80002f6:	dd0c      	ble.n	8000312 <__adddf3+0x52>
 80002f8:	442c      	add	r4, r5
 80002fa:	ea80 0202 	eor.w	r2, r0, r2
 80002fe:	ea81 0303 	eor.w	r3, r1, r3
 8000302:	ea82 0000 	eor.w	r0, r2, r0
 8000306:	ea83 0101 	eor.w	r1, r3, r1
 800030a:	ea80 0202 	eor.w	r2, r0, r2
 800030e:	ea81 0303 	eor.w	r3, r1, r3
 8000312:	2d36      	cmp	r5, #54	; 0x36
 8000314:	bf88      	it	hi
 8000316:	bd30      	pophi	{r4, r5, pc}
 8000318:	f011 4f00 	tst.w	r1, #2147483648	; 0x80000000
 800031c:	ea4f 3101 	mov.w	r1, r1, lsl #12
 8000320:	f44f 1c80 	mov.w	ip, #1048576	; 0x100000
 8000324:	ea4c 3111 	orr.w	r1, ip, r1, lsr #12
 8000328:	d002      	beq.n	8000330 <__adddf3+0x70>
 800032a:	4240      	negs	r0, r0
 800032c:	eb61 0141 	sbc.w	r1, r1, r1, lsl #1
 8000330:	f013 4f00 	tst.w	r3, #2147483648	; 0x80000000
 8000334:	ea4f 3303 	mov.w	r3, r3, lsl #12
 8000338:	ea4c 3313 	orr.w	r3, ip, r3, lsr #12
 800033c:	d002      	beq.n	8000344 <__adddf3+0x84>
 800033e:	4252      	negs	r2, r2
 8000340:	eb63 0343 	sbc.w	r3, r3, r3, lsl #1
 8000344:	ea94 0f05 	teq	r4, r5
 8000348:	f000 80a7 	beq.w	800049a <__adddf3+0x1da>
 800034c:	f1a4 0401 	sub.w	r4, r4, #1
 8000350:	f1d5 0e20 	rsbs	lr, r5, #32
 8000354:	db0d      	blt.n	8000372 <__adddf3+0xb2>
 8000356:	fa02 fc0e 	lsl.w	ip, r2, lr
 800035a:	fa22 f205 	lsr.w	r2, r2, r5
 800035e:	1880      	adds	r0, r0, r2
 8000360:	f141 0100 	adc.w	r1, r1, #0
 8000364:	fa03 f20e 	lsl.w	r2, r3, lr
 8000368:	1880      	adds	r0, r0, r2
 800036a:	fa43 f305 	asr.w	r3, r3, r5
 800036e:	4159      	adcs	r1, r3
 8000370:	e00e      	b.n	8000390 <__adddf3+0xd0>
 8000372:	f1a5 0520 	sub.w	r5, r5, #32
 8000376:	f10e 0e20 	add.w	lr, lr, #32
 800037a:	2a01      	cmp	r2, #1
 800037c:	fa03 fc0e 	lsl.w	ip, r3, lr
 8000380:	bf28      	it	cs
 8000382:	f04c 0c02 	orrcs.w	ip, ip, #2
 8000386:	fa43 f305 	asr.w	r3, r3, r5
 800038a:	18c0      	adds	r0, r0, r3
 800038c:	eb51 71e3 	adcs.w	r1, r1, r3, asr #31
 8000390:	f001 4500 	and.w	r5, r1, #2147483648	; 0x80000000
 8000394:	d507      	bpl.n	80003a6 <__adddf3+0xe6>
 8000396:	f04f 0e00 	mov.w	lr, #0
 800039a:	f1dc 0c00 	rsbs	ip, ip, #0
 800039e:	eb7e 0000 	sbcs.w	r0, lr, r0
 80003a2:	eb6e 0101 	sbc.w	r1, lr, r1
 80003a6:	f5b1 1f80 	cmp.w	r1, #1048576	; 0x100000
 80003aa:	d31b      	bcc.n	80003e4 <__adddf3+0x124>
 80003ac:	f5b1 1f00 	cmp.w	r1, #2097152	; 0x200000
 80003b0:	d30c      	bcc.n	80003cc <__adddf3+0x10c>
 80003b2:	0849      	lsrs	r1, r1, #1
 80003b4:	ea5f 0030 	movs.w	r0, r0, rrx
 80003b8:	ea4f 0c3c 	mov.w	ip, ip, rrx
 80003bc:	f104 0401 	add.w	r4, r4, #1
 80003c0:	ea4f 5244 	mov.w	r2, r4, lsl #21
 80003c4:	f512 0f80 	cmn.w	r2, #4194304	; 0x400000
 80003c8:	f080 809a 	bcs.w	8000500 <__adddf3+0x240>
 80003cc:	f1bc 4f00 	cmp.w	ip, #2147483648	; 0x80000000
 80003d0:	bf08      	it	eq
 80003d2:	ea5f 0c50 	movseq.w	ip, r0, lsr #1
 80003d6:	f150 0000 	adcs.w	r0, r0, #0
 80003da:	eb41 5104 	adc.w	r1, r1, r4, lsl #20
 80003de:	ea41 0105 	orr.w	r1, r1, r5
 80003e2:	bd30      	pop	{r4, r5, pc}
 80003e4:	ea5f 0c4c 	movs.w	ip, ip, lsl #1
 80003e8:	4140      	adcs	r0, r0
 80003ea:	eb41 0101 	adc.w	r1, r1, r1
 80003ee:	3c01      	subs	r4, #1
 80003f0:	bf28      	it	cs
 80003f2:	f5b1 1f80 	cmpcs.w	r1, #1048576	; 0x100000
 80003f6:	d2e9      	bcs.n	80003cc <__adddf3+0x10c>
 80003f8:	f091 0f00 	teq	r1, #0
 80003fc:	bf04      	itt	eq
 80003fe:	4601      	moveq	r1, r0
 8000400:	2000      	moveq	r0, #0
 8000402:	fab1 f381 	clz	r3, r1
 8000406:	bf08      	it	eq
 8000408:	3320      	addeq	r3, #32
 800040a:	f1a3 030b 	sub.w	r3, r3, #11
 800040e:	f1b3 0220 	subs.w	r2, r3, #32
 8000412:	da0c      	bge.n	800042e <__adddf3+0x16e>
 8000414:	320c      	adds	r2, #12
 8000416:	dd08      	ble.n	800042a <__adddf3+0x16a>
 8000418:	f102 0c14 	add.w	ip, r2, #20
 800041c:	f1c2 020c 	rsb	r2, r2, #12
 8000420:	fa01 f00c 	lsl.w	r0, r1, ip
 8000424:	fa21 f102 	lsr.w	r1, r1, r2
 8000428:	e00c      	b.n	8000444 <__adddf3+0x184>
 800042a:	f102 0214 	add.w	r2, r2, #20
 800042e:	bfd8      	it	le
 8000430:	f1c2 0c20 	rsble	ip, r2, #32
 8000434:	fa01 f102 	lsl.w	r1, r1, r2
 8000438:	fa20 fc0c 	lsr.w	ip, r0, ip
 800043c:	bfdc      	itt	le
 800043e:	ea41 010c 	orrle.w	r1, r1, ip
 8000442:	4090      	lslle	r0, r2
 8000444:	1ae4      	subs	r4, r4, r3
 8000446:	bfa2      	ittt	ge
 8000448:	eb01 5104 	addge.w	r1, r1, r4, lsl #20
 800044c:	4329      	orrge	r1, r5
 800044e:	bd30      	popge	{r4, r5, pc}
 8000450:	ea6f 0404 	mvn.w	r4, r4
 8000454:	3c1f      	subs	r4, #31
 8000456:	da1c      	bge.n	8000492 <__adddf3+0x1d2>
 8000458:	340c      	adds	r4, #12
 800045a:	dc0e      	bgt.n	800047a <__adddf3+0x1ba>
 800045c:	f104 0414 	add.w	r4, r4, #20
 8000460:	f1c4 0220 	rsb	r2, r4, #32
 8000464:	fa20 f004 	lsr.w	r0, r0, r4
 8000468:	fa01 f302 	lsl.w	r3, r1, r2
 800046c:	ea40 0003 	orr.w	r0, r0, r3
 8000470:	fa21 f304 	lsr.w	r3, r1, r4
 8000474:	ea45 0103 	orr.w	r1, r5, r3
 8000478:	bd30      	pop	{r4, r5, pc}
 800047a:	f1c4 040c 	rsb	r4, r4, #12
 800047e:	f1c4 0220 	rsb	r2, r4, #32
 8000482:	fa20 f002 	lsr.w	r0, r0, r2
 8000486:	fa01 f304 	lsl.w	r3, r1, r4
 800048a:	ea40 0003 	orr.w	r0, r0, r3
 800048e:	4629      	mov	r1, r5
 8000490:	bd30      	pop	{r4, r5, pc}
 8000492:	fa21 f004 	lsr.w	r0, r1, r4
 8000496:	4629      	mov	r1, r5
 8000498:	bd30      	pop	{r4, r5, pc}
 800049a:	f094 0f00 	teq	r4, #0
 800049e:	f483 1380 	eor.w	r3, r3, #1048576	; 0x100000
 80004a2:	bf06      	itte	eq
 80004a4:	f481 1180 	eoreq.w	r1, r1, #1048576	; 0x100000
 80004a8:	3401      	addeq	r4, #1
 80004aa:	3d01      	subne	r5, #1
 80004ac:	e74e      	b.n	800034c <__adddf3+0x8c>
 80004ae:	ea7f 5c64 	mvns.w	ip, r4, asr #21
 80004b2:	bf18      	it	ne
 80004b4:	ea7f 5c65 	mvnsne.w	ip, r5, asr #21
 80004b8:	d029      	beq.n	800050e <__adddf3+0x24e>
 80004ba:	ea94 0f05 	teq	r4, r5
 80004be:	bf08      	it	eq
 80004c0:	ea90 0f02 	teqeq	r0, r2
 80004c4:	d005      	beq.n	80004d2 <__adddf3+0x212>
 80004c6:	ea54 0c00 	orrs.w	ip, r4, r0
 80004ca:	bf04      	itt	eq
 80004cc:	4619      	moveq	r1, r3
 80004ce:	4610      	moveq	r0, r2
 80004d0:	bd30      	pop	{r4, r5, pc}
 80004d2:	ea91 0f03 	teq	r1, r3
 80004d6:	bf1e      	ittt	ne
 80004d8:	2100      	movne	r1, #0
 80004da:	2000      	movne	r0, #0
 80004dc:	bd30      	popne	{r4, r5, pc}
 80004de:	ea5f 5c54 	movs.w	ip, r4, lsr #21
 80004e2:	d105      	bne.n	80004f0 <__adddf3+0x230>
 80004e4:	0040      	lsls	r0, r0, #1
 80004e6:	4149      	adcs	r1, r1
 80004e8:	bf28      	it	cs
 80004ea:	f041 4100 	orrcs.w	r1, r1, #2147483648	; 0x80000000
 80004ee:	bd30      	pop	{r4, r5, pc}
 80004f0:	f514 0480 	adds.w	r4, r4, #4194304	; 0x400000
 80004f4:	bf3c      	itt	cc
 80004f6:	f501 1180 	addcc.w	r1, r1, #1048576	; 0x100000
 80004fa:	bd30      	popcc	{r4, r5, pc}
 80004fc:	f001 4500 	and.w	r5, r1, #2147483648	; 0x80000000
 8000500:	f045 41fe 	orr.w	r1, r5, #2130706432	; 0x7f000000
 8000504:	f441 0170 	orr.w	r1, r1, #15728640	; 0xf00000
 8000508:	f04f 0000 	mov.w	r0, #0
 800050c:	bd30      	pop	{r4, r5, pc}
 800050e:	ea7f 5c64 	mvns.w	ip, r4, asr #21
 8000512:	bf1a      	itte	ne
 8000514:	4619      	movne	r1, r3
 8000516:	4610      	movne	r0, r2
 8000518:	ea7f 5c65 	mvnseq.w	ip, r5, asr #21
 800051c:	bf1c      	itt	ne
 800051e:	460b      	movne	r3, r1
 8000520:	4602      	movne	r2, r0
 8000522:	ea50 3401 	orrs.w	r4, r0, r1, lsl #12
 8000526:	bf06      	itte	eq
 8000528:	ea52 3503 	orrseq.w	r5, r2, r3, lsl #12
 800052c:	ea91 0f03 	teqeq	r1, r3
 8000530:	f441 2100 	orrne.w	r1, r1, #524288	; 0x80000
 8000534:	bd30      	pop	{r4, r5, pc}
 8000536:	bf00      	nop

08000538 <__aeabi_ui2d>:
 8000538:	f090 0f00 	teq	r0, #0
 800053c:	bf04      	itt	eq
 800053e:	2100      	moveq	r1, #0
 8000540:	4770      	bxeq	lr
 8000542:	b530      	push	{r4, r5, lr}
 8000544:	f44f 6480 	mov.w	r4, #1024	; 0x400
 8000548:	f104 0432 	add.w	r4, r4, #50	; 0x32
 800054c:	f04f 0500 	mov.w	r5, #0
 8000550:	f04f 0100 	mov.w	r1, #0
 8000554:	e750      	b.n	80003f8 <__adddf3+0x138>
 8000556:	bf00      	nop

08000558 <__aeabi_i2d>:
 8000558:	f090 0f00 	teq	r0, #0
 800055c:	bf04      	itt	eq
 800055e:	2100      	moveq	r1, #0
 8000560:	4770      	bxeq	lr
 8000562:	b530      	push	{r4, r5, lr}
 8000564:	f44f 6480 	mov.w	r4, #1024	; 0x400
 8000568:	f104 0432 	add.w	r4, r4, #50	; 0x32
 800056c:	f010 4500 	ands.w	r5, r0, #2147483648	; 0x80000000
 8000570:	bf48      	it	mi
 8000572:	4240      	negmi	r0, r0
 8000574:	f04f 0100 	mov.w	r1, #0
 8000578:	e73e      	b.n	80003f8 <__adddf3+0x138>
 800057a:	bf00      	nop

0800057c <__aeabi_f2d>:
 800057c:	0042      	lsls	r2, r0, #1
 800057e:	ea4f 01e2 	mov.w	r1, r2, asr #3
 8000582:	ea4f 0131 	mov.w	r1, r1, rrx
 8000586:	ea4f 7002 	mov.w	r0, r2, lsl #28
 800058a:	bf1f      	itttt	ne
 800058c:	f012 437f 	andsne.w	r3, r2, #4278190080	; 0xff000000
 8000590:	f093 4f7f 	teqne	r3, #4278190080	; 0xff000000
 8000594:	f081 5160 	eorne.w	r1, r1, #939524096	; 0x38000000
 8000598:	4770      	bxne	lr
 800059a:	f032 427f 	bics.w	r2, r2, #4278190080	; 0xff000000
 800059e:	bf08      	it	eq
 80005a0:	4770      	bxeq	lr
 80005a2:	f093 4f7f 	teq	r3, #4278190080	; 0xff000000
 80005a6:	bf04      	itt	eq
 80005a8:	f441 2100 	orreq.w	r1, r1, #524288	; 0x80000
 80005ac:	4770      	bxeq	lr
 80005ae:	b530      	push	{r4, r5, lr}
 80005b0:	f44f 7460 	mov.w	r4, #896	; 0x380
 80005b4:	f001 4500 	and.w	r5, r1, #2147483648	; 0x80000000
 80005b8:	f021 4100 	bic.w	r1, r1, #2147483648	; 0x80000000
 80005bc:	e71c      	b.n	80003f8 <__adddf3+0x138>
 80005be:	bf00      	nop

080005c0 <__aeabi_ul2d>:
 80005c0:	ea50 0201 	orrs.w	r2, r0, r1
 80005c4:	bf08      	it	eq
 80005c6:	4770      	bxeq	lr
 80005c8:	b530      	push	{r4, r5, lr}
 80005ca:	f04f 0500 	mov.w	r5, #0
 80005ce:	e00a      	b.n	80005e6 <__aeabi_l2d+0x16>

080005d0 <__aeabi_l2d>:
 80005d0:	ea50 0201 	orrs.w	r2, r0, r1
 80005d4:	bf08      	it	eq
 80005d6:	4770      	bxeq	lr
 80005d8:	b530      	push	{r4, r5, lr}
 80005da:	f011 4500 	ands.w	r5, r1, #2147483648	; 0x80000000
 80005de:	d502      	bpl.n	80005e6 <__aeabi_l2d+0x16>
 80005e0:	4240      	negs	r0, r0
 80005e2:	eb61 0141 	sbc.w	r1, r1, r1, lsl #1
 80005e6:	f44f 6480 	mov.w	r4, #1024	; 0x400
 80005ea:	f104 0432 	add.w	r4, r4, #50	; 0x32
 80005ee:	ea5f 5c91 	movs.w	ip, r1, lsr #22
 80005f2:	f43f aed8 	beq.w	80003a6 <__adddf3+0xe6>
 80005f6:	f04f 0203 	mov.w	r2, #3
 80005fa:	ea5f 0cdc 	movs.w	ip, ip, lsr #3
 80005fe:	bf18      	it	ne
 8000600:	3203      	addne	r2, #3
 8000602:	ea5f 0cdc 	movs.w	ip, ip, lsr #3
 8000606:	bf18      	it	ne
 8000608:	3203      	addne	r2, #3
 800060a:	eb02 02dc 	add.w	r2, r2, ip, lsr #3
 800060e:	f1c2 0320 	rsb	r3, r2, #32
 8000612:	fa00 fc03 	lsl.w	ip, r0, r3
 8000616:	fa20 f002 	lsr.w	r0, r0, r2
 800061a:	fa01 fe03 	lsl.w	lr, r1, r3
 800061e:	ea40 000e 	orr.w	r0, r0, lr
 8000622:	fa21 f102 	lsr.w	r1, r1, r2
 8000626:	4414      	add	r4, r2
 8000628:	e6bd      	b.n	80003a6 <__adddf3+0xe6>
 800062a:	bf00      	nop

0800062c <__aeabi_dmul>:
 800062c:	b570      	push	{r4, r5, r6, lr}
 800062e:	f04f 0cff 	mov.w	ip, #255	; 0xff
 8000632:	f44c 6ce0 	orr.w	ip, ip, #1792	; 0x700
 8000636:	ea1c 5411 	ands.w	r4, ip, r1, lsr #20
 800063a:	bf1d      	ittte	ne
 800063c:	ea1c 5513 	andsne.w	r5, ip, r3, lsr #20
 8000640:	ea94 0f0c 	teqne	r4, ip
 8000644:	ea95 0f0c 	teqne	r5, ip
 8000648:	f000 f8de 	bleq	8000808 <__aeabi_dmul+0x1dc>
 800064c:	442c      	add	r4, r5
 800064e:	ea81 0603 	eor.w	r6, r1, r3
 8000652:	ea21 514c 	bic.w	r1, r1, ip, lsl #21
 8000656:	ea23 534c 	bic.w	r3, r3, ip, lsl #21
 800065a:	ea50 3501 	orrs.w	r5, r0, r1, lsl #12
 800065e:	bf18      	it	ne
 8000660:	ea52 3503 	orrsne.w	r5, r2, r3, lsl #12
 8000664:	f441 1180 	orr.w	r1, r1, #1048576	; 0x100000
 8000668:	f443 1380 	orr.w	r3, r3, #1048576	; 0x100000
 800066c:	d038      	beq.n	80006e0 <__aeabi_dmul+0xb4>
 800066e:	fba0 ce02 	umull	ip, lr, r0, r2
 8000672:	f04f 0500 	mov.w	r5, #0
 8000676:	fbe1 e502 	umlal	lr, r5, r1, r2
 800067a:	f006 4200 	and.w	r2, r6, #2147483648	; 0x80000000
 800067e:	fbe0 e503 	umlal	lr, r5, r0, r3
 8000682:	f04f 0600 	mov.w	r6, #0
 8000686:	fbe1 5603 	umlal	r5, r6, r1, r3
 800068a:	f09c 0f00 	teq	ip, #0
 800068e:	bf18      	it	ne
 8000690:	f04e 0e01 	orrne.w	lr, lr, #1
 8000694:	f1a4 04ff 	sub.w	r4, r4, #255	; 0xff
 8000698:	f5b6 7f00 	cmp.w	r6, #512	; 0x200
 800069c:	f564 7440 	sbc.w	r4, r4, #768	; 0x300
 80006a0:	d204      	bcs.n	80006ac <__aeabi_dmul+0x80>
 80006a2:	ea5f 0e4e 	movs.w	lr, lr, lsl #1
 80006a6:	416d      	adcs	r5, r5
 80006a8:	eb46 0606 	adc.w	r6, r6, r6
 80006ac:	ea42 21c6 	orr.w	r1, r2, r6, lsl #11
 80006b0:	ea41 5155 	orr.w	r1, r1, r5, lsr #21
 80006b4:	ea4f 20c5 	mov.w	r0, r5, lsl #11
 80006b8:	ea40 505e 	orr.w	r0, r0, lr, lsr #21
 80006bc:	ea4f 2ece 	mov.w	lr, lr, lsl #11
 80006c0:	f1b4 0cfd 	subs.w	ip, r4, #253	; 0xfd
 80006c4:	bf88      	it	hi
 80006c6:	f5bc 6fe0 	cmphi.w	ip, #1792	; 0x700
 80006ca:	d81e      	bhi.n	800070a <__aeabi_dmul+0xde>
 80006cc:	f1be 4f00 	cmp.w	lr, #2147483648	; 0x80000000
 80006d0:	bf08      	it	eq
 80006d2:	ea5f 0e50 	movseq.w	lr, r0, lsr #1
 80006d6:	f150 0000 	adcs.w	r0, r0, #0
 80006da:	eb41 5104 	adc.w	r1, r1, r4, lsl #20
 80006de:	bd70      	pop	{r4, r5, r6, pc}
 80006e0:	f006 4600 	and.w	r6, r6, #2147483648	; 0x80000000
 80006e4:	ea46 0101 	orr.w	r1, r6, r1
 80006e8:	ea40 0002 	orr.w	r0, r0, r2
 80006ec:	ea81 0103 	eor.w	r1, r1, r3
 80006f0:	ebb4 045c 	subs.w	r4, r4, ip, lsr #1
 80006f4:	bfc2      	ittt	gt
 80006f6:	ebd4 050c 	rsbsgt	r5, r4, ip
 80006fa:	ea41 5104 	orrgt.w	r1, r1, r4, lsl #20
 80006fe:	bd70      	popgt	{r4, r5, r6, pc}
 8000700:	f441 1180 	orr.w	r1, r1, #1048576	; 0x100000
 8000704:	f04f 0e00 	mov.w	lr, #0
 8000708:	3c01      	subs	r4, #1
 800070a:	f300 80ab 	bgt.w	8000864 <__aeabi_dmul+0x238>
 800070e:	f114 0f36 	cmn.w	r4, #54	; 0x36
 8000712:	bfde      	ittt	le
 8000714:	2000      	movle	r0, #0
 8000716:	f001 4100 	andle.w	r1, r1, #2147483648	; 0x80000000
 800071a:	bd70      	pople	{r4, r5, r6, pc}
 800071c:	f1c4 0400 	rsb	r4, r4, #0
 8000720:	3c20      	subs	r4, #32
 8000722:	da35      	bge.n	8000790 <__aeabi_dmul+0x164>
 8000724:	340c      	adds	r4, #12
 8000726:	dc1b      	bgt.n	8000760 <__aeabi_dmul+0x134>
 8000728:	f104 0414 	add.w	r4, r4, #20
 800072c:	f1c4 0520 	rsb	r5, r4, #32
 8000730:	fa00 f305 	lsl.w	r3, r0, r5
 8000734:	fa20 f004 	lsr.w	r0, r0, r4
 8000738:	fa01 f205 	lsl.w	r2, r1, r5
 800073c:	ea40 0002 	orr.w	r0, r0, r2
 8000740:	f001 4200 	and.w	r2, r1, #2147483648	; 0x80000000
 8000744:	f021 4100 	bic.w	r1, r1, #2147483648	; 0x80000000
 8000748:	eb10 70d3 	adds.w	r0, r0, r3, lsr #31
 800074c:	fa21 f604 	lsr.w	r6, r1, r4
 8000750:	eb42 0106 	adc.w	r1, r2, r6
 8000754:	ea5e 0e43 	orrs.w	lr, lr, r3, lsl #1
 8000758:	bf08      	it	eq
 800075a:	ea20 70d3 	biceq.w	r0, r0, r3, lsr #31
 800075e:	bd70      	pop	{r4, r5, r6, pc}
 8000760:	f1c4 040c 	rsb	r4, r4, #12
 8000764:	f1c4 0520 	rsb	r5, r4, #32
 8000768:	fa00 f304 	lsl.w	r3, r0, r4
 800076c:	fa20 f005 	lsr.w	r0, r0, r5
 8000770:	fa01 f204 	lsl.w	r2, r1, r4
 8000774:	ea40 0002 	orr.w	r0, r0, r2
 8000778:	f001 4100 	and.w	r1, r1, #2147483648	; 0x80000000
 800077c:	eb10 70d3 	adds.w	r0, r0, r3, lsr #31
 8000780:	f141 0100 	adc.w	r1, r1, #0
 8000784:	ea5e 0e43 	orrs.w	lr, lr, r3, lsl #1
 8000788:	bf08      	it	eq
 800078a:	ea20 70d3 	biceq.w	r0, r0, r3, lsr #31
 800078e:	bd70      	pop	{r4, r5, r6, pc}
 8000790:	f1c4 0520 	rsb	r5, r4, #32
 8000794:	fa00 f205 	lsl.w	r2, r0, r5
 8000798:	ea4e 0e02 	orr.w	lr, lr, r2
 800079c:	fa20 f304 	lsr.w	r3, r0, r4
 80007a0:	fa01 f205 	lsl.w	r2, r1, r5
 80007a4:	ea43 0302 	orr.w	r3, r3, r2
 80007a8:	fa21 f004 	lsr.w	r0, r1, r4
 80007ac:	f001 4100 	and.w	r1, r1, #2147483648	; 0x80000000
 80007b0:	fa21 f204 	lsr.w	r2, r1, r4
 80007b4:	ea20 0002 	bic.w	r0, r0, r2
 80007b8:	eb00 70d3 	add.w	r0, r0, r3, lsr #31
 80007bc:	ea5e 0e43 	orrs.w	lr, lr, r3, lsl #1
 80007c0:	bf08      	it	eq
 80007c2:	ea20 70d3 	biceq.w	r0, r0, r3, lsr #31
 80007c6:	bd70      	pop	{r4, r5, r6, pc}
 80007c8:	f094 0f00 	teq	r4, #0
 80007cc:	d10f      	bne.n	80007ee <__aeabi_dmul+0x1c2>
 80007ce:	f001 4600 	and.w	r6, r1, #2147483648	; 0x80000000
 80007d2:	0040      	lsls	r0, r0, #1
 80007d4:	eb41 0101 	adc.w	r1, r1, r1
 80007d8:	f411 1f80 	tst.w	r1, #1048576	; 0x100000
 80007dc:	bf08      	it	eq
 80007de:	3c01      	subeq	r4, #1
 80007e0:	d0f7      	beq.n	80007d2 <__aeabi_dmul+0x1a6>
 80007e2:	ea41 0106 	orr.w	r1, r1, r6
 80007e6:	f095 0f00 	teq	r5, #0
 80007ea:	bf18      	it	ne
 80007ec:	4770      	bxne	lr
 80007ee:	f003 4600 	and.w	r6, r3, #2147483648	; 0x80000000
 80007f2:	0052      	lsls	r2, r2, #1
 80007f4:	eb43 0303 	adc.w	r3, r3, r3
 80007f8:	f413 1f80 	tst.w	r3, #1048576	; 0x100000
 80007fc:	bf08      	it	eq
 80007fe:	3d01      	subeq	r5, #1
 8000800:	d0f7      	beq.n	80007f2 <__aeabi_dmul+0x1c6>
 8000802:	ea43 0306 	orr.w	r3, r3, r6
 8000806:	4770      	bx	lr
 8000808:	ea94 0f0c 	teq	r4, ip
 800080c:	ea0c 5513 	and.w	r5, ip, r3, lsr #20
 8000810:	bf18      	it	ne
 8000812:	ea95 0f0c 	teqne	r5, ip
 8000816:	d00c      	beq.n	8000832 <__aeabi_dmul+0x206>
 8000818:	ea50 0641 	orrs.w	r6, r0, r1, lsl #1
 800081c:	bf18      	it	ne
 800081e:	ea52 0643 	orrsne.w	r6, r2, r3, lsl #1
 8000822:	d1d1      	bne.n	80007c8 <__aeabi_dmul+0x19c>
 8000824:	ea81 0103 	eor.w	r1, r1, r3
 8000828:	f001 4100 	and.w	r1, r1, #2147483648	; 0x80000000
 800082c:	f04f 0000 	mov.w	r0, #0
 8000830:	bd70      	pop	{r4, r5, r6, pc}
 8000832:	ea50 0641 	orrs.w	r6, r0, r1, lsl #1
 8000836:	bf06      	itte	eq
 8000838:	4610      	moveq	r0, r2
 800083a:	4619      	moveq	r1, r3
 800083c:	ea52 0643 	orrsne.w	r6, r2, r3, lsl #1
 8000840:	d019      	beq.n	8000876 <__aeabi_dmul+0x24a>
 8000842:	ea94 0f0c 	teq	r4, ip
 8000846:	d102      	bne.n	800084e <__aeabi_dmul+0x222>
 8000848:	ea50 3601 	orrs.w	r6, r0, r1, lsl #12
 800084c:	d113      	bne.n	8000876 <__aeabi_dmul+0x24a>
 800084e:	ea95 0f0c 	teq	r5, ip
 8000852:	d105      	bne.n	8000860 <__aeabi_dmul+0x234>
 8000854:	ea52 3603 	orrs.w	r6, r2, r3, lsl #12
 8000858:	bf1c      	itt	ne
 800085a:	4610      	movne	r0, r2
 800085c:	4619      	movne	r1, r3
 800085e:	d10a      	bne.n	8000876 <__aeabi_dmul+0x24a>
 8000860:	ea81 0103 	eor.w	r1, r1, r3
 8000864:	f001 4100 	and.w	r1, r1, #2147483648	; 0x80000000
 8000868:	f041 41fe 	orr.w	r1, r1, #2130706432	; 0x7f000000
 800086c:	f441 0170 	orr.w	r1, r1, #15728640	; 0xf00000
 8000870:	f04f 0000 	mov.w	r0, #0
 8000874:	bd70      	pop	{r4, r5, r6, pc}
 8000876:	f041 41fe 	orr.w	r1, r1, #2130706432	; 0x7f000000
 800087a:	f441 0178 	orr.w	r1, r1, #16252928	; 0xf80000
 800087e:	bd70      	pop	{r4, r5, r6, pc}

08000880 <__aeabi_ddiv>:
 8000880:	b570      	push	{r4, r5, r6, lr}
 8000882:	f04f 0cff 	mov.w	ip, #255	; 0xff
 8000886:	f44c 6ce0 	orr.w	ip, ip, #1792	; 0x700
 800088a:	ea1c 5411 	ands.w	r4, ip, r1, lsr #20
 800088e:	bf1d      	ittte	ne
 8000890:	ea1c 5513 	andsne.w	r5, ip, r3, lsr #20
 8000894:	ea94 0f0c 	teqne	r4, ip
 8000898:	ea95 0f0c 	teqne	r5, ip
 800089c:	f000 f8a7 	bleq	80009ee <__aeabi_ddiv+0x16e>
 80008a0:	eba4 0405 	sub.w	r4, r4, r5
 80008a4:	ea81 0e03 	eor.w	lr, r1, r3
 80008a8:	ea52 3503 	orrs.w	r5, r2, r3, lsl #12
 80008ac:	ea4f 3101 	mov.w	r1, r1, lsl #12
 80008b0:	f000 8088 	beq.w	80009c4 <__aeabi_ddiv+0x144>
 80008b4:	ea4f 3303 	mov.w	r3, r3, lsl #12
 80008b8:	f04f 5580 	mov.w	r5, #268435456	; 0x10000000
 80008bc:	ea45 1313 	orr.w	r3, r5, r3, lsr #4
 80008c0:	ea43 6312 	orr.w	r3, r3, r2, lsr #24
 80008c4:	ea4f 2202 	mov.w	r2, r2, lsl #8
 80008c8:	ea45 1511 	orr.w	r5, r5, r1, lsr #4
 80008cc:	ea45 6510 	orr.w	r5, r5, r0, lsr #24
 80008d0:	ea4f 2600 	mov.w	r6, r0, lsl #8
 80008d4:	f00e 4100 	and.w	r1, lr, #2147483648	; 0x80000000
 80008d8:	429d      	cmp	r5, r3
 80008da:	bf08      	it	eq
 80008dc:	4296      	cmpeq	r6, r2
 80008de:	f144 04fd 	adc.w	r4, r4, #253	; 0xfd
 80008e2:	f504 7440 	add.w	r4, r4, #768	; 0x300
 80008e6:	d202      	bcs.n	80008ee <__aeabi_ddiv+0x6e>
 80008e8:	085b      	lsrs	r3, r3, #1
 80008ea:	ea4f 0232 	mov.w	r2, r2, rrx
 80008ee:	1ab6      	subs	r6, r6, r2
 80008f0:	eb65 0503 	sbc.w	r5, r5, r3
 80008f4:	085b      	lsrs	r3, r3, #1
 80008f6:	ea4f 0232 	mov.w	r2, r2, rrx
 80008fa:	f44f 1080 	mov.w	r0, #1048576	; 0x100000
 80008fe:	f44f 2c00 	mov.w	ip, #524288	; 0x80000
 8000902:	ebb6 0e02 	subs.w	lr, r6, r2
 8000906:	eb75 0e03 	sbcs.w	lr, r5, r3
 800090a:	bf22      	ittt	cs
 800090c:	1ab6      	subcs	r6, r6, r2
 800090e:	4675      	movcs	r5, lr
 8000910:	ea40 000c 	orrcs.w	r0, r0, ip
 8000914:	085b      	lsrs	r3, r3, #1
 8000916:	ea4f 0232 	mov.w	r2, r2, rrx
 800091a:	ebb6 0e02 	subs.w	lr, r6, r2
 800091e:	eb75 0e03 	sbcs.w	lr, r5, r3
 8000922:	bf22      	ittt	cs
 8000924:	1ab6      	subcs	r6, r6, r2
 8000926:	4675      	movcs	r5, lr
 8000928:	ea40 005c 	orrcs.w	r0, r0, ip, lsr #1
 800092c:	085b      	lsrs	r3, r3, #1
 800092e:	ea4f 0232 	mov.w	r2, r2, rrx
 8000932:	ebb6 0e02 	subs.w	lr, r6, r2
 8000936:	eb75 0e03 	sbcs.w	lr, r5, r3
 800093a:	bf22      	ittt	cs
 800093c:	1ab6      	subcs	r6, r6, r2
 800093e:	4675      	movcs	r5, lr
 8000940:	ea40 009c 	orrcs.w	r0, r0, ip, lsr #2
 8000944:	085b      	lsrs	r3, r3, #1
 8000946:	ea4f 0232 	mov.w	r2, r2, rrx
 800094a:	ebb6 0e02 	subs.w	lr, r6, r2
 800094e:	eb75 0e03 	sbcs.w	lr, r5, r3
 8000952:	bf22      	ittt	cs
 8000954:	1ab6      	subcs	r6, r6, r2
 8000956:	4675      	movcs	r5, lr
 8000958:	ea40 00dc 	orrcs.w	r0, r0, ip, lsr #3
 800095c:	ea55 0e06 	orrs.w	lr, r5, r6
 8000960:	d018      	beq.n	8000994 <__aeabi_ddiv+0x114>
 8000962:	ea4f 1505 	mov.w	r5, r5, lsl #4
 8000966:	ea45 7516 	orr.w	r5, r5, r6, lsr #28
 800096a:	ea4f 1606 	mov.w	r6, r6, lsl #4
 800096e:	ea4f 03c3 	mov.w	r3, r3, lsl #3
 8000972:	ea43 7352 	orr.w	r3, r3, r2, lsr #29
 8000976:	ea4f 02c2 	mov.w	r2, r2, lsl #3
 800097a:	ea5f 1c1c 	movs.w	ip, ip, lsr #4
 800097e:	d1c0      	bne.n	8000902 <__aeabi_ddiv+0x82>
 8000980:	f411 1f80 	tst.w	r1, #1048576	; 0x100000
 8000984:	d10b      	bne.n	800099e <__aeabi_ddiv+0x11e>
 8000986:	ea41 0100 	orr.w	r1, r1, r0
 800098a:	f04f 0000 	mov.w	r0, #0
 800098e:	f04f 4c00 	mov.w	ip, #2147483648	; 0x80000000
 8000992:	e7b6      	b.n	8000902 <__aeabi_ddiv+0x82>
 8000994:	f411 1f80 	tst.w	r1, #1048576	; 0x100000
 8000998:	bf04      	itt	eq
 800099a:	4301      	orreq	r1, r0
 800099c:	2000      	moveq	r0, #0
 800099e:	f1b4 0cfd 	subs.w	ip, r4, #253	; 0xfd
 80009a2:	bf88      	it	hi
 80009a4:	f5bc 6fe0 	cmphi.w	ip, #1792	; 0x700
 80009a8:	f63f aeaf 	bhi.w	800070a <__aeabi_dmul+0xde>
 80009ac:	ebb5 0c03 	subs.w	ip, r5, r3
 80009b0:	bf04      	itt	eq
 80009b2:	ebb6 0c02 	subseq.w	ip, r6, r2
 80009b6:	ea5f 0c50 	movseq.w	ip, r0, lsr #1
 80009ba:	f150 0000 	adcs.w	r0, r0, #0
 80009be:	eb41 5104 	adc.w	r1, r1, r4, lsl #20
 80009c2:	bd70      	pop	{r4, r5, r6, pc}
 80009c4:	f00e 4e00 	and.w	lr, lr, #2147483648	; 0x80000000
 80009c8:	ea4e 3111 	orr.w	r1, lr, r1, lsr #12
 80009cc:	eb14 045c 	adds.w	r4, r4, ip, lsr #1
 80009d0:	bfc2      	ittt	gt
 80009d2:	ebd4 050c 	rsbsgt	r5, r4, ip
 80009d6:	ea41 5104 	orrgt.w	r1, r1, r4, lsl #20
 80009da:	bd70      	popgt	{r4, r5, r6, pc}
 80009dc:	f441 1180 	orr.w	r1, r1, #1048576	; 0x100000
 80009e0:	f04f 0e00 	mov.w	lr, #0
 80009e4:	3c01      	subs	r4, #1
 80009e6:	e690      	b.n	800070a <__aeabi_dmul+0xde>
 80009e8:	ea45 0e06 	orr.w	lr, r5, r6
 80009ec:	e68d      	b.n	800070a <__aeabi_dmul+0xde>
 80009ee:	ea0c 5513 	and.w	r5, ip, r3, lsr #20
 80009f2:	ea94 0f0c 	teq	r4, ip
 80009f6:	bf08      	it	eq
 80009f8:	ea95 0f0c 	teqeq	r5, ip
 80009fc:	f43f af3b 	beq.w	8000876 <__aeabi_dmul+0x24a>
 8000a00:	ea94 0f0c 	teq	r4, ip
 8000a04:	d10a      	bne.n	8000a1c <__aeabi_ddiv+0x19c>
 8000a06:	ea50 3401 	orrs.w	r4, r0, r1, lsl #12
 8000a0a:	f47f af34 	bne.w	8000876 <__aeabi_dmul+0x24a>
 8000a0e:	ea95 0f0c 	teq	r5, ip
 8000a12:	f47f af25 	bne.w	8000860 <__aeabi_dmul+0x234>
 8000a16:	4610      	mov	r0, r2
 8000a18:	4619      	mov	r1, r3
 8000a1a:	e72c      	b.n	8000876 <__aeabi_dmul+0x24a>
 8000a1c:	ea95 0f0c 	teq	r5, ip
 8000a20:	d106      	bne.n	8000a30 <__aeabi_ddiv+0x1b0>
 8000a22:	ea52 3503 	orrs.w	r5, r2, r3, lsl #12
 8000a26:	f43f aefd 	beq.w	8000824 <__aeabi_dmul+0x1f8>
 8000a2a:	4610      	mov	r0, r2
 8000a2c:	4619      	mov	r1, r3
 8000a2e:	e722      	b.n	8000876 <__aeabi_dmul+0x24a>
 8000a30:	ea50 0641 	orrs.w	r6, r0, r1, lsl #1
 8000a34:	bf18      	it	ne
 8000a36:	ea52 0643 	orrsne.w	r6, r2, r3, lsl #1
 8000a3a:	f47f aec5 	bne.w	80007c8 <__aeabi_dmul+0x19c>
 8000a3e:	ea50 0441 	orrs.w	r4, r0, r1, lsl #1
 8000a42:	f47f af0d 	bne.w	8000860 <__aeabi_dmul+0x234>
 8000a46:	ea52 0543 	orrs.w	r5, r2, r3, lsl #1
 8000a4a:	f47f aeeb 	bne.w	8000824 <__aeabi_dmul+0x1f8>
 8000a4e:	e712      	b.n	8000876 <__aeabi_dmul+0x24a>

08000a50 <__aeabi_d2f>:
 8000a50:	ea4f 0241 	mov.w	r2, r1, lsl #1
 8000a54:	f1b2 43e0 	subs.w	r3, r2, #1879048192	; 0x70000000
 8000a58:	bf24      	itt	cs
 8000a5a:	f5b3 1c00 	subscs.w	ip, r3, #2097152	; 0x200000
 8000a5e:	f1dc 5cfe 	rsbscs	ip, ip, #532676608	; 0x1fc00000
 8000a62:	d90d      	bls.n	8000a80 <__aeabi_d2f+0x30>
 8000a64:	f001 4c00 	and.w	ip, r1, #2147483648	; 0x80000000
 8000a68:	ea4f 02c0 	mov.w	r2, r0, lsl #3
 8000a6c:	ea4c 7050 	orr.w	r0, ip, r0, lsr #29
 8000a70:	f1b2 4f00 	cmp.w	r2, #2147483648	; 0x80000000
 8000a74:	eb40 0083 	adc.w	r0, r0, r3, lsl #2
 8000a78:	bf08      	it	eq
 8000a7a:	f020 0001 	biceq.w	r0, r0, #1
 8000a7e:	4770      	bx	lr
 8000a80:	f011 4f80 	tst.w	r1, #1073741824	; 0x40000000
 8000a84:	d121      	bne.n	8000aca <__aeabi_d2f+0x7a>
 8000a86:	f113 7238 	adds.w	r2, r3, #48234496	; 0x2e00000
 8000a8a:	bfbc      	itt	lt
 8000a8c:	f001 4000 	andlt.w	r0, r1, #2147483648	; 0x80000000
 8000a90:	4770      	bxlt	lr
 8000a92:	f441 1180 	orr.w	r1, r1, #1048576	; 0x100000
 8000a96:	ea4f 5252 	mov.w	r2, r2, lsr #21
 8000a9a:	f1c2 0218 	rsb	r2, r2, #24
 8000a9e:	f1c2 0c20 	rsb	ip, r2, #32
 8000aa2:	fa10 f30c 	lsls.w	r3, r0, ip
 8000aa6:	fa20 f002 	lsr.w	r0, r0, r2
 8000aaa:	bf18      	it	ne
 8000aac:	f040 0001 	orrne.w	r0, r0, #1
 8000ab0:	ea4f 23c1 	mov.w	r3, r1, lsl #11
 8000ab4:	ea4f 23d3 	mov.w	r3, r3, lsr #11
 8000ab8:	fa03 fc0c 	lsl.w	ip, r3, ip
 8000abc:	ea40 000c 	orr.w	r0, r0, ip
 8000ac0:	fa23 f302 	lsr.w	r3, r3, r2
 8000ac4:	ea4f 0343 	mov.w	r3, r3, lsl #1
 8000ac8:	e7cc      	b.n	8000a64 <__aeabi_d2f+0x14>
 8000aca:	ea7f 5362 	mvns.w	r3, r2, asr #21
 8000ace:	d107      	bne.n	8000ae0 <__aeabi_d2f+0x90>
 8000ad0:	ea50 3301 	orrs.w	r3, r0, r1, lsl #12
 8000ad4:	bf1e      	ittt	ne
 8000ad6:	f04f 40fe 	movne.w	r0, #2130706432	; 0x7f000000
 8000ada:	f440 0040 	orrne.w	r0, r0, #12582912	; 0xc00000
 8000ade:	4770      	bxne	lr
 8000ae0:	f001 4000 	and.w	r0, r1, #2147483648	; 0x80000000
 8000ae4:	f040 40fe 	orr.w	r0, r0, #2130706432	; 0x7f000000
 8000ae8:	f440 0000 	orr.w	r0, r0, #8388608	; 0x800000
 8000aec:	4770      	bx	lr
 8000aee:	bf00      	nop

08000af0 <__aeabi_frsub>:
 8000af0:	f080 4000 	eor.w	r0, r0, #2147483648	; 0x80000000
 8000af4:	e002      	b.n	8000afc <__addsf3>
 8000af6:	bf00      	nop

08000af8 <__aeabi_fsub>:
 8000af8:	f081 4100 	eor.w	r1, r1, #2147483648	; 0x80000000

08000afc <__addsf3>:
 8000afc:	0042      	lsls	r2, r0, #1
 8000afe:	bf1f      	itttt	ne
 8000b00:	ea5f 0341 	movsne.w	r3, r1, lsl #1
 8000b04:	ea92 0f03 	teqne	r2, r3
 8000b08:	ea7f 6c22 	mvnsne.w	ip, r2, asr #24
 8000b0c:	ea7f 6c23 	mvnsne.w	ip, r3, asr #24
 8000b10:	d06a      	beq.n	8000be8 <__addsf3+0xec>
 8000b12:	ea4f 6212 	mov.w	r2, r2, lsr #24
 8000b16:	ebd2 6313 	rsbs	r3, r2, r3, lsr #24
 8000b1a:	bfc1      	itttt	gt
 8000b1c:	18d2      	addgt	r2, r2, r3
 8000b1e:	4041      	eorgt	r1, r0
 8000b20:	4048      	eorgt	r0, r1
 8000b22:	4041      	eorgt	r1, r0
 8000b24:	bfb8      	it	lt
 8000b26:	425b      	neglt	r3, r3
 8000b28:	2b19      	cmp	r3, #25
 8000b2a:	bf88      	it	hi
 8000b2c:	4770      	bxhi	lr
 8000b2e:	f010 4f00 	tst.w	r0, #2147483648	; 0x80000000
 8000b32:	f440 0000 	orr.w	r0, r0, #8388608	; 0x800000
 8000b36:	f020 407f 	bic.w	r0, r0, #4278190080	; 0xff000000
 8000b3a:	bf18      	it	ne
 8000b3c:	4240      	negne	r0, r0
 8000b3e:	f011 4f00 	tst.w	r1, #2147483648	; 0x80000000
 8000b42:	f441 0100 	orr.w	r1, r1, #8388608	; 0x800000
 8000b46:	f021 417f 	bic.w	r1, r1, #4278190080	; 0xff000000
 8000b4a:	bf18      	it	ne
 8000b4c:	4249      	negne	r1, r1
 8000b4e:	ea92 0f03 	teq	r2, r3
 8000b52:	d03f      	beq.n	8000bd4 <__addsf3+0xd8>
 8000b54:	f1a2 0201 	sub.w	r2, r2, #1
 8000b58:	fa41 fc03 	asr.w	ip, r1, r3
 8000b5c:	eb10 000c 	adds.w	r0, r0, ip
 8000b60:	f1c3 0320 	rsb	r3, r3, #32
 8000b64:	fa01 f103 	lsl.w	r1, r1, r3
 8000b68:	f000 4300 	and.w	r3, r0, #2147483648	; 0x80000000
 8000b6c:	d502      	bpl.n	8000b74 <__addsf3+0x78>
 8000b6e:	4249      	negs	r1, r1
 8000b70:	eb60 0040 	sbc.w	r0, r0, r0, lsl #1
 8000b74:	f5b0 0f00 	cmp.w	r0, #8388608	; 0x800000
 8000b78:	d313      	bcc.n	8000ba2 <__addsf3+0xa6>
 8000b7a:	f1b0 7f80 	cmp.w	r0, #16777216	; 0x1000000
 8000b7e:	d306      	bcc.n	8000b8e <__addsf3+0x92>
 8000b80:	0840      	lsrs	r0, r0, #1
 8000b82:	ea4f 0131 	mov.w	r1, r1, rrx
 8000b86:	f102 0201 	add.w	r2, r2, #1
 8000b8a:	2afe      	cmp	r2, #254	; 0xfe
 8000b8c:	d251      	bcs.n	8000c32 <__addsf3+0x136>
 8000b8e:	f1b1 4f00 	cmp.w	r1, #2147483648	; 0x80000000
 8000b92:	eb40 50c2 	adc.w	r0, r0, r2, lsl #23
 8000b96:	bf08      	it	eq
 8000b98:	f020 0001 	biceq.w	r0, r0, #1
 8000b9c:	ea40 0003 	orr.w	r0, r0, r3
 8000ba0:	4770      	bx	lr
 8000ba2:	0049      	lsls	r1, r1, #1
 8000ba4:	eb40 0000 	adc.w	r0, r0, r0
 8000ba8:	3a01      	subs	r2, #1
 8000baa:	bf28      	it	cs
 8000bac:	f5b0 0f00 	cmpcs.w	r0, #8388608	; 0x800000
 8000bb0:	d2ed      	bcs.n	8000b8e <__addsf3+0x92>
 8000bb2:	fab0 fc80 	clz	ip, r0
 8000bb6:	f1ac 0c08 	sub.w	ip, ip, #8
 8000bba:	ebb2 020c 	subs.w	r2, r2, ip
 8000bbe:	fa00 f00c 	lsl.w	r0, r0, ip
 8000bc2:	bfaa      	itet	ge
 8000bc4:	eb00 50c2 	addge.w	r0, r0, r2, lsl #23
 8000bc8:	4252      	neglt	r2, r2
 8000bca:	4318      	orrge	r0, r3
 8000bcc:	bfbc      	itt	lt
 8000bce:	40d0      	lsrlt	r0, r2
 8000bd0:	4318      	orrlt	r0, r3
 8000bd2:	4770      	bx	lr
 8000bd4:	f092 0f00 	teq	r2, #0
 8000bd8:	f481 0100 	eor.w	r1, r1, #8388608	; 0x800000
 8000bdc:	bf06      	itte	eq
 8000bde:	f480 0000 	eoreq.w	r0, r0, #8388608	; 0x800000
 8000be2:	3201      	addeq	r2, #1
 8000be4:	3b01      	subne	r3, #1
 8000be6:	e7b5      	b.n	8000b54 <__addsf3+0x58>
 8000be8:	ea4f 0341 	mov.w	r3, r1, lsl #1
 8000bec:	ea7f 6c22 	mvns.w	ip, r2, asr #24
 8000bf0:	bf18      	it	ne
 8000bf2:	ea7f 6c23 	mvnsne.w	ip, r3, asr #24
 8000bf6:	d021      	beq.n	8000c3c <__addsf3+0x140>
 8000bf8:	ea92 0f03 	teq	r2, r3
 8000bfc:	d004      	beq.n	8000c08 <__addsf3+0x10c>
 8000bfe:	f092 0f00 	teq	r2, #0
 8000c02:	bf08      	it	eq
 8000c04:	4608      	moveq	r0, r1
 8000c06:	4770      	bx	lr
 8000c08:	ea90 0f01 	teq	r0, r1
 8000c0c:	bf1c      	itt	ne
 8000c0e:	2000      	movne	r0, #0
 8000c10:	4770      	bxne	lr
 8000c12:	f012 4f7f 	tst.w	r2, #4278190080	; 0xff000000
 8000c16:	d104      	bne.n	8000c22 <__addsf3+0x126>
 8000c18:	0040      	lsls	r0, r0, #1
 8000c1a:	bf28      	it	cs
 8000c1c:	f040 4000 	orrcs.w	r0, r0, #2147483648	; 0x80000000
 8000c20:	4770      	bx	lr
 8000c22:	f112 7200 	adds.w	r2, r2, #33554432	; 0x2000000
 8000c26:	bf3c      	itt	cc
 8000c28:	f500 0000 	addcc.w	r0, r0, #8388608	; 0x800000
 8000c2c:	4770      	bxcc	lr
 8000c2e:	f000 4300 	and.w	r3, r0, #2147483648	; 0x80000000
 8000c32:	f043 40fe 	orr.w	r0, r3, #2130706432	; 0x7f000000
 8000c36:	f440 0000 	orr.w	r0, r0, #8388608	; 0x800000
 8000c3a:	4770      	bx	lr
 8000c3c:	ea7f 6222 	mvns.w	r2, r2, asr #24
 8000c40:	bf16      	itet	ne
 8000c42:	4608      	movne	r0, r1
 8000c44:	ea7f 6323 	mvnseq.w	r3, r3, asr #24
 8000c48:	4601      	movne	r1, r0
 8000c4a:	0242      	lsls	r2, r0, #9
 8000c4c:	bf06      	itte	eq
 8000c4e:	ea5f 2341 	movseq.w	r3, r1, lsl #9
 8000c52:	ea90 0f01 	teqeq	r0, r1
 8000c56:	f440 0080 	orrne.w	r0, r0, #4194304	; 0x400000
 8000c5a:	4770      	bx	lr

08000c5c <__aeabi_ui2f>:
 8000c5c:	f04f 0300 	mov.w	r3, #0
 8000c60:	e004      	b.n	8000c6c <__aeabi_i2f+0x8>
 8000c62:	bf00      	nop

08000c64 <__aeabi_i2f>:
 8000c64:	f010 4300 	ands.w	r3, r0, #2147483648	; 0x80000000
 8000c68:	bf48      	it	mi
 8000c6a:	4240      	negmi	r0, r0
 8000c6c:	ea5f 0c00 	movs.w	ip, r0
 8000c70:	bf08      	it	eq
 8000c72:	4770      	bxeq	lr
 8000c74:	f043 4396 	orr.w	r3, r3, #1258291200	; 0x4b000000
 8000c78:	4601      	mov	r1, r0
 8000c7a:	f04f 0000 	mov.w	r0, #0
 8000c7e:	e01c      	b.n	8000cba <__aeabi_l2f+0x2a>

08000c80 <__aeabi_ul2f>:
 8000c80:	ea50 0201 	orrs.w	r2, r0, r1
 8000c84:	bf08      	it	eq
 8000c86:	4770      	bxeq	lr
 8000c88:	f04f 0300 	mov.w	r3, #0
 8000c8c:	e00a      	b.n	8000ca4 <__aeabi_l2f+0x14>
 8000c8e:	bf00      	nop

08000c90 <__aeabi_l2f>:
 8000c90:	ea50 0201 	orrs.w	r2, r0, r1
 8000c94:	bf08      	it	eq
 8000c96:	4770      	bxeq	lr
 8000c98:	f011 4300 	ands.w	r3, r1, #2147483648	; 0x80000000
 8000c9c:	d502      	bpl.n	8000ca4 <__aeabi_l2f+0x14>
 8000c9e:	4240      	negs	r0, r0
 8000ca0:	eb61 0141 	sbc.w	r1, r1, r1, lsl #1
 8000ca4:	ea5f 0c01 	movs.w	ip, r1
 8000ca8:	bf02      	ittt	eq
 8000caa:	4684      	moveq	ip, r0
 8000cac:	4601      	moveq	r1, r0
 8000cae:	2000      	moveq	r0, #0
 8000cb0:	f043 43b6 	orr.w	r3, r3, #1526726656	; 0x5b000000
 8000cb4:	bf08      	it	eq
 8000cb6:	f1a3 5380 	subeq.w	r3, r3, #268435456	; 0x10000000
 8000cba:	f5a3 0300 	sub.w	r3, r3, #8388608	; 0x800000
 8000cbe:	fabc f28c 	clz	r2, ip
 8000cc2:	3a08      	subs	r2, #8
 8000cc4:	eba3 53c2 	sub.w	r3, r3, r2, lsl #23
 8000cc8:	db10      	blt.n	8000cec <__aeabi_l2f+0x5c>
 8000cca:	fa01 fc02 	lsl.w	ip, r1, r2
 8000cce:	4463      	add	r3, ip
 8000cd0:	fa00 fc02 	lsl.w	ip, r0, r2
 8000cd4:	f1c2 0220 	rsb	r2, r2, #32
 8000cd8:	f1bc 4f00 	cmp.w	ip, #2147483648	; 0x80000000
 8000cdc:	fa20 f202 	lsr.w	r2, r0, r2
 8000ce0:	eb43 0002 	adc.w	r0, r3, r2
 8000ce4:	bf08      	it	eq
 8000ce6:	f020 0001 	biceq.w	r0, r0, #1
 8000cea:	4770      	bx	lr
 8000cec:	f102 0220 	add.w	r2, r2, #32
 8000cf0:	fa01 fc02 	lsl.w	ip, r1, r2
 8000cf4:	f1c2 0220 	rsb	r2, r2, #32
 8000cf8:	ea50 004c 	orrs.w	r0, r0, ip, lsl #1
 8000cfc:	fa21 f202 	lsr.w	r2, r1, r2
 8000d00:	eb43 0002 	adc.w	r0, r3, r2
 8000d04:	bf08      	it	eq
 8000d06:	ea20 70dc 	biceq.w	r0, r0, ip, lsr #31
 8000d0a:	4770      	bx	lr

08000d0c <KalmanFilter>:
}



float * KalmanFilter (float altitude, float acceleration, float est_prev[])
{
 8000d0c:	b5f0      	push	{r4, r5, r6, r7, lr}
 8000d0e:	b09b      	sub	sp, #108	; 0x6c
 8000d10:	af00      	add	r7, sp, #0
 8000d12:	60f8      	str	r0, [r7, #12]
 8000d14:	60b9      	str	r1, [r7, #8]
 8000d16:	607a      	str	r2, [r7, #4]
  extern float est[3];

  //float dt = 0.05;
  float Kgain[3][2] = { {0.0262, 0.0004},
 8000d18:	4b96      	ldr	r3, [pc, #600]	; (8000f74 <KalmanFilter+0x268>)
 8000d1a:	f107 0450 	add.w	r4, r7, #80	; 0x50
 8000d1e:	461d      	mov	r5, r3
 8000d20:	cd0f      	ldmia	r5!, {r0, r1, r2, r3}
 8000d22:	c40f      	stmia	r4!, {r0, r1, r2, r3}
 8000d24:	e895 0003 	ldmia.w	r5, {r0, r1}
 8000d28:	e884 0003 	stmia.w	r4, {r0, r1}
    {0.0070, 0.0107},
    {0.0000, 0.7861}
  };


  float A[3][3] = { {1, 0.05, 0.0013},
 8000d2c:	4b92      	ldr	r3, [pc, #584]	; (8000f78 <KalmanFilter+0x26c>)
 8000d2e:	f107 042c 	add.w	r4, r7, #44	; 0x2c
 8000d32:	461d      	mov	r5, r3
 8000d34:	cd0f      	ldmia	r5!, {r0, r1, r2, r3}
 8000d36:	c40f      	stmia	r4!, {r0, r1, r2, r3}
 8000d38:	cd0f      	ldmia	r5!, {r0, r1, r2, r3}
 8000d3a:	c40f      	stmia	r4!, {r0, r1, r2, r3}
 8000d3c:	682b      	ldr	r3, [r5, #0]
 8000d3e:	6023      	str	r3, [r4, #0]
		  { 0, 1.0000, 0.0500},
				  {0, 0, 1.0000}
  };

  float H[2][3] = { {1, 0, 0},
 8000d40:	4b8e      	ldr	r3, [pc, #568]	; (8000f7c <KalmanFilter+0x270>)
 8000d42:	f107 0414 	add.w	r4, r7, #20
 8000d46:	461d      	mov	r5, r3
 8000d48:	cd0f      	ldmia	r5!, {r0, r1, r2, r3}
 8000d4a:	c40f      	stmia	r4!, {r0, r1, r2, r3}
 8000d4c:	e895 0003 	ldmia.w	r5, {r0, r1}
 8000d50:	e884 0003 	stmia.w	r4, {r0, r1}
    {0, 0, 1}
  };

  est[0] =  A[0][0] * est_prev[0] + A[0][1] * est_prev[1] + A[0][2] * est_prev[2];
 8000d54:	6afa      	ldr	r2, [r7, #44]	; 0x2c
 8000d56:	687b      	ldr	r3, [r7, #4]
 8000d58:	681b      	ldr	r3, [r3, #0]
 8000d5a:	4619      	mov	r1, r3
 8000d5c:	4610      	mov	r0, r2
 8000d5e:	f7ff f9f5 	bl	800014c <__aeabi_fmul>
 8000d62:	4603      	mov	r3, r0
 8000d64:	461c      	mov	r4, r3
 8000d66:	6b3a      	ldr	r2, [r7, #48]	; 0x30
 8000d68:	687b      	ldr	r3, [r7, #4]
 8000d6a:	3304      	adds	r3, #4
 8000d6c:	681b      	ldr	r3, [r3, #0]
 8000d6e:	4619      	mov	r1, r3
 8000d70:	4610      	mov	r0, r2
 8000d72:	f7ff f9eb 	bl	800014c <__aeabi_fmul>
 8000d76:	4603      	mov	r3, r0
 8000d78:	4619      	mov	r1, r3
 8000d7a:	4620      	mov	r0, r4
 8000d7c:	f7ff febe 	bl	8000afc <__addsf3>
 8000d80:	4603      	mov	r3, r0
 8000d82:	461c      	mov	r4, r3
 8000d84:	6b7a      	ldr	r2, [r7, #52]	; 0x34
 8000d86:	687b      	ldr	r3, [r7, #4]
 8000d88:	3308      	adds	r3, #8
 8000d8a:	681b      	ldr	r3, [r3, #0]
 8000d8c:	4619      	mov	r1, r3
 8000d8e:	4610      	mov	r0, r2
 8000d90:	f7ff f9dc 	bl	800014c <__aeabi_fmul>
 8000d94:	4603      	mov	r3, r0
 8000d96:	4619      	mov	r1, r3
 8000d98:	4620      	mov	r0, r4
 8000d9a:	f7ff feaf 	bl	8000afc <__addsf3>
 8000d9e:	4603      	mov	r3, r0
 8000da0:	461a      	mov	r2, r3
 8000da2:	4b77      	ldr	r3, [pc, #476]	; (8000f80 <KalmanFilter+0x274>)
 8000da4:	601a      	str	r2, [r3, #0]
  est[1] =  A[1][0] * est_prev[0] + A[1][1] * est_prev[1] + A[1][2] * est_prev[2];
 8000da6:	6bba      	ldr	r2, [r7, #56]	; 0x38
 8000da8:	687b      	ldr	r3, [r7, #4]
 8000daa:	681b      	ldr	r3, [r3, #0]
 8000dac:	4619      	mov	r1, r3
 8000dae:	4610      	mov	r0, r2
 8000db0:	f7ff f9cc 	bl	800014c <__aeabi_fmul>
 8000db4:	4603      	mov	r3, r0
 8000db6:	461c      	mov	r4, r3
 8000db8:	6bfa      	ldr	r2, [r7, #60]	; 0x3c
 8000dba:	687b      	ldr	r3, [r7, #4]
 8000dbc:	3304      	adds	r3, #4
 8000dbe:	681b      	ldr	r3, [r3, #0]
 8000dc0:	4619      	mov	r1, r3
 8000dc2:	4610      	mov	r0, r2
 8000dc4:	f7ff f9c2 	bl	800014c <__aeabi_fmul>
 8000dc8:	4603      	mov	r3, r0
 8000dca:	4619      	mov	r1, r3
 8000dcc:	4620      	mov	r0, r4
 8000dce:	f7ff fe95 	bl	8000afc <__addsf3>
 8000dd2:	4603      	mov	r3, r0
 8000dd4:	461c      	mov	r4, r3
 8000dd6:	6c3a      	ldr	r2, [r7, #64]	; 0x40
 8000dd8:	687b      	ldr	r3, [r7, #4]
 8000dda:	3308      	adds	r3, #8
 8000ddc:	681b      	ldr	r3, [r3, #0]
 8000dde:	4619      	mov	r1, r3
 8000de0:	4610      	mov	r0, r2
 8000de2:	f7ff f9b3 	bl	800014c <__aeabi_fmul>
 8000de6:	4603      	mov	r3, r0
 8000de8:	4619      	mov	r1, r3
 8000dea:	4620      	mov	r0, r4
 8000dec:	f7ff fe86 	bl	8000afc <__addsf3>
 8000df0:	4603      	mov	r3, r0
 8000df2:	461a      	mov	r2, r3
 8000df4:	4b62      	ldr	r3, [pc, #392]	; (8000f80 <KalmanFilter+0x274>)
 8000df6:	605a      	str	r2, [r3, #4]
  est[2] =  A[2][0] * est_prev[0] + A[2][1] * est_prev[1] + A[2][2] * est_prev[2];
 8000df8:	6c7a      	ldr	r2, [r7, #68]	; 0x44
 8000dfa:	687b      	ldr	r3, [r7, #4]
 8000dfc:	681b      	ldr	r3, [r3, #0]
 8000dfe:	4619      	mov	r1, r3
 8000e00:	4610      	mov	r0, r2
 8000e02:	f7ff f9a3 	bl	800014c <__aeabi_fmul>
 8000e06:	4603      	mov	r3, r0
 8000e08:	461c      	mov	r4, r3
 8000e0a:	6cba      	ldr	r2, [r7, #72]	; 0x48
 8000e0c:	687b      	ldr	r3, [r7, #4]
 8000e0e:	3304      	adds	r3, #4
 8000e10:	681b      	ldr	r3, [r3, #0]
 8000e12:	4619      	mov	r1, r3
 8000e14:	4610      	mov	r0, r2
 8000e16:	f7ff f999 	bl	800014c <__aeabi_fmul>
 8000e1a:	4603      	mov	r3, r0
 8000e1c:	4619      	mov	r1, r3
 8000e1e:	4620      	mov	r0, r4
 8000e20:	f7ff fe6c 	bl	8000afc <__addsf3>
 8000e24:	4603      	mov	r3, r0
 8000e26:	461c      	mov	r4, r3
 8000e28:	6cfa      	ldr	r2, [r7, #76]	; 0x4c
 8000e2a:	687b      	ldr	r3, [r7, #4]
 8000e2c:	3308      	adds	r3, #8
 8000e2e:	681b      	ldr	r3, [r3, #0]
 8000e30:	4619      	mov	r1, r3
 8000e32:	4610      	mov	r0, r2
 8000e34:	f7ff f98a 	bl	800014c <__aeabi_fmul>
 8000e38:	4603      	mov	r3, r0
 8000e3a:	4619      	mov	r1, r3
 8000e3c:	4620      	mov	r0, r4
 8000e3e:	f7ff fe5d 	bl	8000afc <__addsf3>
 8000e42:	4603      	mov	r3, r0
 8000e44:	461a      	mov	r2, r3
 8000e46:	4b4e      	ldr	r3, [pc, #312]	; (8000f80 <KalmanFilter+0x274>)
 8000e48:	609a      	str	r2, [r3, #8]

  est[0] =  est[0] + Kgain[0][0] * (altitude - H[0][0] * est[0] - H[0][1] * est[1] - H[0][2] * est[2]) + Kgain[0][1] * (acceleration - H[1][0] * est[0] - H[1][1] *	est[1] - H[1][2] * est[2]);
 8000e4a:	4b4d      	ldr	r3, [pc, #308]	; (8000f80 <KalmanFilter+0x274>)
 8000e4c:	681c      	ldr	r4, [r3, #0]
 8000e4e:	6d3d      	ldr	r5, [r7, #80]	; 0x50
 8000e50:	697b      	ldr	r3, [r7, #20]
 8000e52:	4a4b      	ldr	r2, [pc, #300]	; (8000f80 <KalmanFilter+0x274>)
 8000e54:	6812      	ldr	r2, [r2, #0]
 8000e56:	4611      	mov	r1, r2
 8000e58:	4618      	mov	r0, r3
 8000e5a:	f7ff f977 	bl	800014c <__aeabi_fmul>
 8000e5e:	4603      	mov	r3, r0
 8000e60:	4619      	mov	r1, r3
 8000e62:	68f8      	ldr	r0, [r7, #12]
 8000e64:	f7ff fe48 	bl	8000af8 <__aeabi_fsub>
 8000e68:	4603      	mov	r3, r0
 8000e6a:	461e      	mov	r6, r3
 8000e6c:	69bb      	ldr	r3, [r7, #24]
 8000e6e:	4a44      	ldr	r2, [pc, #272]	; (8000f80 <KalmanFilter+0x274>)
 8000e70:	6852      	ldr	r2, [r2, #4]
 8000e72:	4611      	mov	r1, r2
 8000e74:	4618      	mov	r0, r3
 8000e76:	f7ff f969 	bl	800014c <__aeabi_fmul>
 8000e7a:	4603      	mov	r3, r0
 8000e7c:	4619      	mov	r1, r3
 8000e7e:	4630      	mov	r0, r6
 8000e80:	f7ff fe3a 	bl	8000af8 <__aeabi_fsub>
 8000e84:	4603      	mov	r3, r0
 8000e86:	461e      	mov	r6, r3
 8000e88:	69fb      	ldr	r3, [r7, #28]
 8000e8a:	4a3d      	ldr	r2, [pc, #244]	; (8000f80 <KalmanFilter+0x274>)
 8000e8c:	6892      	ldr	r2, [r2, #8]
 8000e8e:	4611      	mov	r1, r2
 8000e90:	4618      	mov	r0, r3
 8000e92:	f7ff f95b 	bl	800014c <__aeabi_fmul>
 8000e96:	4603      	mov	r3, r0
 8000e98:	4619      	mov	r1, r3
 8000e9a:	4630      	mov	r0, r6
 8000e9c:	f7ff fe2c 	bl	8000af8 <__aeabi_fsub>
 8000ea0:	4603      	mov	r3, r0
 8000ea2:	4619      	mov	r1, r3
 8000ea4:	4628      	mov	r0, r5
 8000ea6:	f7ff f951 	bl	800014c <__aeabi_fmul>
 8000eaa:	4603      	mov	r3, r0
 8000eac:	4619      	mov	r1, r3
 8000eae:	4620      	mov	r0, r4
 8000eb0:	f7ff fe24 	bl	8000afc <__addsf3>
 8000eb4:	4603      	mov	r3, r0
 8000eb6:	461d      	mov	r5, r3
 8000eb8:	6d7c      	ldr	r4, [r7, #84]	; 0x54
 8000eba:	6a3b      	ldr	r3, [r7, #32]
 8000ebc:	4a30      	ldr	r2, [pc, #192]	; (8000f80 <KalmanFilter+0x274>)
 8000ebe:	6812      	ldr	r2, [r2, #0]
 8000ec0:	4611      	mov	r1, r2
 8000ec2:	4618      	mov	r0, r3
 8000ec4:	f7ff f942 	bl	800014c <__aeabi_fmul>
 8000ec8:	4603      	mov	r3, r0
 8000eca:	4619      	mov	r1, r3
 8000ecc:	68b8      	ldr	r0, [r7, #8]
 8000ece:	f7ff fe13 	bl	8000af8 <__aeabi_fsub>
 8000ed2:	4603      	mov	r3, r0
 8000ed4:	461e      	mov	r6, r3
 8000ed6:	6a7b      	ldr	r3, [r7, #36]	; 0x24
 8000ed8:	4a29      	ldr	r2, [pc, #164]	; (8000f80 <KalmanFilter+0x274>)
 8000eda:	6852      	ldr	r2, [r2, #4]
 8000edc:	4611      	mov	r1, r2
 8000ede:	4618      	mov	r0, r3
 8000ee0:	f7ff f934 	bl	800014c <__aeabi_fmul>
 8000ee4:	4603      	mov	r3, r0
 8000ee6:	4619      	mov	r1, r3
 8000ee8:	4630      	mov	r0, r6
 8000eea:	f7ff fe05 	bl	8000af8 <__aeabi_fsub>
 8000eee:	4603      	mov	r3, r0
 8000ef0:	461e      	mov	r6, r3
 8000ef2:	6abb      	ldr	r3, [r7, #40]	; 0x28
 8000ef4:	4a22      	ldr	r2, [pc, #136]	; (8000f80 <KalmanFilter+0x274>)
 8000ef6:	6892      	ldr	r2, [r2, #8]
 8000ef8:	4611      	mov	r1, r2
 8000efa:	4618      	mov	r0, r3
 8000efc:	f7ff f926 	bl	800014c <__aeabi_fmul>
 8000f00:	4603      	mov	r3, r0
 8000f02:	4619      	mov	r1, r3
 8000f04:	4630      	mov	r0, r6
 8000f06:	f7ff fdf7 	bl	8000af8 <__aeabi_fsub>
 8000f0a:	4603      	mov	r3, r0
 8000f0c:	4619      	mov	r1, r3
 8000f0e:	4620      	mov	r0, r4
 8000f10:	f7ff f91c 	bl	800014c <__aeabi_fmul>
 8000f14:	4603      	mov	r3, r0
 8000f16:	4619      	mov	r1, r3
 8000f18:	4628      	mov	r0, r5
 8000f1a:	f7ff fdef 	bl	8000afc <__addsf3>
 8000f1e:	4603      	mov	r3, r0
 8000f20:	461a      	mov	r2, r3
 8000f22:	4b17      	ldr	r3, [pc, #92]	; (8000f80 <KalmanFilter+0x274>)
 8000f24:	601a      	str	r2, [r3, #0]
  est[1] =  est[1] + Kgain[1][0] * (altitude - H[0][0] * est[0] - H[0][1] * est[1] - H[0][2] * est[2]) + Kgain[1][1] * (acceleration - H[1][0] * est[0] - H[1][1] *est[1] -H[1][2] *est[2]);
 8000f26:	4b16      	ldr	r3, [pc, #88]	; (8000f80 <KalmanFilter+0x274>)
 8000f28:	685c      	ldr	r4, [r3, #4]
 8000f2a:	6dbd      	ldr	r5, [r7, #88]	; 0x58
 8000f2c:	697b      	ldr	r3, [r7, #20]
 8000f2e:	4a14      	ldr	r2, [pc, #80]	; (8000f80 <KalmanFilter+0x274>)
 8000f30:	6812      	ldr	r2, [r2, #0]
 8000f32:	4611      	mov	r1, r2
 8000f34:	4618      	mov	r0, r3
 8000f36:	f7ff f909 	bl	800014c <__aeabi_fmul>
 8000f3a:	4603      	mov	r3, r0
 8000f3c:	4619      	mov	r1, r3
 8000f3e:	68f8      	ldr	r0, [r7, #12]
 8000f40:	f7ff fdda 	bl	8000af8 <__aeabi_fsub>
 8000f44:	4603      	mov	r3, r0
 8000f46:	461e      	mov	r6, r3
 8000f48:	69bb      	ldr	r3, [r7, #24]
 8000f4a:	4a0d      	ldr	r2, [pc, #52]	; (8000f80 <KalmanFilter+0x274>)
 8000f4c:	6852      	ldr	r2, [r2, #4]
 8000f4e:	4611      	mov	r1, r2
 8000f50:	4618      	mov	r0, r3
 8000f52:	f7ff f8fb 	bl	800014c <__aeabi_fmul>
 8000f56:	4603      	mov	r3, r0
 8000f58:	4619      	mov	r1, r3
 8000f5a:	4630      	mov	r0, r6
 8000f5c:	f7ff fdcc 	bl	8000af8 <__aeabi_fsub>
 8000f60:	4603      	mov	r3, r0
 8000f62:	461e      	mov	r6, r3
 8000f64:	69fb      	ldr	r3, [r7, #28]
 8000f66:	4a06      	ldr	r2, [pc, #24]	; (8000f80 <KalmanFilter+0x274>)
 8000f68:	6892      	ldr	r2, [r2, #8]
 8000f6a:	4611      	mov	r1, r2
 8000f6c:	4618      	mov	r0, r3
 8000f6e:	f7ff f8ed 	bl	800014c <__aeabi_fmul>
 8000f72:	e007      	b.n	8000f84 <KalmanFilter+0x278>
 8000f74:	08004e0c 	.word	0x08004e0c
 8000f78:	08004e24 	.word	0x08004e24
 8000f7c:	08004e48 	.word	0x08004e48
 8000f80:	20000120 	.word	0x20000120
 8000f84:	4603      	mov	r3, r0
 8000f86:	4619      	mov	r1, r3
 8000f88:	4630      	mov	r0, r6
 8000f8a:	f7ff fdb5 	bl	8000af8 <__aeabi_fsub>
 8000f8e:	4603      	mov	r3, r0
 8000f90:	4619      	mov	r1, r3
 8000f92:	4628      	mov	r0, r5
 8000f94:	f7ff f8da 	bl	800014c <__aeabi_fmul>
 8000f98:	4603      	mov	r3, r0
 8000f9a:	4619      	mov	r1, r3
 8000f9c:	4620      	mov	r0, r4
 8000f9e:	f7ff fdad 	bl	8000afc <__addsf3>
 8000fa2:	4603      	mov	r3, r0
 8000fa4:	461d      	mov	r5, r3
 8000fa6:	6dfc      	ldr	r4, [r7, #92]	; 0x5c
 8000fa8:	6a3b      	ldr	r3, [r7, #32]
 8000faa:	4a54      	ldr	r2, [pc, #336]	; (80010fc <KalmanFilter+0x3f0>)
 8000fac:	6812      	ldr	r2, [r2, #0]
 8000fae:	4611      	mov	r1, r2
 8000fb0:	4618      	mov	r0, r3
 8000fb2:	f7ff f8cb 	bl	800014c <__aeabi_fmul>
 8000fb6:	4603      	mov	r3, r0
 8000fb8:	4619      	mov	r1, r3
 8000fba:	68b8      	ldr	r0, [r7, #8]
 8000fbc:	f7ff fd9c 	bl	8000af8 <__aeabi_fsub>
 8000fc0:	4603      	mov	r3, r0
 8000fc2:	461e      	mov	r6, r3
 8000fc4:	6a7b      	ldr	r3, [r7, #36]	; 0x24
 8000fc6:	4a4d      	ldr	r2, [pc, #308]	; (80010fc <KalmanFilter+0x3f0>)
 8000fc8:	6852      	ldr	r2, [r2, #4]
 8000fca:	4611      	mov	r1, r2
 8000fcc:	4618      	mov	r0, r3
 8000fce:	f7ff f8bd 	bl	800014c <__aeabi_fmul>
 8000fd2:	4603      	mov	r3, r0
 8000fd4:	4619      	mov	r1, r3
 8000fd6:	4630      	mov	r0, r6
 8000fd8:	f7ff fd8e 	bl	8000af8 <__aeabi_fsub>
 8000fdc:	4603      	mov	r3, r0
 8000fde:	461e      	mov	r6, r3
 8000fe0:	6abb      	ldr	r3, [r7, #40]	; 0x28
 8000fe2:	4a46      	ldr	r2, [pc, #280]	; (80010fc <KalmanFilter+0x3f0>)
 8000fe4:	6892      	ldr	r2, [r2, #8]
 8000fe6:	4611      	mov	r1, r2
 8000fe8:	4618      	mov	r0, r3
 8000fea:	f7ff f8af 	bl	800014c <__aeabi_fmul>
 8000fee:	4603      	mov	r3, r0
 8000ff0:	4619      	mov	r1, r3
 8000ff2:	4630      	mov	r0, r6
 8000ff4:	f7ff fd80 	bl	8000af8 <__aeabi_fsub>
 8000ff8:	4603      	mov	r3, r0
 8000ffa:	4619      	mov	r1, r3
 8000ffc:	4620      	mov	r0, r4
 8000ffe:	f7ff f8a5 	bl	800014c <__aeabi_fmul>
 8001002:	4603      	mov	r3, r0
 8001004:	4619      	mov	r1, r3
 8001006:	4628      	mov	r0, r5
 8001008:	f7ff fd78 	bl	8000afc <__addsf3>
 800100c:	4603      	mov	r3, r0
 800100e:	461a      	mov	r2, r3
 8001010:	4b3a      	ldr	r3, [pc, #232]	; (80010fc <KalmanFilter+0x3f0>)
 8001012:	605a      	str	r2, [r3, #4]
  est[2] =  est[1] + Kgain[2][0] * (altitude - H[0][0] * est[0] - H[0][1] * est[1] -H[0][2] * est[2]) + Kgain[2][1] * (acceleration -H[1][0] *est[0] -H[1][1] *est[1] -H[1][2] * est[2]);
 8001014:	4b39      	ldr	r3, [pc, #228]	; (80010fc <KalmanFilter+0x3f0>)
 8001016:	685c      	ldr	r4, [r3, #4]
 8001018:	6e3d      	ldr	r5, [r7, #96]	; 0x60
 800101a:	697b      	ldr	r3, [r7, #20]
 800101c:	4a37      	ldr	r2, [pc, #220]	; (80010fc <KalmanFilter+0x3f0>)
 800101e:	6812      	ldr	r2, [r2, #0]
 8001020:	4611      	mov	r1, r2
 8001022:	4618      	mov	r0, r3
 8001024:	f7ff f892 	bl	800014c <__aeabi_fmul>
 8001028:	4603      	mov	r3, r0
 800102a:	4619      	mov	r1, r3
 800102c:	68f8      	ldr	r0, [r7, #12]
 800102e:	f7ff fd63 	bl	8000af8 <__aeabi_fsub>
 8001032:	4603      	mov	r3, r0
 8001034:	461e      	mov	r6, r3
 8001036:	69bb      	ldr	r3, [r7, #24]
 8001038:	4a30      	ldr	r2, [pc, #192]	; (80010fc <KalmanFilter+0x3f0>)
 800103a:	6852      	ldr	r2, [r2, #4]
 800103c:	4611      	mov	r1, r2
 800103e:	4618      	mov	r0, r3
 8001040:	f7ff f884 	bl	800014c <__aeabi_fmul>
 8001044:	4603      	mov	r3, r0
 8001046:	4619      	mov	r1, r3
 8001048:	4630      	mov	r0, r6
 800104a:	f7ff fd55 	bl	8000af8 <__aeabi_fsub>
 800104e:	4603      	mov	r3, r0
 8001050:	461e      	mov	r6, r3
 8001052:	69fb      	ldr	r3, [r7, #28]
 8001054:	4a29      	ldr	r2, [pc, #164]	; (80010fc <KalmanFilter+0x3f0>)
 8001056:	6892      	ldr	r2, [r2, #8]
 8001058:	4611      	mov	r1, r2
 800105a:	4618      	mov	r0, r3
 800105c:	f7ff f876 	bl	800014c <__aeabi_fmul>
 8001060:	4603      	mov	r3, r0
 8001062:	4619      	mov	r1, r3
 8001064:	4630      	mov	r0, r6
 8001066:	f7ff fd47 	bl	8000af8 <__aeabi_fsub>
 800106a:	4603      	mov	r3, r0
 800106c:	4619      	mov	r1, r3
 800106e:	4628      	mov	r0, r5
 8001070:	f7ff f86c 	bl	800014c <__aeabi_fmul>
 8001074:	4603      	mov	r3, r0
 8001076:	4619      	mov	r1, r3
 8001078:	4620      	mov	r0, r4
 800107a:	f7ff fd3f 	bl	8000afc <__addsf3>
 800107e:	4603      	mov	r3, r0
 8001080:	461d      	mov	r5, r3
 8001082:	6e7c      	ldr	r4, [r7, #100]	; 0x64
 8001084:	6a3b      	ldr	r3, [r7, #32]
 8001086:	4a1d      	ldr	r2, [pc, #116]	; (80010fc <KalmanFilter+0x3f0>)
 8001088:	6812      	ldr	r2, [r2, #0]
 800108a:	4611      	mov	r1, r2
 800108c:	4618      	mov	r0, r3
 800108e:	f7ff f85d 	bl	800014c <__aeabi_fmul>
 8001092:	4603      	mov	r3, r0
 8001094:	4619      	mov	r1, r3
 8001096:	68b8      	ldr	r0, [r7, #8]
 8001098:	f7ff fd2e 	bl	8000af8 <__aeabi_fsub>
 800109c:	4603      	mov	r3, r0
 800109e:	461e      	mov	r6, r3
 80010a0:	6a7b      	ldr	r3, [r7, #36]	; 0x24
 80010a2:	4a16      	ldr	r2, [pc, #88]	; (80010fc <KalmanFilter+0x3f0>)
 80010a4:	6852      	ldr	r2, [r2, #4]
 80010a6:	4611      	mov	r1, r2
 80010a8:	4618      	mov	r0, r3
 80010aa:	f7ff f84f 	bl	800014c <__aeabi_fmul>
 80010ae:	4603      	mov	r3, r0
 80010b0:	4619      	mov	r1, r3
 80010b2:	4630      	mov	r0, r6
 80010b4:	f7ff fd20 	bl	8000af8 <__aeabi_fsub>
 80010b8:	4603      	mov	r3, r0
 80010ba:	461e      	mov	r6, r3
 80010bc:	6abb      	ldr	r3, [r7, #40]	; 0x28
 80010be:	4a0f      	ldr	r2, [pc, #60]	; (80010fc <KalmanFilter+0x3f0>)
 80010c0:	6892      	ldr	r2, [r2, #8]
 80010c2:	4611      	mov	r1, r2
 80010c4:	4618      	mov	r0, r3
 80010c6:	f7ff f841 	bl	800014c <__aeabi_fmul>
 80010ca:	4603      	mov	r3, r0
 80010cc:	4619      	mov	r1, r3
 80010ce:	4630      	mov	r0, r6
 80010d0:	f7ff fd12 	bl	8000af8 <__aeabi_fsub>
 80010d4:	4603      	mov	r3, r0
 80010d6:	4619      	mov	r1, r3
 80010d8:	4620      	mov	r0, r4
 80010da:	f7ff f837 	bl	800014c <__aeabi_fmul>
 80010de:	4603      	mov	r3, r0
 80010e0:	4619      	mov	r1, r3
 80010e2:	4628      	mov	r0, r5
 80010e4:	f7ff fd0a 	bl	8000afc <__addsf3>
 80010e8:	4603      	mov	r3, r0
 80010ea:	461a      	mov	r2, r3
 80010ec:	4b03      	ldr	r3, [pc, #12]	; (80010fc <KalmanFilter+0x3f0>)
 80010ee:	609a      	str	r2, [r3, #8]

  return est;
 80010f0:	4b02      	ldr	r3, [pc, #8]	; (80010fc <KalmanFilter+0x3f0>)
}
 80010f2:	4618      	mov	r0, r3
 80010f4:	376c      	adds	r7, #108	; 0x6c
 80010f6:	46bd      	mov	sp, r7
 80010f8:	bdf0      	pop	{r4, r5, r6, r7, pc}
 80010fa:	bf00      	nop
 80010fc:	20000120 	.word	0x20000120

08001100 <main>:
/**
  * @brief  The application entry point.
  * @retval int
  */
int main(void)
{
 8001100:	b580      	push	{r7, lr}
 8001102:	af00      	add	r7, sp, #0
  /* USER CODE END 1 */

  /* MCU Configuration--------------------------------------------------------*/

  /* Reset of all peripherals, Initializes the Flash interface and the Systick. */
  HAL_Init();
 8001104:	f000 fbf4 	bl	80018f0 <HAL_Init>
  /* USER CODE BEGIN Init */

  /* USER CODE END Init */

  /* Configure the system clock */
  SystemClock_Config();
 8001108:	f000 f81e 	bl	8001148 <SystemClock_Config>
  /* USER CODE BEGIN SysInit */

  /* USER CODE END SysInit */

  /* Initialize all configured peripherals */
  MX_GPIO_Init();
 800110c:	f000 f8aa 	bl	8001264 <MX_GPIO_Init>
  MX_DMA_Init();
 8001110:	f000 f88a 	bl	8001228 <MX_DMA_Init>
  MX_USART2_UART_Init();
 8001114:	f000 f85e 	bl	80011d4 <MX_USART2_UART_Init>
  /* USER CODE BEGIN 2 */
//  HAL_UART_Receive_DMA(&huart2, data_in, DATA_IN_SIZE);
//  HAL_UART_Receive_DMA(&huart2,data_in,DATA_IN_SIZE();
  HAL_UARTEx_ReceiveToIdle_DMA(&huart2,data_in,DATA_IN_SIZE);
 8001118:	2214      	movs	r2, #20
 800111a:	4908      	ldr	r1, [pc, #32]	; (800113c <main+0x3c>)
 800111c:	4808      	ldr	r0, [pc, #32]	; (8001140 <main+0x40>)
 800111e:	f001 fe58 	bl	8002dd2 <HAL_UARTEx_ReceiveToIdle_DMA>
  __HAL_DMA_DISABLE_IT(&hdma_usart2_rx, DMA_IT_HT);
 8001122:	4b08      	ldr	r3, [pc, #32]	; (8001144 <main+0x44>)
 8001124:	681b      	ldr	r3, [r3, #0]
 8001126:	681a      	ldr	r2, [r3, #0]
 8001128:	4b06      	ldr	r3, [pc, #24]	; (8001144 <main+0x44>)
 800112a:	681b      	ldr	r3, [r3, #0]
 800112c:	f022 0204 	bic.w	r2, r2, #4
 8001130:	601a      	str	r2, [r3, #0]
//	  i = DerivativeCounter(altitude_current_est, est_prev[0]);
//	  // Every 50 ms check is Apogee has been reached
//	  Apogee = CheckIfApogee (i);
//	  looptime = HAL_GetTick() - time ;
//	  sprintf(data_out,"%d\n",(int)(1000*est[0]));
	  HAL_Delay(10);
 8001132:	200a      	movs	r0, #10
 8001134:	f000 fc3e 	bl	80019b4 <HAL_Delay>
 8001138:	e7fb      	b.n	8001132 <main+0x32>
 800113a:	bf00      	nop
 800113c:	20000138 	.word	0x20000138
 8001140:	20000098 	.word	0x20000098
 8001144:	200000dc 	.word	0x200000dc

08001148 <SystemClock_Config>:
/**
  * @brief System Clock Configuration
  * @retval None
  */
void SystemClock_Config(void)
{
 8001148:	b580      	push	{r7, lr}
 800114a:	b090      	sub	sp, #64	; 0x40
 800114c:	af00      	add	r7, sp, #0
  RCC_OscInitTypeDef RCC_OscInitStruct = {0};
 800114e:	f107 0318 	add.w	r3, r7, #24
 8001152:	2228      	movs	r2, #40	; 0x28
 8001154:	2100      	movs	r1, #0
 8001156:	4618      	mov	r0, r3
 8001158:	f002 fb86 	bl	8003868 <memset>
  RCC_ClkInitTypeDef RCC_ClkInitStruct = {0};
 800115c:	1d3b      	adds	r3, r7, #4
 800115e:	2200      	movs	r2, #0
 8001160:	601a      	str	r2, [r3, #0]
 8001162:	605a      	str	r2, [r3, #4]
 8001164:	609a      	str	r2, [r3, #8]
 8001166:	60da      	str	r2, [r3, #12]
 8001168:	611a      	str	r2, [r3, #16]

  /** Initializes the RCC Oscillators according to the specified parameters
  * in the RCC_OscInitTypeDef structure.
  */
  RCC_OscInitStruct.OscillatorType = RCC_OSCILLATORTYPE_HSE;
 800116a:	2301      	movs	r3, #1
 800116c:	61bb      	str	r3, [r7, #24]
  RCC_OscInitStruct.HSEState = RCC_HSE_BYPASS;
 800116e:	f44f 23a0 	mov.w	r3, #327680	; 0x50000
 8001172:	61fb      	str	r3, [r7, #28]
  RCC_OscInitStruct.HSEPredivValue = RCC_HSE_PREDIV_DIV1;
 8001174:	2300      	movs	r3, #0
 8001176:	623b      	str	r3, [r7, #32]
  RCC_OscInitStruct.HSIState = RCC_HSI_ON;
 8001178:	2301      	movs	r3, #1
 800117a:	62bb      	str	r3, [r7, #40]	; 0x28
  RCC_OscInitStruct.PLL.PLLState = RCC_PLL_ON;
 800117c:	2302      	movs	r3, #2
 800117e:	637b      	str	r3, [r7, #52]	; 0x34
  RCC_OscInitStruct.PLL.PLLSource = RCC_PLLSOURCE_HSE;
 8001180:	f44f 3380 	mov.w	r3, #65536	; 0x10000
 8001184:	63bb      	str	r3, [r7, #56]	; 0x38
  RCC_OscInitStruct.PLL.PLLMUL = RCC_PLL_MUL9;
 8001186:	f44f 13e0 	mov.w	r3, #1835008	; 0x1c0000
 800118a:	63fb      	str	r3, [r7, #60]	; 0x3c
  if (HAL_RCC_OscConfig(&RCC_OscInitStruct) != HAL_OK)
 800118c:	f107 0318 	add.w	r3, r7, #24
 8001190:	4618      	mov	r0, r3
 8001192:	f001 f9b7 	bl	8002504 <HAL_RCC_OscConfig>
 8001196:	4603      	mov	r3, r0
 8001198:	2b00      	cmp	r3, #0
 800119a:	d001      	beq.n	80011a0 <SystemClock_Config+0x58>
  {
    Error_Handler();
 800119c:	f000 f9c4 	bl	8001528 <Error_Handler>
  }

  /** Initializes the CPU, AHB and APB buses clocks
  */
  RCC_ClkInitStruct.ClockType = RCC_CLOCKTYPE_HCLK|RCC_CLOCKTYPE_SYSCLK
 80011a0:	230f      	movs	r3, #15
 80011a2:	607b      	str	r3, [r7, #4]
                              |RCC_CLOCKTYPE_PCLK1|RCC_CLOCKTYPE_PCLK2;
  RCC_ClkInitStruct.SYSCLKSource = RCC_SYSCLKSOURCE_PLLCLK;
 80011a4:	2302      	movs	r3, #2
 80011a6:	60bb      	str	r3, [r7, #8]
  RCC_ClkInitStruct.AHBCLKDivider = RCC_SYSCLK_DIV1;
 80011a8:	2300      	movs	r3, #0
 80011aa:	60fb      	str	r3, [r7, #12]
  RCC_ClkInitStruct.APB1CLKDivider = RCC_HCLK_DIV2;
 80011ac:	f44f 6380 	mov.w	r3, #1024	; 0x400
 80011b0:	613b      	str	r3, [r7, #16]
  RCC_ClkInitStruct.APB2CLKDivider = RCC_HCLK_DIV1;
 80011b2:	2300      	movs	r3, #0
 80011b4:	617b      	str	r3, [r7, #20]

  if (HAL_RCC_ClockConfig(&RCC_ClkInitStruct, FLASH_LATENCY_2) != HAL_OK)
 80011b6:	1d3b      	adds	r3, r7, #4
 80011b8:	2102      	movs	r1, #2
 80011ba:	4618      	mov	r0, r3
 80011bc:	f001 fc24 	bl	8002a08 <HAL_RCC_ClockConfig>
 80011c0:	4603      	mov	r3, r0
 80011c2:	2b00      	cmp	r3, #0
 80011c4:	d001      	beq.n	80011ca <SystemClock_Config+0x82>
  {
    Error_Handler();
 80011c6:	f000 f9af 	bl	8001528 <Error_Handler>
  }
}
 80011ca:	bf00      	nop
 80011cc:	3740      	adds	r7, #64	; 0x40
 80011ce:	46bd      	mov	sp, r7
 80011d0:	bd80      	pop	{r7, pc}
	...

080011d4 <MX_USART2_UART_Init>:
  * @brief USART2 Initialization Function
  * @param None
  * @retval None
  */
static void MX_USART2_UART_Init(void)
{
 80011d4:	b580      	push	{r7, lr}
 80011d6:	af00      	add	r7, sp, #0
  /* USER CODE END USART2_Init 0 */

  /* USER CODE BEGIN USART2_Init 1 */

  /* USER CODE END USART2_Init 1 */
  huart2.Instance = USART2;
 80011d8:	4b11      	ldr	r3, [pc, #68]	; (8001220 <MX_USART2_UART_Init+0x4c>)
 80011da:	4a12      	ldr	r2, [pc, #72]	; (8001224 <MX_USART2_UART_Init+0x50>)
 80011dc:	601a      	str	r2, [r3, #0]
  huart2.Init.BaudRate = 115200;
 80011de:	4b10      	ldr	r3, [pc, #64]	; (8001220 <MX_USART2_UART_Init+0x4c>)
 80011e0:	f44f 32e1 	mov.w	r2, #115200	; 0x1c200
 80011e4:	605a      	str	r2, [r3, #4]
  huart2.Init.WordLength = UART_WORDLENGTH_8B;
 80011e6:	4b0e      	ldr	r3, [pc, #56]	; (8001220 <MX_USART2_UART_Init+0x4c>)
 80011e8:	2200      	movs	r2, #0
 80011ea:	609a      	str	r2, [r3, #8]
  huart2.Init.StopBits = UART_STOPBITS_1;
 80011ec:	4b0c      	ldr	r3, [pc, #48]	; (8001220 <MX_USART2_UART_Init+0x4c>)
 80011ee:	2200      	movs	r2, #0
 80011f0:	60da      	str	r2, [r3, #12]
  huart2.Init.Parity = UART_PARITY_NONE;
 80011f2:	4b0b      	ldr	r3, [pc, #44]	; (8001220 <MX_USART2_UART_Init+0x4c>)
 80011f4:	2200      	movs	r2, #0
 80011f6:	611a      	str	r2, [r3, #16]
  huart2.Init.Mode = UART_MODE_TX_RX;
 80011f8:	4b09      	ldr	r3, [pc, #36]	; (8001220 <MX_USART2_UART_Init+0x4c>)
 80011fa:	220c      	movs	r2, #12
 80011fc:	615a      	str	r2, [r3, #20]
  huart2.Init.HwFlowCtl = UART_HWCONTROL_NONE;
 80011fe:	4b08      	ldr	r3, [pc, #32]	; (8001220 <MX_USART2_UART_Init+0x4c>)
 8001200:	2200      	movs	r2, #0
 8001202:	619a      	str	r2, [r3, #24]
  huart2.Init.OverSampling = UART_OVERSAMPLING_16;
 8001204:	4b06      	ldr	r3, [pc, #24]	; (8001220 <MX_USART2_UART_Init+0x4c>)
 8001206:	2200      	movs	r2, #0
 8001208:	61da      	str	r2, [r3, #28]
  if (HAL_UART_Init(&huart2) != HAL_OK)
 800120a:	4805      	ldr	r0, [pc, #20]	; (8001220 <MX_USART2_UART_Init+0x4c>)
 800120c:	f001 fd94 	bl	8002d38 <HAL_UART_Init>
 8001210:	4603      	mov	r3, r0
 8001212:	2b00      	cmp	r3, #0
 8001214:	d001      	beq.n	800121a <MX_USART2_UART_Init+0x46>
  {
    Error_Handler();
 8001216:	f000 f987 	bl	8001528 <Error_Handler>
  }
  /* USER CODE BEGIN USART2_Init 2 */

  /* USER CODE END USART2_Init 2 */

}
 800121a:	bf00      	nop
 800121c:	bd80      	pop	{r7, pc}
 800121e:	bf00      	nop
 8001220:	20000098 	.word	0x20000098
 8001224:	40004400 	.word	0x40004400

08001228 <MX_DMA_Init>:

/**
  * Enable DMA controller clock
  */
static void MX_DMA_Init(void)
{
 8001228:	b580      	push	{r7, lr}
 800122a:	b082      	sub	sp, #8
 800122c:	af00      	add	r7, sp, #0

  /* DMA controller clock enable */
  __HAL_RCC_DMA1_CLK_ENABLE();
 800122e:	4b0c      	ldr	r3, [pc, #48]	; (8001260 <MX_DMA_Init+0x38>)
 8001230:	695b      	ldr	r3, [r3, #20]
 8001232:	4a0b      	ldr	r2, [pc, #44]	; (8001260 <MX_DMA_Init+0x38>)
 8001234:	f043 0301 	orr.w	r3, r3, #1
 8001238:	6153      	str	r3, [r2, #20]
 800123a:	4b09      	ldr	r3, [pc, #36]	; (8001260 <MX_DMA_Init+0x38>)
 800123c:	695b      	ldr	r3, [r3, #20]
 800123e:	f003 0301 	and.w	r3, r3, #1
 8001242:	607b      	str	r3, [r7, #4]
 8001244:	687b      	ldr	r3, [r7, #4]

  /* DMA interrupt init */
  /* DMA1_Channel6_IRQn interrupt configuration */
  HAL_NVIC_SetPriority(DMA1_Channel6_IRQn, 0, 0);
 8001246:	2200      	movs	r2, #0
 8001248:	2100      	movs	r1, #0
 800124a:	2010      	movs	r0, #16
 800124c:	f000 fcad 	bl	8001baa <HAL_NVIC_SetPriority>
  HAL_NVIC_EnableIRQ(DMA1_Channel6_IRQn);
 8001250:	2010      	movs	r0, #16
 8001252:	f000 fcc6 	bl	8001be2 <HAL_NVIC_EnableIRQ>

}
 8001256:	bf00      	nop
 8001258:	3708      	adds	r7, #8
 800125a:	46bd      	mov	sp, r7
 800125c:	bd80      	pop	{r7, pc}
 800125e:	bf00      	nop
 8001260:	40021000 	.word	0x40021000

08001264 <MX_GPIO_Init>:
  * @brief GPIO Initialization Function
  * @param None
  * @retval None
  */
static void MX_GPIO_Init(void)
{
 8001264:	b580      	push	{r7, lr}
 8001266:	b088      	sub	sp, #32
 8001268:	af00      	add	r7, sp, #0
  GPIO_InitTypeDef GPIO_InitStruct = {0};
 800126a:	f107 0310 	add.w	r3, r7, #16
 800126e:	2200      	movs	r2, #0
 8001270:	601a      	str	r2, [r3, #0]
 8001272:	605a      	str	r2, [r3, #4]
 8001274:	609a      	str	r2, [r3, #8]
 8001276:	60da      	str	r2, [r3, #12]

  /* GPIO Ports Clock Enable */
  __HAL_RCC_GPIOC_CLK_ENABLE();
 8001278:	4b2d      	ldr	r3, [pc, #180]	; (8001330 <MX_GPIO_Init+0xcc>)
 800127a:	699b      	ldr	r3, [r3, #24]
 800127c:	4a2c      	ldr	r2, [pc, #176]	; (8001330 <MX_GPIO_Init+0xcc>)
 800127e:	f043 0310 	orr.w	r3, r3, #16
 8001282:	6193      	str	r3, [r2, #24]
 8001284:	4b2a      	ldr	r3, [pc, #168]	; (8001330 <MX_GPIO_Init+0xcc>)
 8001286:	699b      	ldr	r3, [r3, #24]
 8001288:	f003 0310 	and.w	r3, r3, #16
 800128c:	60fb      	str	r3, [r7, #12]
 800128e:	68fb      	ldr	r3, [r7, #12]
  __HAL_RCC_GPIOD_CLK_ENABLE();
 8001290:	4b27      	ldr	r3, [pc, #156]	; (8001330 <MX_GPIO_Init+0xcc>)
 8001292:	699b      	ldr	r3, [r3, #24]
 8001294:	4a26      	ldr	r2, [pc, #152]	; (8001330 <MX_GPIO_Init+0xcc>)
 8001296:	f043 0320 	orr.w	r3, r3, #32
 800129a:	6193      	str	r3, [r2, #24]
 800129c:	4b24      	ldr	r3, [pc, #144]	; (8001330 <MX_GPIO_Init+0xcc>)
 800129e:	699b      	ldr	r3, [r3, #24]
 80012a0:	f003 0320 	and.w	r3, r3, #32
 80012a4:	60bb      	str	r3, [r7, #8]
 80012a6:	68bb      	ldr	r3, [r7, #8]
  __HAL_RCC_GPIOA_CLK_ENABLE();
 80012a8:	4b21      	ldr	r3, [pc, #132]	; (8001330 <MX_GPIO_Init+0xcc>)
 80012aa:	699b      	ldr	r3, [r3, #24]
 80012ac:	4a20      	ldr	r2, [pc, #128]	; (8001330 <MX_GPIO_Init+0xcc>)
 80012ae:	f043 0304 	orr.w	r3, r3, #4
 80012b2:	6193      	str	r3, [r2, #24]
 80012b4:	4b1e      	ldr	r3, [pc, #120]	; (8001330 <MX_GPIO_Init+0xcc>)
 80012b6:	699b      	ldr	r3, [r3, #24]
 80012b8:	f003 0304 	and.w	r3, r3, #4
 80012bc:	607b      	str	r3, [r7, #4]
 80012be:	687b      	ldr	r3, [r7, #4]
  __HAL_RCC_GPIOB_CLK_ENABLE();
 80012c0:	4b1b      	ldr	r3, [pc, #108]	; (8001330 <MX_GPIO_Init+0xcc>)
 80012c2:	699b      	ldr	r3, [r3, #24]
 80012c4:	4a1a      	ldr	r2, [pc, #104]	; (8001330 <MX_GPIO_Init+0xcc>)
 80012c6:	f043 0308 	orr.w	r3, r3, #8
 80012ca:	6193      	str	r3, [r2, #24]
 80012cc:	4b18      	ldr	r3, [pc, #96]	; (8001330 <MX_GPIO_Init+0xcc>)
 80012ce:	699b      	ldr	r3, [r3, #24]
 80012d0:	f003 0308 	and.w	r3, r3, #8
 80012d4:	603b      	str	r3, [r7, #0]
 80012d6:	683b      	ldr	r3, [r7, #0]

  /*Configure GPIO pin Output Level */
  HAL_GPIO_WritePin(LD2_GPIO_Port, LD2_Pin, GPIO_PIN_RESET);
 80012d8:	2200      	movs	r2, #0
 80012da:	2120      	movs	r1, #32
 80012dc:	4815      	ldr	r0, [pc, #84]	; (8001334 <MX_GPIO_Init+0xd0>)
 80012de:	f001 f8bd 	bl	800245c <HAL_GPIO_WritePin>

  /*Configure GPIO pin : B1_Pin */
  GPIO_InitStruct.Pin = B1_Pin;
 80012e2:	f44f 5300 	mov.w	r3, #8192	; 0x2000
 80012e6:	613b      	str	r3, [r7, #16]
  GPIO_InitStruct.Mode = GPIO_MODE_IT_RISING;
 80012e8:	4b13      	ldr	r3, [pc, #76]	; (8001338 <MX_GPIO_Init+0xd4>)
 80012ea:	617b      	str	r3, [r7, #20]
  GPIO_InitStruct.Pull = GPIO_NOPULL;
 80012ec:	2300      	movs	r3, #0
 80012ee:	61bb      	str	r3, [r7, #24]
  HAL_GPIO_Init(B1_GPIO_Port, &GPIO_InitStruct);
 80012f0:	f107 0310 	add.w	r3, r7, #16
 80012f4:	4619      	mov	r1, r3
 80012f6:	4811      	ldr	r0, [pc, #68]	; (800133c <MX_GPIO_Init+0xd8>)
 80012f8:	f000 ff2c 	bl	8002154 <HAL_GPIO_Init>

  /*Configure GPIO pin : LD2_Pin */
  GPIO_InitStruct.Pin = LD2_Pin;
 80012fc:	2320      	movs	r3, #32
 80012fe:	613b      	str	r3, [r7, #16]
  GPIO_InitStruct.Mode = GPIO_MODE_OUTPUT_PP;
 8001300:	2301      	movs	r3, #1
 8001302:	617b      	str	r3, [r7, #20]
  GPIO_InitStruct.Pull = GPIO_NOPULL;
 8001304:	2300      	movs	r3, #0
 8001306:	61bb      	str	r3, [r7, #24]
  GPIO_InitStruct.Speed = GPIO_SPEED_FREQ_LOW;
 8001308:	2302      	movs	r3, #2
 800130a:	61fb      	str	r3, [r7, #28]
  HAL_GPIO_Init(LD2_GPIO_Port, &GPIO_InitStruct);
 800130c:	f107 0310 	add.w	r3, r7, #16
 8001310:	4619      	mov	r1, r3
 8001312:	4808      	ldr	r0, [pc, #32]	; (8001334 <MX_GPIO_Init+0xd0>)
 8001314:	f000 ff1e 	bl	8002154 <HAL_GPIO_Init>

  /* EXTI interrupt init*/
  HAL_NVIC_SetPriority(EXTI15_10_IRQn, 0, 0);
 8001318:	2200      	movs	r2, #0
 800131a:	2100      	movs	r1, #0
 800131c:	2028      	movs	r0, #40	; 0x28
 800131e:	f000 fc44 	bl	8001baa <HAL_NVIC_SetPriority>
  HAL_NVIC_EnableIRQ(EXTI15_10_IRQn);
 8001322:	2028      	movs	r0, #40	; 0x28
 8001324:	f000 fc5d 	bl	8001be2 <HAL_NVIC_EnableIRQ>

}
 8001328:	bf00      	nop
 800132a:	3720      	adds	r7, #32
 800132c:	46bd      	mov	sp, r7
 800132e:	bd80      	pop	{r7, pc}
 8001330:	40021000 	.word	0x40021000
 8001334:	40010800 	.word	0x40010800
 8001338:	10110000 	.word	0x10110000
 800133c:	40011000 	.word	0x40011000

08001340 <HAL_UART_RxHalfCpltCallback>:

/* USER CODE BEGIN 4 */


void HAL_UART_RxHalfCpltCallback(UART_HandleTypeDef *huart)
{
 8001340:	b580      	push	{r7, lr}
 8001342:	b082      	sub	sp, #8
 8001344:	af00      	add	r7, sp, #0
 8001346:	6078      	str	r0, [r7, #4]
  HAL_GPIO_TogglePin(LD2_GPIO_Port, LD2_Pin);  // toggle PA0
 8001348:	2120      	movs	r1, #32
 800134a:	4803      	ldr	r0, [pc, #12]	; (8001358 <HAL_UART_RxHalfCpltCallback+0x18>)
 800134c:	f001 f89e 	bl	800248c <HAL_GPIO_TogglePin>
}
 8001350:	bf00      	nop
 8001352:	3708      	adds	r7, #8
 8001354:	46bd      	mov	sp, r7
 8001356:	bd80      	pop	{r7, pc}
 8001358:	40010800 	.word	0x40010800

0800135c <HAL_UARTEx_RxEventCallback>:
//	HAL_UART_Receive_DMA(&huart2,data_in,DATA_IN_SIZE);
//}


void HAL_UARTEx_RxEventCallback(UART_HandleTypeDef *huart, uint16_t Size)
{
 800135c:	b580      	push	{r7, lr}
 800135e:	b082      	sub	sp, #8
 8001360:	af00      	add	r7, sp, #0
 8001362:	6078      	str	r0, [r7, #4]
 8001364:	460b      	mov	r3, r1
 8001366:	807b      	strh	r3, [r7, #2]
	if (huart->Instance == USART2)
 8001368:	687b      	ldr	r3, [r7, #4]
 800136a:	681b      	ldr	r3, [r3, #0]
 800136c:	4a1f      	ldr	r2, [pc, #124]	; (80013ec <HAL_UARTEx_RxEventCallback+0x90>)
 800136e:	4293      	cmp	r3, r2
 8001370:	d138      	bne.n	80013e4 <HAL_UARTEx_RxEventCallback+0x88>
	{
		RX_bytes = Size ;
 8001372:	4a1f      	ldr	r2, [pc, #124]	; (80013f0 <HAL_UARTEx_RxEventCallback+0x94>)
 8001374:	887b      	ldrh	r3, [r7, #2]
 8001376:	8013      	strh	r3, [r2, #0]
		old_pos += Size ;
 8001378:	4b1e      	ldr	r3, [pc, #120]	; (80013f4 <HAL_UARTEx_RxEventCallback+0x98>)
 800137a:	881b      	ldrh	r3, [r3, #0]
 800137c:	b29a      	uxth	r2, r3
 800137e:	887b      	ldrh	r3, [r7, #2]
 8001380:	4413      	add	r3, r2
 8001382:	b29a      	uxth	r2, r3
 8001384:	4b1b      	ldr	r3, [pc, #108]	; (80013f4 <HAL_UARTEx_RxEventCallback+0x98>)
 8001386:	801a      	strh	r2, [r3, #0]
//		RX_bytes += Size ;
//		old_pos += Size ;
		if(old_pos >= DATA_IN_SIZE){
 8001388:	4b1a      	ldr	r3, [pc, #104]	; (80013f4 <HAL_UARTEx_RxEventCallback+0x98>)
 800138a:	881b      	ldrh	r3, [r3, #0]
 800138c:	b29b      	uxth	r3, r3
 800138e:	2b13      	cmp	r3, #19
 8001390:	d906      	bls.n	80013a0 <HAL_UARTEx_RxEventCallback+0x44>
				old_pos = old_pos - DATA_IN_SIZE ;
 8001392:	4b18      	ldr	r3, [pc, #96]	; (80013f4 <HAL_UARTEx_RxEventCallback+0x98>)
 8001394:	881b      	ldrh	r3, [r3, #0]
 8001396:	b29b      	uxth	r3, r3
 8001398:	3b14      	subs	r3, #20
 800139a:	b29a      	uxth	r2, r3
 800139c:	4b15      	ldr	r3, [pc, #84]	; (80013f4 <HAL_UARTEx_RxEventCallback+0x98>)
 800139e:	801a      	strh	r2, [r3, #0]
		}

		edit_text(data_in, numeric_data_in,old_pos,RX_bytes);
 80013a0:	4b14      	ldr	r3, [pc, #80]	; (80013f4 <HAL_UARTEx_RxEventCallback+0x98>)
 80013a2:	881b      	ldrh	r3, [r3, #0]
 80013a4:	b29a      	uxth	r2, r3
 80013a6:	4b12      	ldr	r3, [pc, #72]	; (80013f0 <HAL_UARTEx_RxEventCallback+0x94>)
 80013a8:	881b      	ldrh	r3, [r3, #0]
 80013aa:	b29b      	uxth	r3, r3
 80013ac:	4912      	ldr	r1, [pc, #72]	; (80013f8 <HAL_UARTEx_RxEventCallback+0x9c>)
 80013ae:	4813      	ldr	r0, [pc, #76]	; (80013fc <HAL_UARTEx_RxEventCallback+0xa0>)
 80013b0:	f000 f832 	bl	8001418 <edit_text>
		estimate = KalmanFilter (Altitude_measurement, Acceleration_measurement, est_prev);
 80013b4:	4b12      	ldr	r3, [pc, #72]	; (8001400 <HAL_UARTEx_RxEventCallback+0xa4>)
 80013b6:	681b      	ldr	r3, [r3, #0]
 80013b8:	4a12      	ldr	r2, [pc, #72]	; (8001404 <HAL_UARTEx_RxEventCallback+0xa8>)
 80013ba:	6811      	ldr	r1, [r2, #0]
 80013bc:	4a12      	ldr	r2, [pc, #72]	; (8001408 <HAL_UARTEx_RxEventCallback+0xac>)
 80013be:	4618      	mov	r0, r3
 80013c0:	f7ff fca4 	bl	8000d0c <KalmanFilter>
 80013c4:	4603      	mov	r3, r0
 80013c6:	4a11      	ldr	r2, [pc, #68]	; (800140c <HAL_UARTEx_RxEventCallback+0xb0>)
 80013c8:	6013      	str	r3, [r2, #0]
		HAL_UARTEx_ReceiveToIdle_DMA(&huart2,data_in,DATA_IN_SIZE);
 80013ca:	2214      	movs	r2, #20
 80013cc:	490b      	ldr	r1, [pc, #44]	; (80013fc <HAL_UARTEx_RxEventCallback+0xa0>)
 80013ce:	4810      	ldr	r0, [pc, #64]	; (8001410 <HAL_UARTEx_RxEventCallback+0xb4>)
 80013d0:	f001 fcff 	bl	8002dd2 <HAL_UARTEx_ReceiveToIdle_DMA>
		__HAL_DMA_DISABLE_IT(&hdma_usart2_rx, DMA_IT_HT);
 80013d4:	4b0f      	ldr	r3, [pc, #60]	; (8001414 <HAL_UARTEx_RxEventCallback+0xb8>)
 80013d6:	681b      	ldr	r3, [r3, #0]
 80013d8:	681a      	ldr	r2, [r3, #0]
 80013da:	4b0e      	ldr	r3, [pc, #56]	; (8001414 <HAL_UARTEx_RxEventCallback+0xb8>)
 80013dc:	681b      	ldr	r3, [r3, #0]
 80013de:	f022 0204 	bic.w	r2, r2, #4
 80013e2:	601a      	str	r2, [r3, #0]

	}

}
 80013e4:	bf00      	nop
 80013e6:	3708      	adds	r7, #8
 80013e8:	46bd      	mov	sp, r7
 80013ea:	bd80      	pop	{r7, pc}
 80013ec:	40004400 	.word	0x40004400
 80013f0:	20000162 	.word	0x20000162
 80013f4:	20000160 	.word	0x20000160
 80013f8:	2000014c 	.word	0x2000014c
 80013fc:	20000138 	.word	0x20000138
 8001400:	20000130 	.word	0x20000130
 8001404:	20000134 	.word	0x20000134
 8001408:	20000000 	.word	0x20000000
 800140c:	2000012c 	.word	0x2000012c
 8001410:	20000098 	.word	0x20000098
 8001414:	200000dc 	.word	0x200000dc

08001418 <edit_text>:


void edit_text(char text_in[], char numtext[], uint16_t RX_in_pos,uint16_t RX_bytes){
 8001418:	b580      	push	{r7, lr}
 800141a:	b09c      	sub	sp, #112	; 0x70
 800141c:	af00      	add	r7, sp, #0
 800141e:	60f8      	str	r0, [r7, #12]
 8001420:	60b9      	str	r1, [r7, #8]
 8001422:	4611      	mov	r1, r2
 8001424:	461a      	mov	r2, r3
 8001426:	460b      	mov	r3, r1
 8001428:	80fb      	strh	r3, [r7, #6]
 800142a:	4613      	mov	r3, r2
 800142c:	80bb      	strh	r3, [r7, #4]
	//	if(text_in[RX_bytes-1] =='f'){
	//		process_idx = 0 ;
	//		return ;
	//	}

	for(int j=0; j<RX_bytes ;j++){
 800142e:	2300      	movs	r3, #0
 8001430:	66fb      	str	r3, [r7, #108]	; 0x6c
 8001432:	e00a      	b.n	800144a <edit_text+0x32>
		numtext[j] = text_in[j];
 8001434:	6efb      	ldr	r3, [r7, #108]	; 0x6c
 8001436:	68fa      	ldr	r2, [r7, #12]
 8001438:	441a      	add	r2, r3
 800143a:	6efb      	ldr	r3, [r7, #108]	; 0x6c
 800143c:	68b9      	ldr	r1, [r7, #8]
 800143e:	440b      	add	r3, r1
 8001440:	7812      	ldrb	r2, [r2, #0]
 8001442:	701a      	strb	r2, [r3, #0]
	for(int j=0; j<RX_bytes ;j++){
 8001444:	6efb      	ldr	r3, [r7, #108]	; 0x6c
 8001446:	3301      	adds	r3, #1
 8001448:	66fb      	str	r3, [r7, #108]	; 0x6c
 800144a:	88bb      	ldrh	r3, [r7, #4]
 800144c:	6efa      	ldr	r2, [r7, #108]	; 0x6c
 800144e:	429a      	cmp	r2, r3
 8001450:	dbf0      	blt.n	8001434 <edit_text+0x1c>



	// Separate string and convert it to floats
	char * data_in_copy[DATA_IN_SIZE];
	sprintf(data_in_copy,data_in);
 8001452:	f107 0310 	add.w	r3, r7, #16
 8001456:	492e      	ldr	r1, [pc, #184]	; (8001510 <edit_text+0xf8>)
 8001458:	4618      	mov	r0, r3
 800145a:	f002 fa0d 	bl	8003878 <siprintf>
	char* token = strtok(data_in_copy,",");
 800145e:	f107 0310 	add.w	r3, r7, #16
 8001462:	492c      	ldr	r1, [pc, #176]	; (8001514 <edit_text+0xfc>)
 8001464:	4618      	mov	r0, r3
 8001466:	f002 fa27 	bl	80038b8 <strtok>
 800146a:	66b8      	str	r0, [r7, #104]	; 0x68
	int i = 0 ;
 800146c:	2300      	movs	r3, #0
 800146e:	667b      	str	r3, [r7, #100]	; 0x64
	while( token != NULL ) {
 8001470:	e037      	b.n	80014e2 <edit_text+0xca>
		if(i == 0){
 8001472:	6e7b      	ldr	r3, [r7, #100]	; 0x64
 8001474:	2b00      	cmp	r3, #0
 8001476:	d114      	bne.n	80014a2 <edit_text+0x8a>
			Altitude_measurement = atoi(token)/1000.0;
 8001478:	6eb8      	ldr	r0, [r7, #104]	; 0x68
 800147a:	f002 f9c7 	bl	800380c <atoi>
 800147e:	4603      	mov	r3, r0
 8001480:	4618      	mov	r0, r3
 8001482:	f7ff f869 	bl	8000558 <__aeabi_i2d>
 8001486:	f04f 0200 	mov.w	r2, #0
 800148a:	4b23      	ldr	r3, [pc, #140]	; (8001518 <edit_text+0x100>)
 800148c:	f7ff f9f8 	bl	8000880 <__aeabi_ddiv>
 8001490:	4602      	mov	r2, r0
 8001492:	460b      	mov	r3, r1
 8001494:	4610      	mov	r0, r2
 8001496:	4619      	mov	r1, r3
 8001498:	f7ff fada 	bl	8000a50 <__aeabi_d2f>
 800149c:	4603      	mov	r3, r0
 800149e:	4a1f      	ldr	r2, [pc, #124]	; (800151c <edit_text+0x104>)
 80014a0:	6013      	str	r3, [r2, #0]
		}

		if(i == 1){
 80014a2:	6e7b      	ldr	r3, [r7, #100]	; 0x64
 80014a4:	2b01      	cmp	r3, #1
 80014a6:	d114      	bne.n	80014d2 <edit_text+0xba>
			Acceleration_measurement = atoi(token)/1000.0;
 80014a8:	6eb8      	ldr	r0, [r7, #104]	; 0x68
 80014aa:	f002 f9af 	bl	800380c <atoi>
 80014ae:	4603      	mov	r3, r0
 80014b0:	4618      	mov	r0, r3
 80014b2:	f7ff f851 	bl	8000558 <__aeabi_i2d>
 80014b6:	f04f 0200 	mov.w	r2, #0
 80014ba:	4b17      	ldr	r3, [pc, #92]	; (8001518 <edit_text+0x100>)
 80014bc:	f7ff f9e0 	bl	8000880 <__aeabi_ddiv>
 80014c0:	4602      	mov	r2, r0
 80014c2:	460b      	mov	r3, r1
 80014c4:	4610      	mov	r0, r2
 80014c6:	4619      	mov	r1, r3
 80014c8:	f7ff fac2 	bl	8000a50 <__aeabi_d2f>
 80014cc:	4603      	mov	r3, r0
 80014ce:	4a14      	ldr	r2, [pc, #80]	; (8001520 <edit_text+0x108>)
 80014d0:	6013      	str	r3, [r2, #0]
		}
		token = strtok(NULL, " ");
 80014d2:	4914      	ldr	r1, [pc, #80]	; (8001524 <edit_text+0x10c>)
 80014d4:	2000      	movs	r0, #0
 80014d6:	f002 f9ef 	bl	80038b8 <strtok>
 80014da:	66b8      	str	r0, [r7, #104]	; 0x68
		i++ ;
 80014dc:	6e7b      	ldr	r3, [r7, #100]	; 0x64
 80014de:	3301      	adds	r3, #1
 80014e0:	667b      	str	r3, [r7, #100]	; 0x64
	while( token != NULL ) {
 80014e2:	6ebb      	ldr	r3, [r7, #104]	; 0x68
 80014e4:	2b00      	cmp	r3, #0
 80014e6:	d1c4      	bne.n	8001472 <edit_text+0x5a>
	}

	// re-set usefull input data buffer
	for(int i = 0; i<DATA_IN_SIZE;i++){
 80014e8:	2300      	movs	r3, #0
 80014ea:	663b      	str	r3, [r7, #96]	; 0x60
 80014ec:	e007      	b.n	80014fe <edit_text+0xe6>
		numtext[i] = 0 ;
 80014ee:	6e3b      	ldr	r3, [r7, #96]	; 0x60
 80014f0:	68ba      	ldr	r2, [r7, #8]
 80014f2:	4413      	add	r3, r2
 80014f4:	2200      	movs	r2, #0
 80014f6:	701a      	strb	r2, [r3, #0]
	for(int i = 0; i<DATA_IN_SIZE;i++){
 80014f8:	6e3b      	ldr	r3, [r7, #96]	; 0x60
 80014fa:	3301      	adds	r3, #1
 80014fc:	663b      	str	r3, [r7, #96]	; 0x60
 80014fe:	6e3b      	ldr	r3, [r7, #96]	; 0x60
 8001500:	2b13      	cmp	r3, #19
 8001502:	ddf4      	ble.n	80014ee <edit_text+0xd6>

	// update index on the data processing string
//	process_idx += RX_bytes ;
//	return ;

}
 8001504:	bf00      	nop
 8001506:	bf00      	nop
 8001508:	3770      	adds	r7, #112	; 0x70
 800150a:	46bd      	mov	sp, r7
 800150c:	bd80      	pop	{r7, pc}
 800150e:	bf00      	nop
 8001510:	20000138 	.word	0x20000138
 8001514:	08004e60 	.word	0x08004e60
 8001518:	408f4000 	.word	0x408f4000
 800151c:	20000130 	.word	0x20000130
 8001520:	20000134 	.word	0x20000134
 8001524:	08004e64 	.word	0x08004e64

08001528 <Error_Handler>:
/**
  * @brief  This function is executed in case of error occurrence.
  * @retval None
  */
void Error_Handler(void)
{
 8001528:	b480      	push	{r7}
 800152a:	af00      	add	r7, sp, #0
  \details Disables IRQ interrupts by setting the I-bit in the CPSR.
           Can only be executed in Privileged modes.
 */
__STATIC_FORCEINLINE void __disable_irq(void)
{
  __ASM volatile ("cpsid i" : : : "memory");
 800152c:	b672      	cpsid	i
}
 800152e:	bf00      	nop
  /* USER CODE BEGIN Error_Handler_Debug */
  /* User can add his own implementation to report the HAL error return state */
  __disable_irq();
  while (1)
 8001530:	e7fe      	b.n	8001530 <Error_Handler+0x8>
	...

08001534 <HAL_MspInit>:
/* USER CODE END 0 */
/**
  * Initializes the Global MSP.
  */
void HAL_MspInit(void)
{
 8001534:	b480      	push	{r7}
 8001536:	b085      	sub	sp, #20
 8001538:	af00      	add	r7, sp, #0
  /* USER CODE BEGIN MspInit 0 */

  /* USER CODE END MspInit 0 */

  __HAL_RCC_AFIO_CLK_ENABLE();
 800153a:	4b15      	ldr	r3, [pc, #84]	; (8001590 <HAL_MspInit+0x5c>)
 800153c:	699b      	ldr	r3, [r3, #24]
 800153e:	4a14      	ldr	r2, [pc, #80]	; (8001590 <HAL_MspInit+0x5c>)
 8001540:	f043 0301 	orr.w	r3, r3, #1
 8001544:	6193      	str	r3, [r2, #24]
 8001546:	4b12      	ldr	r3, [pc, #72]	; (8001590 <HAL_MspInit+0x5c>)
 8001548:	699b      	ldr	r3, [r3, #24]
 800154a:	f003 0301 	and.w	r3, r3, #1
 800154e:	60bb      	str	r3, [r7, #8]
 8001550:	68bb      	ldr	r3, [r7, #8]
  __HAL_RCC_PWR_CLK_ENABLE();
 8001552:	4b0f      	ldr	r3, [pc, #60]	; (8001590 <HAL_MspInit+0x5c>)
 8001554:	69db      	ldr	r3, [r3, #28]
 8001556:	4a0e      	ldr	r2, [pc, #56]	; (8001590 <HAL_MspInit+0x5c>)
 8001558:	f043 5380 	orr.w	r3, r3, #268435456	; 0x10000000
 800155c:	61d3      	str	r3, [r2, #28]
 800155e:	4b0c      	ldr	r3, [pc, #48]	; (8001590 <HAL_MspInit+0x5c>)
 8001560:	69db      	ldr	r3, [r3, #28]
 8001562:	f003 5380 	and.w	r3, r3, #268435456	; 0x10000000
 8001566:	607b      	str	r3, [r7, #4]
 8001568:	687b      	ldr	r3, [r7, #4]

  /* System interrupt init*/

  /** NOJTAG: JTAG-DP Disabled and SW-DP Enabled
  */
  __HAL_AFIO_REMAP_SWJ_NOJTAG();
 800156a:	4b0a      	ldr	r3, [pc, #40]	; (8001594 <HAL_MspInit+0x60>)
 800156c:	685b      	ldr	r3, [r3, #4]
 800156e:	60fb      	str	r3, [r7, #12]
 8001570:	68fb      	ldr	r3, [r7, #12]
 8001572:	f023 63e0 	bic.w	r3, r3, #117440512	; 0x7000000
 8001576:	60fb      	str	r3, [r7, #12]
 8001578:	68fb      	ldr	r3, [r7, #12]
 800157a:	f043 7300 	orr.w	r3, r3, #33554432	; 0x2000000
 800157e:	60fb      	str	r3, [r7, #12]
 8001580:	4a04      	ldr	r2, [pc, #16]	; (8001594 <HAL_MspInit+0x60>)
 8001582:	68fb      	ldr	r3, [r7, #12]
 8001584:	6053      	str	r3, [r2, #4]

  /* USER CODE BEGIN MspInit 1 */

  /* USER CODE END MspInit 1 */
}
 8001586:	bf00      	nop
 8001588:	3714      	adds	r7, #20
 800158a:	46bd      	mov	sp, r7
 800158c:	bc80      	pop	{r7}
 800158e:	4770      	bx	lr
 8001590:	40021000 	.word	0x40021000
 8001594:	40010000 	.word	0x40010000

08001598 <HAL_UART_MspInit>:
* This function configures the hardware resources used in this example
* @param huart: UART handle pointer
* @retval None
*/
void HAL_UART_MspInit(UART_HandleTypeDef* huart)
{
 8001598:	b580      	push	{r7, lr}
 800159a:	b088      	sub	sp, #32
 800159c:	af00      	add	r7, sp, #0
 800159e:	6078      	str	r0, [r7, #4]
  GPIO_InitTypeDef GPIO_InitStruct = {0};
 80015a0:	f107 0310 	add.w	r3, r7, #16
 80015a4:	2200      	movs	r2, #0
 80015a6:	601a      	str	r2, [r3, #0]
 80015a8:	605a      	str	r2, [r3, #4]
 80015aa:	609a      	str	r2, [r3, #8]
 80015ac:	60da      	str	r2, [r3, #12]
  if(huart->Instance==USART2)
 80015ae:	687b      	ldr	r3, [r7, #4]
 80015b0:	681b      	ldr	r3, [r3, #0]
 80015b2:	4a32      	ldr	r2, [pc, #200]	; (800167c <HAL_UART_MspInit+0xe4>)
 80015b4:	4293      	cmp	r3, r2
 80015b6:	d15d      	bne.n	8001674 <HAL_UART_MspInit+0xdc>
  {
  /* USER CODE BEGIN USART2_MspInit 0 */

  /* USER CODE END USART2_MspInit 0 */
    /* Peripheral clock enable */
    __HAL_RCC_USART2_CLK_ENABLE();
 80015b8:	4b31      	ldr	r3, [pc, #196]	; (8001680 <HAL_UART_MspInit+0xe8>)
 80015ba:	69db      	ldr	r3, [r3, #28]
 80015bc:	4a30      	ldr	r2, [pc, #192]	; (8001680 <HAL_UART_MspInit+0xe8>)
 80015be:	f443 3300 	orr.w	r3, r3, #131072	; 0x20000
 80015c2:	61d3      	str	r3, [r2, #28]
 80015c4:	4b2e      	ldr	r3, [pc, #184]	; (8001680 <HAL_UART_MspInit+0xe8>)
 80015c6:	69db      	ldr	r3, [r3, #28]
 80015c8:	f403 3300 	and.w	r3, r3, #131072	; 0x20000
 80015cc:	60fb      	str	r3, [r7, #12]
 80015ce:	68fb      	ldr	r3, [r7, #12]

    __HAL_RCC_GPIOA_CLK_ENABLE();
 80015d0:	4b2b      	ldr	r3, [pc, #172]	; (8001680 <HAL_UART_MspInit+0xe8>)
 80015d2:	699b      	ldr	r3, [r3, #24]
 80015d4:	4a2a      	ldr	r2, [pc, #168]	; (8001680 <HAL_UART_MspInit+0xe8>)
 80015d6:	f043 0304 	orr.w	r3, r3, #4
 80015da:	6193      	str	r3, [r2, #24]
 80015dc:	4b28      	ldr	r3, [pc, #160]	; (8001680 <HAL_UART_MspInit+0xe8>)
 80015de:	699b      	ldr	r3, [r3, #24]
 80015e0:	f003 0304 	and.w	r3, r3, #4
 80015e4:	60bb      	str	r3, [r7, #8]
 80015e6:	68bb      	ldr	r3, [r7, #8]
    /**USART2 GPIO Configuration
    PA2     ------> USART2_TX
    PA3     ------> USART2_RX
    */
    GPIO_InitStruct.Pin = GPIO_PIN_2;
 80015e8:	2304      	movs	r3, #4
 80015ea:	613b      	str	r3, [r7, #16]
    GPIO_InitStruct.Mode = GPIO_MODE_AF_PP;
 80015ec:	2302      	movs	r3, #2
 80015ee:	617b      	str	r3, [r7, #20]
    GPIO_InitStruct.Speed = GPIO_SPEED_FREQ_HIGH;
 80015f0:	2303      	movs	r3, #3
 80015f2:	61fb      	str	r3, [r7, #28]
    HAL_GPIO_Init(GPIOA, &GPIO_InitStruct);
 80015f4:	f107 0310 	add.w	r3, r7, #16
 80015f8:	4619      	mov	r1, r3
 80015fa:	4822      	ldr	r0, [pc, #136]	; (8001684 <HAL_UART_MspInit+0xec>)
 80015fc:	f000 fdaa 	bl	8002154 <HAL_GPIO_Init>

    GPIO_InitStruct.Pin = GPIO_PIN_3;
 8001600:	2308      	movs	r3, #8
 8001602:	613b      	str	r3, [r7, #16]
    GPIO_InitStruct.Mode = GPIO_MODE_INPUT;
 8001604:	2300      	movs	r3, #0
 8001606:	617b      	str	r3, [r7, #20]
    GPIO_InitStruct.Pull = GPIO_NOPULL;
 8001608:	2300      	movs	r3, #0
 800160a:	61bb      	str	r3, [r7, #24]
    HAL_GPIO_Init(GPIOA, &GPIO_InitStruct);
 800160c:	f107 0310 	add.w	r3, r7, #16
 8001610:	4619      	mov	r1, r3
 8001612:	481c      	ldr	r0, [pc, #112]	; (8001684 <HAL_UART_MspInit+0xec>)
 8001614:	f000 fd9e 	bl	8002154 <HAL_GPIO_Init>

    /* USART2 DMA Init */
    /* USART2_RX Init */
    hdma_usart2_rx.Instance = DMA1_Channel6;
 8001618:	4b1b      	ldr	r3, [pc, #108]	; (8001688 <HAL_UART_MspInit+0xf0>)
 800161a:	4a1c      	ldr	r2, [pc, #112]	; (800168c <HAL_UART_MspInit+0xf4>)
 800161c:	601a      	str	r2, [r3, #0]
    hdma_usart2_rx.Init.Direction = DMA_PERIPH_TO_MEMORY;
 800161e:	4b1a      	ldr	r3, [pc, #104]	; (8001688 <HAL_UART_MspInit+0xf0>)
 8001620:	2200      	movs	r2, #0
 8001622:	605a      	str	r2, [r3, #4]
    hdma_usart2_rx.Init.PeriphInc = DMA_PINC_DISABLE;
 8001624:	4b18      	ldr	r3, [pc, #96]	; (8001688 <HAL_UART_MspInit+0xf0>)
 8001626:	2200      	movs	r2, #0
 8001628:	609a      	str	r2, [r3, #8]
    hdma_usart2_rx.Init.MemInc = DMA_MINC_ENABLE;
 800162a:	4b17      	ldr	r3, [pc, #92]	; (8001688 <HAL_UART_MspInit+0xf0>)
 800162c:	2280      	movs	r2, #128	; 0x80
 800162e:	60da      	str	r2, [r3, #12]
    hdma_usart2_rx.Init.PeriphDataAlignment = DMA_PDATAALIGN_BYTE;
 8001630:	4b15      	ldr	r3, [pc, #84]	; (8001688 <HAL_UART_MspInit+0xf0>)
 8001632:	2200      	movs	r2, #0
 8001634:	611a      	str	r2, [r3, #16]
    hdma_usart2_rx.Init.MemDataAlignment = DMA_MDATAALIGN_BYTE;
 8001636:	4b14      	ldr	r3, [pc, #80]	; (8001688 <HAL_UART_MspInit+0xf0>)
 8001638:	2200      	movs	r2, #0
 800163a:	615a      	str	r2, [r3, #20]
    hdma_usart2_rx.Init.Mode = DMA_NORMAL;
 800163c:	4b12      	ldr	r3, [pc, #72]	; (8001688 <HAL_UART_MspInit+0xf0>)
 800163e:	2200      	movs	r2, #0
 8001640:	619a      	str	r2, [r3, #24]
    hdma_usart2_rx.Init.Priority = DMA_PRIORITY_LOW;
 8001642:	4b11      	ldr	r3, [pc, #68]	; (8001688 <HAL_UART_MspInit+0xf0>)
 8001644:	2200      	movs	r2, #0
 8001646:	61da      	str	r2, [r3, #28]
    if (HAL_DMA_Init(&hdma_usart2_rx) != HAL_OK)
 8001648:	480f      	ldr	r0, [pc, #60]	; (8001688 <HAL_UART_MspInit+0xf0>)
 800164a:	f000 fae5 	bl	8001c18 <HAL_DMA_Init>
 800164e:	4603      	mov	r3, r0
 8001650:	2b00      	cmp	r3, #0
 8001652:	d001      	beq.n	8001658 <HAL_UART_MspInit+0xc0>
    {
      Error_Handler();
 8001654:	f7ff ff68 	bl	8001528 <Error_Handler>
    }

    __HAL_LINKDMA(huart,hdmarx,hdma_usart2_rx);
 8001658:	687b      	ldr	r3, [r7, #4]
 800165a:	4a0b      	ldr	r2, [pc, #44]	; (8001688 <HAL_UART_MspInit+0xf0>)
 800165c:	639a      	str	r2, [r3, #56]	; 0x38
 800165e:	4a0a      	ldr	r2, [pc, #40]	; (8001688 <HAL_UART_MspInit+0xf0>)
 8001660:	687b      	ldr	r3, [r7, #4]
 8001662:	6253      	str	r3, [r2, #36]	; 0x24

    /* USART2 interrupt Init */
    HAL_NVIC_SetPriority(USART2_IRQn, 0, 0);
 8001664:	2200      	movs	r2, #0
 8001666:	2100      	movs	r1, #0
 8001668:	2026      	movs	r0, #38	; 0x26
 800166a:	f000 fa9e 	bl	8001baa <HAL_NVIC_SetPriority>
    HAL_NVIC_EnableIRQ(USART2_IRQn);
 800166e:	2026      	movs	r0, #38	; 0x26
 8001670:	f000 fab7 	bl	8001be2 <HAL_NVIC_EnableIRQ>
  /* USER CODE BEGIN USART2_MspInit 1 */

  /* USER CODE END USART2_MspInit 1 */
  }

}
 8001674:	bf00      	nop
 8001676:	3720      	adds	r7, #32
 8001678:	46bd      	mov	sp, r7
 800167a:	bd80      	pop	{r7, pc}
 800167c:	40004400 	.word	0x40004400
 8001680:	40021000 	.word	0x40021000
 8001684:	40010800 	.word	0x40010800
 8001688:	200000dc 	.word	0x200000dc
 800168c:	4002006c 	.word	0x4002006c

08001690 <NMI_Handler>:
/******************************************************************************/
/**
  * @brief This function handles Non maskable interrupt.
  */
void NMI_Handler(void)
{
 8001690:	b480      	push	{r7}
 8001692:	af00      	add	r7, sp, #0
  /* USER CODE BEGIN NonMaskableInt_IRQn 0 */

  /* USER CODE END NonMaskableInt_IRQn 0 */
  /* USER CODE BEGIN NonMaskableInt_IRQn 1 */
  while (1)
 8001694:	e7fe      	b.n	8001694 <NMI_Handler+0x4>

08001696 <HardFault_Handler>:

/**
  * @brief This function handles Hard fault interrupt.
  */
void HardFault_Handler(void)
{
 8001696:	b480      	push	{r7}
 8001698:	af00      	add	r7, sp, #0
  /* USER CODE BEGIN HardFault_IRQn 0 */

  /* USER CODE END HardFault_IRQn 0 */
  while (1)
 800169a:	e7fe      	b.n	800169a <HardFault_Handler+0x4>

0800169c <MemManage_Handler>:

/**
  * @brief This function handles Memory management fault.
  */
void MemManage_Handler(void)
{
 800169c:	b480      	push	{r7}
 800169e:	af00      	add	r7, sp, #0
  /* USER CODE BEGIN MemoryManagement_IRQn 0 */

  /* USER CODE END MemoryManagement_IRQn 0 */
  while (1)
 80016a0:	e7fe      	b.n	80016a0 <MemManage_Handler+0x4>

080016a2 <BusFault_Handler>:

/**
  * @brief This function handles Prefetch fault, memory access fault.
  */
void BusFault_Handler(void)
{
 80016a2:	b480      	push	{r7}
 80016a4:	af00      	add	r7, sp, #0
  /* USER CODE BEGIN BusFault_IRQn 0 */

  /* USER CODE END BusFault_IRQn 0 */
  while (1)
 80016a6:	e7fe      	b.n	80016a6 <BusFault_Handler+0x4>

080016a8 <UsageFault_Handler>:

/**
  * @brief This function handles Undefined instruction or illegal state.
  */
void UsageFault_Handler(void)
{
 80016a8:	b480      	push	{r7}
 80016aa:	af00      	add	r7, sp, #0
  /* USER CODE BEGIN UsageFault_IRQn 0 */

  /* USER CODE END UsageFault_IRQn 0 */
  while (1)
 80016ac:	e7fe      	b.n	80016ac <UsageFault_Handler+0x4>

080016ae <SVC_Handler>:

/**
  * @brief This function handles System service call via SWI instruction.
  */
void SVC_Handler(void)
{
 80016ae:	b480      	push	{r7}
 80016b0:	af00      	add	r7, sp, #0

  /* USER CODE END SVCall_IRQn 0 */
  /* USER CODE BEGIN SVCall_IRQn 1 */

  /* USER CODE END SVCall_IRQn 1 */
}
 80016b2:	bf00      	nop
 80016b4:	46bd      	mov	sp, r7
 80016b6:	bc80      	pop	{r7}
 80016b8:	4770      	bx	lr

080016ba <DebugMon_Handler>:

/**
  * @brief This function handles Debug monitor.
  */
void DebugMon_Handler(void)
{
 80016ba:	b480      	push	{r7}
 80016bc:	af00      	add	r7, sp, #0

  /* USER CODE END DebugMonitor_IRQn 0 */
  /* USER CODE BEGIN DebugMonitor_IRQn 1 */

  /* USER CODE END DebugMonitor_IRQn 1 */
}
 80016be:	bf00      	nop
 80016c0:	46bd      	mov	sp, r7
 80016c2:	bc80      	pop	{r7}
 80016c4:	4770      	bx	lr

080016c6 <PendSV_Handler>:

/**
  * @brief This function handles Pendable request for system service.
  */
void PendSV_Handler(void)
{
 80016c6:	b480      	push	{r7}
 80016c8:	af00      	add	r7, sp, #0

  /* USER CODE END PendSV_IRQn 0 */
  /* USER CODE BEGIN PendSV_IRQn 1 */

  /* USER CODE END PendSV_IRQn 1 */
}
 80016ca:	bf00      	nop
 80016cc:	46bd      	mov	sp, r7
 80016ce:	bc80      	pop	{r7}
 80016d0:	4770      	bx	lr

080016d2 <SysTick_Handler>:

/**
  * @brief This function handles System tick timer.
  */
void SysTick_Handler(void)
{
 80016d2:	b580      	push	{r7, lr}
 80016d4:	af00      	add	r7, sp, #0
  /* USER CODE BEGIN SysTick_IRQn 0 */

  /* USER CODE END SysTick_IRQn 0 */
  HAL_IncTick();
 80016d6:	f000 f951 	bl	800197c <HAL_IncTick>
  /* USER CODE BEGIN SysTick_IRQn 1 */

  /* USER CODE END SysTick_IRQn 1 */
}
 80016da:	bf00      	nop
 80016dc:	bd80      	pop	{r7, pc}
	...

080016e0 <DMA1_Channel6_IRQHandler>:

/**
  * @brief This function handles DMA1 channel6 global interrupt.
  */
void DMA1_Channel6_IRQHandler(void)
{
 80016e0:	b580      	push	{r7, lr}
 80016e2:	af00      	add	r7, sp, #0
  /* USER CODE BEGIN DMA1_Channel6_IRQn 0 */

  /* USER CODE END DMA1_Channel6_IRQn 0 */
  HAL_DMA_IRQHandler(&hdma_usart2_rx);
 80016e4:	4802      	ldr	r0, [pc, #8]	; (80016f0 <DMA1_Channel6_IRQHandler+0x10>)
 80016e6:	f000 fc01 	bl	8001eec <HAL_DMA_IRQHandler>
  /* USER CODE BEGIN DMA1_Channel6_IRQn 1 */

  /* USER CODE END DMA1_Channel6_IRQn 1 */
}
 80016ea:	bf00      	nop
 80016ec:	bd80      	pop	{r7, pc}
 80016ee:	bf00      	nop
 80016f0:	200000dc 	.word	0x200000dc

080016f4 <USART2_IRQHandler>:

/**
  * @brief This function handles USART2 global interrupt.
  */
void USART2_IRQHandler(void)
{
 80016f4:	b580      	push	{r7, lr}
 80016f6:	af00      	add	r7, sp, #0
  /* USER CODE BEGIN USART2_IRQn 0 */

  /* USER CODE END USART2_IRQn 0 */
  HAL_UART_IRQHandler(&huart2);
 80016f8:	4802      	ldr	r0, [pc, #8]	; (8001704 <USART2_IRQHandler+0x10>)
 80016fa:	f001 fbb9 	bl	8002e70 <HAL_UART_IRQHandler>
  /* USER CODE BEGIN USART2_IRQn 1 */

  /* USER CODE END USART2_IRQn 1 */
}
 80016fe:	bf00      	nop
 8001700:	bd80      	pop	{r7, pc}
 8001702:	bf00      	nop
 8001704:	20000098 	.word	0x20000098

08001708 <EXTI15_10_IRQHandler>:

/**
  * @brief This function handles EXTI line[15:10] interrupts.
  */
void EXTI15_10_IRQHandler(void)
{
 8001708:	b580      	push	{r7, lr}
 800170a:	af00      	add	r7, sp, #0
  /* USER CODE BEGIN EXTI15_10_IRQn 0 */

  /* USER CODE END EXTI15_10_IRQn 0 */
  HAL_GPIO_EXTI_IRQHandler(B1_Pin);
 800170c:	f44f 5000 	mov.w	r0, #8192	; 0x2000
 8001710:	f000 fed6 	bl	80024c0 <HAL_GPIO_EXTI_IRQHandler>
  /* USER CODE BEGIN EXTI15_10_IRQn 1 */

  /* USER CODE END EXTI15_10_IRQn 1 */
}
 8001714:	bf00      	nop
 8001716:	bd80      	pop	{r7, pc}

08001718 <_getpid>:
void initialise_monitor_handles()
{
}

int _getpid(void)
{
 8001718:	b480      	push	{r7}
 800171a:	af00      	add	r7, sp, #0
	return 1;
 800171c:	2301      	movs	r3, #1
}
 800171e:	4618      	mov	r0, r3
 8001720:	46bd      	mov	sp, r7
 8001722:	bc80      	pop	{r7}
 8001724:	4770      	bx	lr

08001726 <_kill>:

int _kill(int pid, int sig)
{
 8001726:	b580      	push	{r7, lr}
 8001728:	b082      	sub	sp, #8
 800172a:	af00      	add	r7, sp, #0
 800172c:	6078      	str	r0, [r7, #4]
 800172e:	6039      	str	r1, [r7, #0]
	errno = EINVAL;
 8001730:	f002 f870 	bl	8003814 <__errno>
 8001734:	4603      	mov	r3, r0
 8001736:	2216      	movs	r2, #22
 8001738:	601a      	str	r2, [r3, #0]
	return -1;
 800173a:	f04f 33ff 	mov.w	r3, #4294967295	; 0xffffffff
}
 800173e:	4618      	mov	r0, r3
 8001740:	3708      	adds	r7, #8
 8001742:	46bd      	mov	sp, r7
 8001744:	bd80      	pop	{r7, pc}

08001746 <_exit>:

void _exit (int status)
{
 8001746:	b580      	push	{r7, lr}
 8001748:	b082      	sub	sp, #8
 800174a:	af00      	add	r7, sp, #0
 800174c:	6078      	str	r0, [r7, #4]
	_kill(status, -1);
 800174e:	f04f 31ff 	mov.w	r1, #4294967295	; 0xffffffff
 8001752:	6878      	ldr	r0, [r7, #4]
 8001754:	f7ff ffe7 	bl	8001726 <_kill>
	while (1) {}		/* Make sure we hang here */
 8001758:	e7fe      	b.n	8001758 <_exit+0x12>

0800175a <_read>:
}

__attribute__((weak)) int _read(int file, char *ptr, int len)
{
 800175a:	b580      	push	{r7, lr}
 800175c:	b086      	sub	sp, #24
 800175e:	af00      	add	r7, sp, #0
 8001760:	60f8      	str	r0, [r7, #12]
 8001762:	60b9      	str	r1, [r7, #8]
 8001764:	607a      	str	r2, [r7, #4]
	int DataIdx;

	for (DataIdx = 0; DataIdx < len; DataIdx++)
 8001766:	2300      	movs	r3, #0
 8001768:	617b      	str	r3, [r7, #20]
 800176a:	e00a      	b.n	8001782 <_read+0x28>
	{
		*ptr++ = __io_getchar();
 800176c:	f3af 8000 	nop.w
 8001770:	4601      	mov	r1, r0
 8001772:	68bb      	ldr	r3, [r7, #8]
 8001774:	1c5a      	adds	r2, r3, #1
 8001776:	60ba      	str	r2, [r7, #8]
 8001778:	b2ca      	uxtb	r2, r1
 800177a:	701a      	strb	r2, [r3, #0]
	for (DataIdx = 0; DataIdx < len; DataIdx++)
 800177c:	697b      	ldr	r3, [r7, #20]
 800177e:	3301      	adds	r3, #1
 8001780:	617b      	str	r3, [r7, #20]
 8001782:	697a      	ldr	r2, [r7, #20]
 8001784:	687b      	ldr	r3, [r7, #4]
 8001786:	429a      	cmp	r2, r3
 8001788:	dbf0      	blt.n	800176c <_read+0x12>
	}

return len;
 800178a:	687b      	ldr	r3, [r7, #4]
}
 800178c:	4618      	mov	r0, r3
 800178e:	3718      	adds	r7, #24
 8001790:	46bd      	mov	sp, r7
 8001792:	bd80      	pop	{r7, pc}

08001794 <_write>:

__attribute__((weak)) int _write(int file, char *ptr, int len)
{
 8001794:	b580      	push	{r7, lr}
 8001796:	b086      	sub	sp, #24
 8001798:	af00      	add	r7, sp, #0
 800179a:	60f8      	str	r0, [r7, #12]
 800179c:	60b9      	str	r1, [r7, #8]
 800179e:	607a      	str	r2, [r7, #4]
	int DataIdx;

	for (DataIdx = 0; DataIdx < len; DataIdx++)
 80017a0:	2300      	movs	r3, #0
 80017a2:	617b      	str	r3, [r7, #20]
 80017a4:	e009      	b.n	80017ba <_write+0x26>
	{
		__io_putchar(*ptr++);
 80017a6:	68bb      	ldr	r3, [r7, #8]
 80017a8:	1c5a      	adds	r2, r3, #1
 80017aa:	60ba      	str	r2, [r7, #8]
 80017ac:	781b      	ldrb	r3, [r3, #0]
 80017ae:	4618      	mov	r0, r3
 80017b0:	f3af 8000 	nop.w
	for (DataIdx = 0; DataIdx < len; DataIdx++)
 80017b4:	697b      	ldr	r3, [r7, #20]
 80017b6:	3301      	adds	r3, #1
 80017b8:	617b      	str	r3, [r7, #20]
 80017ba:	697a      	ldr	r2, [r7, #20]
 80017bc:	687b      	ldr	r3, [r7, #4]
 80017be:	429a      	cmp	r2, r3
 80017c0:	dbf1      	blt.n	80017a6 <_write+0x12>
	}
	return len;
 80017c2:	687b      	ldr	r3, [r7, #4]
}
 80017c4:	4618      	mov	r0, r3
 80017c6:	3718      	adds	r7, #24
 80017c8:	46bd      	mov	sp, r7
 80017ca:	bd80      	pop	{r7, pc}

080017cc <_close>:

int _close(int file)
{
 80017cc:	b480      	push	{r7}
 80017ce:	b083      	sub	sp, #12
 80017d0:	af00      	add	r7, sp, #0
 80017d2:	6078      	str	r0, [r7, #4]
	return -1;
 80017d4:	f04f 33ff 	mov.w	r3, #4294967295	; 0xffffffff
}
 80017d8:	4618      	mov	r0, r3
 80017da:	370c      	adds	r7, #12
 80017dc:	46bd      	mov	sp, r7
 80017de:	bc80      	pop	{r7}
 80017e0:	4770      	bx	lr

080017e2 <_fstat>:


int _fstat(int file, struct stat *st)
{
 80017e2:	b480      	push	{r7}
 80017e4:	b083      	sub	sp, #12
 80017e6:	af00      	add	r7, sp, #0
 80017e8:	6078      	str	r0, [r7, #4]
 80017ea:	6039      	str	r1, [r7, #0]
	st->st_mode = S_IFCHR;
 80017ec:	683b      	ldr	r3, [r7, #0]
 80017ee:	f44f 5200 	mov.w	r2, #8192	; 0x2000
 80017f2:	605a      	str	r2, [r3, #4]
	return 0;
 80017f4:	2300      	movs	r3, #0
}
 80017f6:	4618      	mov	r0, r3
 80017f8:	370c      	adds	r7, #12
 80017fa:	46bd      	mov	sp, r7
 80017fc:	bc80      	pop	{r7}
 80017fe:	4770      	bx	lr

08001800 <_isatty>:

int _isatty(int file)
{
 8001800:	b480      	push	{r7}
 8001802:	b083      	sub	sp, #12
 8001804:	af00      	add	r7, sp, #0
 8001806:	6078      	str	r0, [r7, #4]
	return 1;
 8001808:	2301      	movs	r3, #1
}
 800180a:	4618      	mov	r0, r3
 800180c:	370c      	adds	r7, #12
 800180e:	46bd      	mov	sp, r7
 8001810:	bc80      	pop	{r7}
 8001812:	4770      	bx	lr

08001814 <_lseek>:

int _lseek(int file, int ptr, int dir)
{
 8001814:	b480      	push	{r7}
 8001816:	b085      	sub	sp, #20
 8001818:	af00      	add	r7, sp, #0
 800181a:	60f8      	str	r0, [r7, #12]
 800181c:	60b9      	str	r1, [r7, #8]
 800181e:	607a      	str	r2, [r7, #4]
	return 0;
 8001820:	2300      	movs	r3, #0
}
 8001822:	4618      	mov	r0, r3
 8001824:	3714      	adds	r7, #20
 8001826:	46bd      	mov	sp, r7
 8001828:	bc80      	pop	{r7}
 800182a:	4770      	bx	lr

0800182c <_sbrk>:
 *
 * @param incr Memory size
 * @return Pointer to allocated memory
 */
void *_sbrk(ptrdiff_t incr)
{
 800182c:	b580      	push	{r7, lr}
 800182e:	b086      	sub	sp, #24
 8001830:	af00      	add	r7, sp, #0
 8001832:	6078      	str	r0, [r7, #4]
  extern uint8_t _end; /* Symbol defined in the linker script */
  extern uint8_t _estack; /* Symbol defined in the linker script */
  extern uint32_t _Min_Stack_Size; /* Symbol defined in the linker script */
  const uint32_t stack_limit = (uint32_t)&_estack - (uint32_t)&_Min_Stack_Size;
 8001834:	4a14      	ldr	r2, [pc, #80]	; (8001888 <_sbrk+0x5c>)
 8001836:	4b15      	ldr	r3, [pc, #84]	; (800188c <_sbrk+0x60>)
 8001838:	1ad3      	subs	r3, r2, r3
 800183a:	617b      	str	r3, [r7, #20]
  const uint8_t *max_heap = (uint8_t *)stack_limit;
 800183c:	697b      	ldr	r3, [r7, #20]
 800183e:	613b      	str	r3, [r7, #16]
  uint8_t *prev_heap_end;

  /* Initialize heap end at first call */
  if (NULL == __sbrk_heap_end)
 8001840:	4b13      	ldr	r3, [pc, #76]	; (8001890 <_sbrk+0x64>)
 8001842:	681b      	ldr	r3, [r3, #0]
 8001844:	2b00      	cmp	r3, #0
 8001846:	d102      	bne.n	800184e <_sbrk+0x22>
  {
    __sbrk_heap_end = &_end;
 8001848:	4b11      	ldr	r3, [pc, #68]	; (8001890 <_sbrk+0x64>)
 800184a:	4a12      	ldr	r2, [pc, #72]	; (8001894 <_sbrk+0x68>)
 800184c:	601a      	str	r2, [r3, #0]
  }

  /* Protect heap from growing into the reserved MSP stack */
  if (__sbrk_heap_end + incr > max_heap)
 800184e:	4b10      	ldr	r3, [pc, #64]	; (8001890 <_sbrk+0x64>)
 8001850:	681a      	ldr	r2, [r3, #0]
 8001852:	687b      	ldr	r3, [r7, #4]
 8001854:	4413      	add	r3, r2
 8001856:	693a      	ldr	r2, [r7, #16]
 8001858:	429a      	cmp	r2, r3
 800185a:	d207      	bcs.n	800186c <_sbrk+0x40>
  {
    errno = ENOMEM;
 800185c:	f001 ffda 	bl	8003814 <__errno>
 8001860:	4603      	mov	r3, r0
 8001862:	220c      	movs	r2, #12
 8001864:	601a      	str	r2, [r3, #0]
    return (void *)-1;
 8001866:	f04f 33ff 	mov.w	r3, #4294967295	; 0xffffffff
 800186a:	e009      	b.n	8001880 <_sbrk+0x54>
  }

  prev_heap_end = __sbrk_heap_end;
 800186c:	4b08      	ldr	r3, [pc, #32]	; (8001890 <_sbrk+0x64>)
 800186e:	681b      	ldr	r3, [r3, #0]
 8001870:	60fb      	str	r3, [r7, #12]
  __sbrk_heap_end += incr;
 8001872:	4b07      	ldr	r3, [pc, #28]	; (8001890 <_sbrk+0x64>)
 8001874:	681a      	ldr	r2, [r3, #0]
 8001876:	687b      	ldr	r3, [r7, #4]
 8001878:	4413      	add	r3, r2
 800187a:	4a05      	ldr	r2, [pc, #20]	; (8001890 <_sbrk+0x64>)
 800187c:	6013      	str	r3, [r2, #0]

  return (void *)prev_heap_end;
 800187e:	68fb      	ldr	r3, [r7, #12]
}
 8001880:	4618      	mov	r0, r3
 8001882:	3718      	adds	r7, #24
 8001884:	46bd      	mov	sp, r7
 8001886:	bd80      	pop	{r7, pc}
 8001888:	20005000 	.word	0x20005000
 800188c:	00000400 	.word	0x00000400
 8001890:	20000164 	.word	0x20000164
 8001894:	20000180 	.word	0x20000180

08001898 <SystemInit>:
  * @note   This function should be used only after reset.
  * @param  None
  * @retval None
  */
void SystemInit (void)
{
 8001898:	b480      	push	{r7}
 800189a:	af00      	add	r7, sp, #0

  /* Configure the Vector Table location -------------------------------------*/
#if defined(USER_VECT_TAB_ADDRESS)
  SCB->VTOR = VECT_TAB_BASE_ADDRESS | VECT_TAB_OFFSET; /* Vector Table Relocation in Internal SRAM. */
#endif /* USER_VECT_TAB_ADDRESS */
}
 800189c:	bf00      	nop
 800189e:	46bd      	mov	sp, r7
 80018a0:	bc80      	pop	{r7}
 80018a2:	4770      	bx	lr

080018a4 <Reset_Handler>:
  .weak Reset_Handler
  .type Reset_Handler, %function
Reset_Handler:

/* Copy the data segment initializers from flash to SRAM */
  ldr r0, =_sdata
 80018a4:	480c      	ldr	r0, [pc, #48]	; (80018d8 <LoopFillZerobss+0x12>)
  ldr r1, =_edata
 80018a6:	490d      	ldr	r1, [pc, #52]	; (80018dc <LoopFillZerobss+0x16>)
  ldr r2, =_sidata
 80018a8:	4a0d      	ldr	r2, [pc, #52]	; (80018e0 <LoopFillZerobss+0x1a>)
  movs r3, #0
 80018aa:	2300      	movs	r3, #0
  b LoopCopyDataInit
 80018ac:	e002      	b.n	80018b4 <LoopCopyDataInit>

080018ae <CopyDataInit>:

CopyDataInit:
  ldr r4, [r2, r3]
 80018ae:	58d4      	ldr	r4, [r2, r3]
  str r4, [r0, r3]
 80018b0:	50c4      	str	r4, [r0, r3]
  adds r3, r3, #4
 80018b2:	3304      	adds	r3, #4

080018b4 <LoopCopyDataInit>:

LoopCopyDataInit:
  adds r4, r0, r3
 80018b4:	18c4      	adds	r4, r0, r3
  cmp r4, r1
 80018b6:	428c      	cmp	r4, r1
  bcc CopyDataInit
 80018b8:	d3f9      	bcc.n	80018ae <CopyDataInit>
  
/* Zero fill the bss segment. */
  ldr r2, =_sbss
 80018ba:	4a0a      	ldr	r2, [pc, #40]	; (80018e4 <LoopFillZerobss+0x1e>)
  ldr r4, =_ebss
 80018bc:	4c0a      	ldr	r4, [pc, #40]	; (80018e8 <LoopFillZerobss+0x22>)
  movs r3, #0
 80018be:	2300      	movs	r3, #0
  b LoopFillZerobss
 80018c0:	e001      	b.n	80018c6 <LoopFillZerobss>

080018c2 <FillZerobss>:

FillZerobss:
  str  r3, [r2]
 80018c2:	6013      	str	r3, [r2, #0]
  adds r2, r2, #4
 80018c4:	3204      	adds	r2, #4

080018c6 <LoopFillZerobss>:

LoopFillZerobss:
  cmp r2, r4
 80018c6:	42a2      	cmp	r2, r4
  bcc FillZerobss
 80018c8:	d3fb      	bcc.n	80018c2 <FillZerobss>

/* Call the clock system intitialization function.*/
    bl  SystemInit
 80018ca:	f7ff ffe5 	bl	8001898 <SystemInit>
/* Call static constructors */
    bl __libc_init_array
 80018ce:	f001 ffa7 	bl	8003820 <__libc_init_array>
/* Call the application's entry point.*/
  bl main
 80018d2:	f7ff fc15 	bl	8001100 <main>
  bx lr
 80018d6:	4770      	bx	lr
  ldr r0, =_sdata
 80018d8:	20000000 	.word	0x20000000
  ldr r1, =_edata
 80018dc:	2000007c 	.word	0x2000007c
  ldr r2, =_sidata
 80018e0:	080050e0 	.word	0x080050e0
  ldr r2, =_sbss
 80018e4:	2000007c 	.word	0x2000007c
  ldr r4, =_ebss
 80018e8:	2000017c 	.word	0x2000017c

080018ec <ADC1_2_IRQHandler>:
 * @retval : None
*/
    .section .text.Default_Handler,"ax",%progbits
Default_Handler:
Infinite_Loop:
  b Infinite_Loop
 80018ec:	e7fe      	b.n	80018ec <ADC1_2_IRQHandler>
	...

080018f0 <HAL_Init>:
  *         need to ensure that the SysTick time base is always set to 1 millisecond
  *         to have correct HAL operation.
  * @retval HAL status
  */
HAL_StatusTypeDef HAL_Init(void)
{
 80018f0:	b580      	push	{r7, lr}
 80018f2:	af00      	add	r7, sp, #0
    defined(STM32F102x6) || defined(STM32F102xB) || \
    defined(STM32F103x6) || defined(STM32F103xB) || defined(STM32F103xE) || defined(STM32F103xG) || \
    defined(STM32F105xC) || defined(STM32F107xC)

  /* Prefetch buffer is not available on value line devices */
  __HAL_FLASH_PREFETCH_BUFFER_ENABLE();
 80018f4:	4b08      	ldr	r3, [pc, #32]	; (8001918 <HAL_Init+0x28>)
 80018f6:	681b      	ldr	r3, [r3, #0]
 80018f8:	4a07      	ldr	r2, [pc, #28]	; (8001918 <HAL_Init+0x28>)
 80018fa:	f043 0310 	orr.w	r3, r3, #16
 80018fe:	6013      	str	r3, [r2, #0]
#endif
#endif /* PREFETCH_ENABLE */

  /* Set Interrupt Group Priority */
  HAL_NVIC_SetPriorityGrouping(NVIC_PRIORITYGROUP_4);
 8001900:	2003      	movs	r0, #3
 8001902:	f000 f947 	bl	8001b94 <HAL_NVIC_SetPriorityGrouping>

  /* Use systick as time base source and configure 1ms tick (default clock after Reset is HSI) */
  HAL_InitTick(TICK_INT_PRIORITY);
 8001906:	2000      	movs	r0, #0
 8001908:	f000 f808 	bl	800191c <HAL_InitTick>

  /* Init the low level hardware */
  HAL_MspInit();
 800190c:	f7ff fe12 	bl	8001534 <HAL_MspInit>

  /* Return function status */
  return HAL_OK;
 8001910:	2300      	movs	r3, #0
}
 8001912:	4618      	mov	r0, r3
 8001914:	bd80      	pop	{r7, pc}
 8001916:	bf00      	nop
 8001918:	40022000 	.word	0x40022000

0800191c <HAL_InitTick>:
  *       implementation  in user file.
  * @param TickPriority Tick interrupt priority.
  * @retval HAL status
  */
__weak HAL_StatusTypeDef HAL_InitTick(uint32_t TickPriority)
{
 800191c:	b580      	push	{r7, lr}
 800191e:	b082      	sub	sp, #8
 8001920:	af00      	add	r7, sp, #0
 8001922:	6078      	str	r0, [r7, #4]
  /* Configure the SysTick to have interrupt in 1ms time basis*/
  if (HAL_SYSTICK_Config(SystemCoreClock / (1000U / uwTickFreq)) > 0U)
 8001924:	4b12      	ldr	r3, [pc, #72]	; (8001970 <HAL_InitTick+0x54>)
 8001926:	681a      	ldr	r2, [r3, #0]
 8001928:	4b12      	ldr	r3, [pc, #72]	; (8001974 <HAL_InitTick+0x58>)
 800192a:	781b      	ldrb	r3, [r3, #0]
 800192c:	4619      	mov	r1, r3
 800192e:	f44f 737a 	mov.w	r3, #1000	; 0x3e8
 8001932:	fbb3 f3f1 	udiv	r3, r3, r1
 8001936:	fbb2 f3f3 	udiv	r3, r2, r3
 800193a:	4618      	mov	r0, r3
 800193c:	f000 f95f 	bl	8001bfe <HAL_SYSTICK_Config>
 8001940:	4603      	mov	r3, r0
 8001942:	2b00      	cmp	r3, #0
 8001944:	d001      	beq.n	800194a <HAL_InitTick+0x2e>
  {
    return HAL_ERROR;
 8001946:	2301      	movs	r3, #1
 8001948:	e00e      	b.n	8001968 <HAL_InitTick+0x4c>
  }

  /* Configure the SysTick IRQ priority */
  if (TickPriority < (1UL << __NVIC_PRIO_BITS))
 800194a:	687b      	ldr	r3, [r7, #4]
 800194c:	2b0f      	cmp	r3, #15
 800194e:	d80a      	bhi.n	8001966 <HAL_InitTick+0x4a>
  {
    HAL_NVIC_SetPriority(SysTick_IRQn, TickPriority, 0U);
 8001950:	2200      	movs	r2, #0
 8001952:	6879      	ldr	r1, [r7, #4]
 8001954:	f04f 30ff 	mov.w	r0, #4294967295	; 0xffffffff
 8001958:	f000 f927 	bl	8001baa <HAL_NVIC_SetPriority>
    uwTickPrio = TickPriority;
 800195c:	4a06      	ldr	r2, [pc, #24]	; (8001978 <HAL_InitTick+0x5c>)
 800195e:	687b      	ldr	r3, [r7, #4]
 8001960:	6013      	str	r3, [r2, #0]
  {
    return HAL_ERROR;
  }

  /* Return function status */
  return HAL_OK;
 8001962:	2300      	movs	r3, #0
 8001964:	e000      	b.n	8001968 <HAL_InitTick+0x4c>
    return HAL_ERROR;
 8001966:	2301      	movs	r3, #1
}
 8001968:	4618      	mov	r0, r3
 800196a:	3708      	adds	r7, #8
 800196c:	46bd      	mov	sp, r7
 800196e:	bd80      	pop	{r7, pc}
 8001970:	2000000c 	.word	0x2000000c
 8001974:	20000014 	.word	0x20000014
 8001978:	20000010 	.word	0x20000010

0800197c <HAL_IncTick>:
  * @note This function is declared as __weak to be overwritten in case of other
  *      implementations in user file.
  * @retval None
  */
__weak void HAL_IncTick(void)
{
 800197c:	b480      	push	{r7}
 800197e:	af00      	add	r7, sp, #0
  uwTick += uwTickFreq;
 8001980:	4b05      	ldr	r3, [pc, #20]	; (8001998 <HAL_IncTick+0x1c>)
 8001982:	781b      	ldrb	r3, [r3, #0]
 8001984:	461a      	mov	r2, r3
 8001986:	4b05      	ldr	r3, [pc, #20]	; (800199c <HAL_IncTick+0x20>)
 8001988:	681b      	ldr	r3, [r3, #0]
 800198a:	4413      	add	r3, r2
 800198c:	4a03      	ldr	r2, [pc, #12]	; (800199c <HAL_IncTick+0x20>)
 800198e:	6013      	str	r3, [r2, #0]
}
 8001990:	bf00      	nop
 8001992:	46bd      	mov	sp, r7
 8001994:	bc80      	pop	{r7}
 8001996:	4770      	bx	lr
 8001998:	20000014 	.word	0x20000014
 800199c:	20000168 	.word	0x20000168

080019a0 <HAL_GetTick>:
  * @note  This function is declared as __weak to be overwritten in case of other
  *       implementations in user file.
  * @retval tick value
  */
__weak uint32_t HAL_GetTick(void)
{
 80019a0:	b480      	push	{r7}
 80019a2:	af00      	add	r7, sp, #0
  return uwTick;
 80019a4:	4b02      	ldr	r3, [pc, #8]	; (80019b0 <HAL_GetTick+0x10>)
 80019a6:	681b      	ldr	r3, [r3, #0]
}
 80019a8:	4618      	mov	r0, r3
 80019aa:	46bd      	mov	sp, r7
 80019ac:	bc80      	pop	{r7}
 80019ae:	4770      	bx	lr
 80019b0:	20000168 	.word	0x20000168

080019b4 <HAL_Delay>:
  *       implementations in user file.
  * @param Delay specifies the delay time length, in milliseconds.
  * @retval None
  */
__weak void HAL_Delay(uint32_t Delay)
{
 80019b4:	b580      	push	{r7, lr}
 80019b6:	b084      	sub	sp, #16
 80019b8:	af00      	add	r7, sp, #0
 80019ba:	6078      	str	r0, [r7, #4]
  uint32_t tickstart = HAL_GetTick();
 80019bc:	f7ff fff0 	bl	80019a0 <HAL_GetTick>
 80019c0:	60b8      	str	r0, [r7, #8]
  uint32_t wait = Delay;
 80019c2:	687b      	ldr	r3, [r7, #4]
 80019c4:	60fb      	str	r3, [r7, #12]

  /* Add a freq to guarantee minimum wait */
  if (wait < HAL_MAX_DELAY)
 80019c6:	68fb      	ldr	r3, [r7, #12]
 80019c8:	f1b3 3fff 	cmp.w	r3, #4294967295	; 0xffffffff
 80019cc:	d005      	beq.n	80019da <HAL_Delay+0x26>
  {
    wait += (uint32_t)(uwTickFreq);
 80019ce:	4b0a      	ldr	r3, [pc, #40]	; (80019f8 <HAL_Delay+0x44>)
 80019d0:	781b      	ldrb	r3, [r3, #0]
 80019d2:	461a      	mov	r2, r3
 80019d4:	68fb      	ldr	r3, [r7, #12]
 80019d6:	4413      	add	r3, r2
 80019d8:	60fb      	str	r3, [r7, #12]
  }

  while ((HAL_GetTick() - tickstart) < wait)
 80019da:	bf00      	nop
 80019dc:	f7ff ffe0 	bl	80019a0 <HAL_GetTick>
 80019e0:	4602      	mov	r2, r0
 80019e2:	68bb      	ldr	r3, [r7, #8]
 80019e4:	1ad3      	subs	r3, r2, r3
 80019e6:	68fa      	ldr	r2, [r7, #12]
 80019e8:	429a      	cmp	r2, r3
 80019ea:	d8f7      	bhi.n	80019dc <HAL_Delay+0x28>
  {
  }
}
 80019ec:	bf00      	nop
 80019ee:	bf00      	nop
 80019f0:	3710      	adds	r7, #16
 80019f2:	46bd      	mov	sp, r7
 80019f4:	bd80      	pop	{r7, pc}
 80019f6:	bf00      	nop
 80019f8:	20000014 	.word	0x20000014

080019fc <__NVIC_SetPriorityGrouping>:
           In case of a conflict between priority grouping and available
           priority bits (__NVIC_PRIO_BITS), the smallest possible priority group is set.
  \param [in]      PriorityGroup  Priority grouping field.
 */
__STATIC_INLINE void __NVIC_SetPriorityGrouping(uint32_t PriorityGroup)
{
 80019fc:	b480      	push	{r7}
 80019fe:	b085      	sub	sp, #20
 8001a00:	af00      	add	r7, sp, #0
 8001a02:	6078      	str	r0, [r7, #4]
  uint32_t reg_value;
  uint32_t PriorityGroupTmp = (PriorityGroup & (uint32_t)0x07UL);             /* only values 0..7 are used          */
 8001a04:	687b      	ldr	r3, [r7, #4]
 8001a06:	f003 0307 	and.w	r3, r3, #7
 8001a0a:	60fb      	str	r3, [r7, #12]

  reg_value  =  SCB->AIRCR;                                                   /* read old register configuration    */
 8001a0c:	4b0c      	ldr	r3, [pc, #48]	; (8001a40 <__NVIC_SetPriorityGrouping+0x44>)
 8001a0e:	68db      	ldr	r3, [r3, #12]
 8001a10:	60bb      	str	r3, [r7, #8]
  reg_value &= ~((uint32_t)(SCB_AIRCR_VECTKEY_Msk | SCB_AIRCR_PRIGROUP_Msk)); /* clear bits to change               */
 8001a12:	68ba      	ldr	r2, [r7, #8]
 8001a14:	f64f 03ff 	movw	r3, #63743	; 0xf8ff
 8001a18:	4013      	ands	r3, r2
 8001a1a:	60bb      	str	r3, [r7, #8]
  reg_value  =  (reg_value                                   |
                ((uint32_t)0x5FAUL << SCB_AIRCR_VECTKEY_Pos) |
                (PriorityGroupTmp << SCB_AIRCR_PRIGROUP_Pos) );               /* Insert write key and priority group */
 8001a1c:	68fb      	ldr	r3, [r7, #12]
 8001a1e:	021a      	lsls	r2, r3, #8
                ((uint32_t)0x5FAUL << SCB_AIRCR_VECTKEY_Pos) |
 8001a20:	68bb      	ldr	r3, [r7, #8]
 8001a22:	4313      	orrs	r3, r2
  reg_value  =  (reg_value                                   |
 8001a24:	f043 63bf 	orr.w	r3, r3, #100139008	; 0x5f80000
 8001a28:	f443 3300 	orr.w	r3, r3, #131072	; 0x20000
 8001a2c:	60bb      	str	r3, [r7, #8]
  SCB->AIRCR =  reg_value;
 8001a2e:	4a04      	ldr	r2, [pc, #16]	; (8001a40 <__NVIC_SetPriorityGrouping+0x44>)
 8001a30:	68bb      	ldr	r3, [r7, #8]
 8001a32:	60d3      	str	r3, [r2, #12]
}
 8001a34:	bf00      	nop
 8001a36:	3714      	adds	r7, #20
 8001a38:	46bd      	mov	sp, r7
 8001a3a:	bc80      	pop	{r7}
 8001a3c:	4770      	bx	lr
 8001a3e:	bf00      	nop
 8001a40:	e000ed00 	.word	0xe000ed00

08001a44 <__NVIC_GetPriorityGrouping>:
  \brief   Get Priority Grouping
  \details Reads the priority grouping field from the NVIC Interrupt Controller.
  \return                Priority grouping field (SCB->AIRCR [10:8] PRIGROUP field).
 */
__STATIC_INLINE uint32_t __NVIC_GetPriorityGrouping(void)
{
 8001a44:	b480      	push	{r7}
 8001a46:	af00      	add	r7, sp, #0
  return ((uint32_t)((SCB->AIRCR & SCB_AIRCR_PRIGROUP_Msk) >> SCB_AIRCR_PRIGROUP_Pos));
 8001a48:	4b04      	ldr	r3, [pc, #16]	; (8001a5c <__NVIC_GetPriorityGrouping+0x18>)
 8001a4a:	68db      	ldr	r3, [r3, #12]
 8001a4c:	0a1b      	lsrs	r3, r3, #8
 8001a4e:	f003 0307 	and.w	r3, r3, #7
}
 8001a52:	4618      	mov	r0, r3
 8001a54:	46bd      	mov	sp, r7
 8001a56:	bc80      	pop	{r7}
 8001a58:	4770      	bx	lr
 8001a5a:	bf00      	nop
 8001a5c:	e000ed00 	.word	0xe000ed00

08001a60 <__NVIC_EnableIRQ>:
  \details Enables a device specific interrupt in the NVIC interrupt controller.
  \param [in]      IRQn  Device specific interrupt number.
  \note    IRQn must not be negative.
 */
__STATIC_INLINE void __NVIC_EnableIRQ(IRQn_Type IRQn)
{
 8001a60:	b480      	push	{r7}
 8001a62:	b083      	sub	sp, #12
 8001a64:	af00      	add	r7, sp, #0
 8001a66:	4603      	mov	r3, r0
 8001a68:	71fb      	strb	r3, [r7, #7]
  if ((int32_t)(IRQn) >= 0)
 8001a6a:	f997 3007 	ldrsb.w	r3, [r7, #7]
 8001a6e:	2b00      	cmp	r3, #0
 8001a70:	db0b      	blt.n	8001a8a <__NVIC_EnableIRQ+0x2a>
  {
    NVIC->ISER[(((uint32_t)IRQn) >> 5UL)] = (uint32_t)(1UL << (((uint32_t)IRQn) & 0x1FUL));
 8001a72:	79fb      	ldrb	r3, [r7, #7]
 8001a74:	f003 021f 	and.w	r2, r3, #31
 8001a78:	4906      	ldr	r1, [pc, #24]	; (8001a94 <__NVIC_EnableIRQ+0x34>)
 8001a7a:	f997 3007 	ldrsb.w	r3, [r7, #7]
 8001a7e:	095b      	lsrs	r3, r3, #5
 8001a80:	2001      	movs	r0, #1
 8001a82:	fa00 f202 	lsl.w	r2, r0, r2
 8001a86:	f841 2023 	str.w	r2, [r1, r3, lsl #2]
  }
}
 8001a8a:	bf00      	nop
 8001a8c:	370c      	adds	r7, #12
 8001a8e:	46bd      	mov	sp, r7
 8001a90:	bc80      	pop	{r7}
 8001a92:	4770      	bx	lr
 8001a94:	e000e100 	.word	0xe000e100

08001a98 <__NVIC_SetPriority>:
  \param [in]      IRQn  Interrupt number.
  \param [in]  priority  Priority to set.
  \note    The priority cannot be set for every processor exception.
 */
__STATIC_INLINE void __NVIC_SetPriority(IRQn_Type IRQn, uint32_t priority)
{
 8001a98:	b480      	push	{r7}
 8001a9a:	b083      	sub	sp, #12
 8001a9c:	af00      	add	r7, sp, #0
 8001a9e:	4603      	mov	r3, r0
 8001aa0:	6039      	str	r1, [r7, #0]
 8001aa2:	71fb      	strb	r3, [r7, #7]
  if ((int32_t)(IRQn) >= 0)
 8001aa4:	f997 3007 	ldrsb.w	r3, [r7, #7]
 8001aa8:	2b00      	cmp	r3, #0
 8001aaa:	db0a      	blt.n	8001ac2 <__NVIC_SetPriority+0x2a>
  {
    NVIC->IP[((uint32_t)IRQn)]               = (uint8_t)((priority << (8U - __NVIC_PRIO_BITS)) & (uint32_t)0xFFUL);
 8001aac:	683b      	ldr	r3, [r7, #0]
 8001aae:	b2da      	uxtb	r2, r3
 8001ab0:	490c      	ldr	r1, [pc, #48]	; (8001ae4 <__NVIC_SetPriority+0x4c>)
 8001ab2:	f997 3007 	ldrsb.w	r3, [r7, #7]
 8001ab6:	0112      	lsls	r2, r2, #4
 8001ab8:	b2d2      	uxtb	r2, r2
 8001aba:	440b      	add	r3, r1
 8001abc:	f883 2300 	strb.w	r2, [r3, #768]	; 0x300
  }
  else
  {
    SCB->SHP[(((uint32_t)IRQn) & 0xFUL)-4UL] = (uint8_t)((priority << (8U - __NVIC_PRIO_BITS)) & (uint32_t)0xFFUL);
  }
}
 8001ac0:	e00a      	b.n	8001ad8 <__NVIC_SetPriority+0x40>
    SCB->SHP[(((uint32_t)IRQn) & 0xFUL)-4UL] = (uint8_t)((priority << (8U - __NVIC_PRIO_BITS)) & (uint32_t)0xFFUL);
 8001ac2:	683b      	ldr	r3, [r7, #0]
 8001ac4:	b2da      	uxtb	r2, r3
 8001ac6:	4908      	ldr	r1, [pc, #32]	; (8001ae8 <__NVIC_SetPriority+0x50>)
 8001ac8:	79fb      	ldrb	r3, [r7, #7]
 8001aca:	f003 030f 	and.w	r3, r3, #15
 8001ace:	3b04      	subs	r3, #4
 8001ad0:	0112      	lsls	r2, r2, #4
 8001ad2:	b2d2      	uxtb	r2, r2
 8001ad4:	440b      	add	r3, r1
 8001ad6:	761a      	strb	r2, [r3, #24]
}
 8001ad8:	bf00      	nop
 8001ada:	370c      	adds	r7, #12
 8001adc:	46bd      	mov	sp, r7
 8001ade:	bc80      	pop	{r7}
 8001ae0:	4770      	bx	lr
 8001ae2:	bf00      	nop
 8001ae4:	e000e100 	.word	0xe000e100
 8001ae8:	e000ed00 	.word	0xe000ed00

08001aec <NVIC_EncodePriority>:
  \param [in]   PreemptPriority  Preemptive priority value (starting from 0).
  \param [in]       SubPriority  Subpriority value (starting from 0).
  \return                        Encoded priority. Value can be used in the function \ref NVIC_SetPriority().
 */
__STATIC_INLINE uint32_t NVIC_EncodePriority (uint32_t PriorityGroup, uint32_t PreemptPriority, uint32_t SubPriority)
{
 8001aec:	b480      	push	{r7}
 8001aee:	b089      	sub	sp, #36	; 0x24
 8001af0:	af00      	add	r7, sp, #0
 8001af2:	60f8      	str	r0, [r7, #12]
 8001af4:	60b9      	str	r1, [r7, #8]
 8001af6:	607a      	str	r2, [r7, #4]
  uint32_t PriorityGroupTmp = (PriorityGroup & (uint32_t)0x07UL);   /* only values 0..7 are used          */
 8001af8:	68fb      	ldr	r3, [r7, #12]
 8001afa:	f003 0307 	and.w	r3, r3, #7
 8001afe:	61fb      	str	r3, [r7, #28]
  uint32_t PreemptPriorityBits;
  uint32_t SubPriorityBits;

  PreemptPriorityBits = ((7UL - PriorityGroupTmp) > (uint32_t)(__NVIC_PRIO_BITS)) ? (uint32_t)(__NVIC_PRIO_BITS) : (uint32_t)(7UL - PriorityGroupTmp);
 8001b00:	69fb      	ldr	r3, [r7, #28]
 8001b02:	f1c3 0307 	rsb	r3, r3, #7
 8001b06:	2b04      	cmp	r3, #4
 8001b08:	bf28      	it	cs
 8001b0a:	2304      	movcs	r3, #4
 8001b0c:	61bb      	str	r3, [r7, #24]
  SubPriorityBits     = ((PriorityGroupTmp + (uint32_t)(__NVIC_PRIO_BITS)) < (uint32_t)7UL) ? (uint32_t)0UL : (uint32_t)((PriorityGroupTmp - 7UL) + (uint32_t)(__NVIC_PRIO_BITS));
 8001b0e:	69fb      	ldr	r3, [r7, #28]
 8001b10:	3304      	adds	r3, #4
 8001b12:	2b06      	cmp	r3, #6
 8001b14:	d902      	bls.n	8001b1c <NVIC_EncodePriority+0x30>
 8001b16:	69fb      	ldr	r3, [r7, #28]
 8001b18:	3b03      	subs	r3, #3
 8001b1a:	e000      	b.n	8001b1e <NVIC_EncodePriority+0x32>
 8001b1c:	2300      	movs	r3, #0
 8001b1e:	617b      	str	r3, [r7, #20]

  return (
           ((PreemptPriority & (uint32_t)((1UL << (PreemptPriorityBits)) - 1UL)) << SubPriorityBits) |
 8001b20:	f04f 32ff 	mov.w	r2, #4294967295	; 0xffffffff
 8001b24:	69bb      	ldr	r3, [r7, #24]
 8001b26:	fa02 f303 	lsl.w	r3, r2, r3
 8001b2a:	43da      	mvns	r2, r3
 8001b2c:	68bb      	ldr	r3, [r7, #8]
 8001b2e:	401a      	ands	r2, r3
 8001b30:	697b      	ldr	r3, [r7, #20]
 8001b32:	409a      	lsls	r2, r3
           ((SubPriority     & (uint32_t)((1UL << (SubPriorityBits    )) - 1UL)))
 8001b34:	f04f 31ff 	mov.w	r1, #4294967295	; 0xffffffff
 8001b38:	697b      	ldr	r3, [r7, #20]
 8001b3a:	fa01 f303 	lsl.w	r3, r1, r3
 8001b3e:	43d9      	mvns	r1, r3
 8001b40:	687b      	ldr	r3, [r7, #4]
 8001b42:	400b      	ands	r3, r1
           ((PreemptPriority & (uint32_t)((1UL << (PreemptPriorityBits)) - 1UL)) << SubPriorityBits) |
 8001b44:	4313      	orrs	r3, r2
         );
}
 8001b46:	4618      	mov	r0, r3
 8001b48:	3724      	adds	r7, #36	; 0x24
 8001b4a:	46bd      	mov	sp, r7
 8001b4c:	bc80      	pop	{r7}
 8001b4e:	4770      	bx	lr

08001b50 <SysTick_Config>:
  \note    When the variable <b>__Vendor_SysTickConfig</b> is set to 1, then the
           function <b>SysTick_Config</b> is not included. In this case, the file <b><i>device</i>.h</b>
           must contain a vendor-specific implementation of this function.
 */
__STATIC_INLINE uint32_t SysTick_Config(uint32_t ticks)
{
 8001b50:	b580      	push	{r7, lr}
 8001b52:	b082      	sub	sp, #8
 8001b54:	af00      	add	r7, sp, #0
 8001b56:	6078      	str	r0, [r7, #4]
  if ((ticks - 1UL) > SysTick_LOAD_RELOAD_Msk)
 8001b58:	687b      	ldr	r3, [r7, #4]
 8001b5a:	3b01      	subs	r3, #1
 8001b5c:	f1b3 7f80 	cmp.w	r3, #16777216	; 0x1000000
 8001b60:	d301      	bcc.n	8001b66 <SysTick_Config+0x16>
  {
    return (1UL);                                                   /* Reload value impossible */
 8001b62:	2301      	movs	r3, #1
 8001b64:	e00f      	b.n	8001b86 <SysTick_Config+0x36>
  }

  SysTick->LOAD  = (uint32_t)(ticks - 1UL);                         /* set reload register */
 8001b66:	4a0a      	ldr	r2, [pc, #40]	; (8001b90 <SysTick_Config+0x40>)
 8001b68:	687b      	ldr	r3, [r7, #4]
 8001b6a:	3b01      	subs	r3, #1
 8001b6c:	6053      	str	r3, [r2, #4]
  NVIC_SetPriority (SysTick_IRQn, (1UL << __NVIC_PRIO_BITS) - 1UL); /* set Priority for Systick Interrupt */
 8001b6e:	210f      	movs	r1, #15
 8001b70:	f04f 30ff 	mov.w	r0, #4294967295	; 0xffffffff
 8001b74:	f7ff ff90 	bl	8001a98 <__NVIC_SetPriority>
  SysTick->VAL   = 0UL;                                             /* Load the SysTick Counter Value */
 8001b78:	4b05      	ldr	r3, [pc, #20]	; (8001b90 <SysTick_Config+0x40>)
 8001b7a:	2200      	movs	r2, #0
 8001b7c:	609a      	str	r2, [r3, #8]
  SysTick->CTRL  = SysTick_CTRL_CLKSOURCE_Msk |
 8001b7e:	4b04      	ldr	r3, [pc, #16]	; (8001b90 <SysTick_Config+0x40>)
 8001b80:	2207      	movs	r2, #7
 8001b82:	601a      	str	r2, [r3, #0]
                   SysTick_CTRL_TICKINT_Msk   |
                   SysTick_CTRL_ENABLE_Msk;                         /* Enable SysTick IRQ and SysTick Timer */
  return (0UL);                                                     /* Function successful */
 8001b84:	2300      	movs	r3, #0
}
 8001b86:	4618      	mov	r0, r3
 8001b88:	3708      	adds	r7, #8
 8001b8a:	46bd      	mov	sp, r7
 8001b8c:	bd80      	pop	{r7, pc}
 8001b8e:	bf00      	nop
 8001b90:	e000e010 	.word	0xe000e010

08001b94 <HAL_NVIC_SetPriorityGrouping>:
  * @note   When the NVIC_PriorityGroup_0 is selected, IRQ preemption is no more possible. 
  *         The pending IRQ priority will be managed only by the subpriority. 
  * @retval None
  */
void HAL_NVIC_SetPriorityGrouping(uint32_t PriorityGroup)
{
 8001b94:	b580      	push	{r7, lr}
 8001b96:	b082      	sub	sp, #8
 8001b98:	af00      	add	r7, sp, #0
 8001b9a:	6078      	str	r0, [r7, #4]
  /* Check the parameters */
  assert_param(IS_NVIC_PRIORITY_GROUP(PriorityGroup));
  
  /* Set the PRIGROUP[10:8] bits according to the PriorityGroup parameter value */
  NVIC_SetPriorityGrouping(PriorityGroup);
 8001b9c:	6878      	ldr	r0, [r7, #4]
 8001b9e:	f7ff ff2d 	bl	80019fc <__NVIC_SetPriorityGrouping>
}
 8001ba2:	bf00      	nop
 8001ba4:	3708      	adds	r7, #8
 8001ba6:	46bd      	mov	sp, r7
 8001ba8:	bd80      	pop	{r7, pc}

08001baa <HAL_NVIC_SetPriority>:
  *         This parameter can be a value between 0 and 15
  *         A lower priority value indicates a higher priority.          
  * @retval None
  */
void HAL_NVIC_SetPriority(IRQn_Type IRQn, uint32_t PreemptPriority, uint32_t SubPriority)
{ 
 8001baa:	b580      	push	{r7, lr}
 8001bac:	b086      	sub	sp, #24
 8001bae:	af00      	add	r7, sp, #0
 8001bb0:	4603      	mov	r3, r0
 8001bb2:	60b9      	str	r1, [r7, #8]
 8001bb4:	607a      	str	r2, [r7, #4]
 8001bb6:	73fb      	strb	r3, [r7, #15]
  uint32_t prioritygroup = 0x00U;
 8001bb8:	2300      	movs	r3, #0
 8001bba:	617b      	str	r3, [r7, #20]
  
  /* Check the parameters */
  assert_param(IS_NVIC_SUB_PRIORITY(SubPriority));
  assert_param(IS_NVIC_PREEMPTION_PRIORITY(PreemptPriority));
  
  prioritygroup = NVIC_GetPriorityGrouping();
 8001bbc:	f7ff ff42 	bl	8001a44 <__NVIC_GetPriorityGrouping>
 8001bc0:	6178      	str	r0, [r7, #20]
  
  NVIC_SetPriority(IRQn, NVIC_EncodePriority(prioritygroup, PreemptPriority, SubPriority));
 8001bc2:	687a      	ldr	r2, [r7, #4]
 8001bc4:	68b9      	ldr	r1, [r7, #8]
 8001bc6:	6978      	ldr	r0, [r7, #20]
 8001bc8:	f7ff ff90 	bl	8001aec <NVIC_EncodePriority>
 8001bcc:	4602      	mov	r2, r0
 8001bce:	f997 300f 	ldrsb.w	r3, [r7, #15]
 8001bd2:	4611      	mov	r1, r2
 8001bd4:	4618      	mov	r0, r3
 8001bd6:	f7ff ff5f 	bl	8001a98 <__NVIC_SetPriority>
}
 8001bda:	bf00      	nop
 8001bdc:	3718      	adds	r7, #24
 8001bde:	46bd      	mov	sp, r7
 8001be0:	bd80      	pop	{r7, pc}

08001be2 <HAL_NVIC_EnableIRQ>:
  *         This parameter can be an enumerator of IRQn_Type enumeration
  *         (For the complete STM32 Devices IRQ Channels list, please refer to the appropriate CMSIS device file (stm32f10xxx.h))
  * @retval None
  */
void HAL_NVIC_EnableIRQ(IRQn_Type IRQn)
{
 8001be2:	b580      	push	{r7, lr}
 8001be4:	b082      	sub	sp, #8
 8001be6:	af00      	add	r7, sp, #0
 8001be8:	4603      	mov	r3, r0
 8001bea:	71fb      	strb	r3, [r7, #7]
  /* Check the parameters */
  assert_param(IS_NVIC_DEVICE_IRQ(IRQn));

  /* Enable interrupt */
  NVIC_EnableIRQ(IRQn);
 8001bec:	f997 3007 	ldrsb.w	r3, [r7, #7]
 8001bf0:	4618      	mov	r0, r3
 8001bf2:	f7ff ff35 	bl	8001a60 <__NVIC_EnableIRQ>
}
 8001bf6:	bf00      	nop
 8001bf8:	3708      	adds	r7, #8
 8001bfa:	46bd      	mov	sp, r7
 8001bfc:	bd80      	pop	{r7, pc}

08001bfe <HAL_SYSTICK_Config>:
  * @param  TicksNumb: Specifies the ticks Number of ticks between two interrupts.
  * @retval status:  - 0  Function succeeded.
  *                  - 1  Function failed.
  */
uint32_t HAL_SYSTICK_Config(uint32_t TicksNumb)
{
 8001bfe:	b580      	push	{r7, lr}
 8001c00:	b082      	sub	sp, #8
 8001c02:	af00      	add	r7, sp, #0
 8001c04:	6078      	str	r0, [r7, #4]
   return SysTick_Config(TicksNumb);
 8001c06:	6878      	ldr	r0, [r7, #4]
 8001c08:	f7ff ffa2 	bl	8001b50 <SysTick_Config>
 8001c0c:	4603      	mov	r3, r0
}
 8001c0e:	4618      	mov	r0, r3
 8001c10:	3708      	adds	r7, #8
 8001c12:	46bd      	mov	sp, r7
 8001c14:	bd80      	pop	{r7, pc}
	...

08001c18 <HAL_DMA_Init>:
  * @param  hdma: Pointer to a DMA_HandleTypeDef structure that contains
  *               the configuration information for the specified DMA Channel.
  * @retval HAL status
  */
HAL_StatusTypeDef HAL_DMA_Init(DMA_HandleTypeDef *hdma)
{
 8001c18:	b480      	push	{r7}
 8001c1a:	b085      	sub	sp, #20
 8001c1c:	af00      	add	r7, sp, #0
 8001c1e:	6078      	str	r0, [r7, #4]
  uint32_t tmp = 0U;
 8001c20:	2300      	movs	r3, #0
 8001c22:	60fb      	str	r3, [r7, #12]

  /* Check the DMA handle allocation */
  if(hdma == NULL)
 8001c24:	687b      	ldr	r3, [r7, #4]
 8001c26:	2b00      	cmp	r3, #0
 8001c28:	d101      	bne.n	8001c2e <HAL_DMA_Init+0x16>
  {
    return HAL_ERROR;
 8001c2a:	2301      	movs	r3, #1
 8001c2c:	e043      	b.n	8001cb6 <HAL_DMA_Init+0x9e>
    hdma->ChannelIndex = (((uint32_t)hdma->Instance - (uint32_t)DMA2_Channel1) / ((uint32_t)DMA2_Channel2 - (uint32_t)DMA2_Channel1)) << 2;
    hdma->DmaBaseAddress = DMA2;
  }
#else
  /* DMA1 */
  hdma->ChannelIndex = (((uint32_t)hdma->Instance - (uint32_t)DMA1_Channel1) / ((uint32_t)DMA1_Channel2 - (uint32_t)DMA1_Channel1)) << 2;
 8001c2e:	687b      	ldr	r3, [r7, #4]
 8001c30:	681b      	ldr	r3, [r3, #0]
 8001c32:	461a      	mov	r2, r3
 8001c34:	4b22      	ldr	r3, [pc, #136]	; (8001cc0 <HAL_DMA_Init+0xa8>)
 8001c36:	4413      	add	r3, r2
 8001c38:	4a22      	ldr	r2, [pc, #136]	; (8001cc4 <HAL_DMA_Init+0xac>)
 8001c3a:	fba2 2303 	umull	r2, r3, r2, r3
 8001c3e:	091b      	lsrs	r3, r3, #4
 8001c40:	009a      	lsls	r2, r3, #2
 8001c42:	687b      	ldr	r3, [r7, #4]
 8001c44:	641a      	str	r2, [r3, #64]	; 0x40
  hdma->DmaBaseAddress = DMA1;
 8001c46:	687b      	ldr	r3, [r7, #4]
 8001c48:	4a1f      	ldr	r2, [pc, #124]	; (8001cc8 <HAL_DMA_Init+0xb0>)
 8001c4a:	63da      	str	r2, [r3, #60]	; 0x3c
#endif /* DMA2 */

  /* Change DMA peripheral state */
  hdma->State = HAL_DMA_STATE_BUSY;
 8001c4c:	687b      	ldr	r3, [r7, #4]
 8001c4e:	2202      	movs	r2, #2
 8001c50:	f883 2021 	strb.w	r2, [r3, #33]	; 0x21

  /* Get the CR register value */
  tmp = hdma->Instance->CCR;
 8001c54:	687b      	ldr	r3, [r7, #4]
 8001c56:	681b      	ldr	r3, [r3, #0]
 8001c58:	681b      	ldr	r3, [r3, #0]
 8001c5a:	60fb      	str	r3, [r7, #12]

  /* Clear PL, MSIZE, PSIZE, MINC, PINC, CIRC and DIR bits */
  tmp &= ((uint32_t)~(DMA_CCR_PL    | DMA_CCR_MSIZE  | DMA_CCR_PSIZE  | \
 8001c5c:	68fb      	ldr	r3, [r7, #12]
 8001c5e:	f423 537f 	bic.w	r3, r3, #16320	; 0x3fc0
 8001c62:	f023 0330 	bic.w	r3, r3, #48	; 0x30
 8001c66:	60fb      	str	r3, [r7, #12]
                      DMA_CCR_MINC  | DMA_CCR_PINC   | DMA_CCR_CIRC   | \
                      DMA_CCR_DIR));

  /* Prepare the DMA Channel configuration */
  tmp |=  hdma->Init.Direction        |
 8001c68:	687b      	ldr	r3, [r7, #4]
 8001c6a:	685a      	ldr	r2, [r3, #4]
          hdma->Init.PeriphInc           | hdma->Init.MemInc           |
 8001c6c:	687b      	ldr	r3, [r7, #4]
 8001c6e:	689b      	ldr	r3, [r3, #8]
  tmp |=  hdma->Init.Direction        |
 8001c70:	431a      	orrs	r2, r3
          hdma->Init.PeriphInc           | hdma->Init.MemInc           |
 8001c72:	687b      	ldr	r3, [r7, #4]
 8001c74:	68db      	ldr	r3, [r3, #12]
 8001c76:	431a      	orrs	r2, r3
          hdma->Init.PeriphDataAlignment | hdma->Init.MemDataAlignment |
 8001c78:	687b      	ldr	r3, [r7, #4]
 8001c7a:	691b      	ldr	r3, [r3, #16]
          hdma->Init.PeriphInc           | hdma->Init.MemInc           |
 8001c7c:	431a      	orrs	r2, r3
          hdma->Init.PeriphDataAlignment | hdma->Init.MemDataAlignment |
 8001c7e:	687b      	ldr	r3, [r7, #4]
 8001c80:	695b      	ldr	r3, [r3, #20]
 8001c82:	431a      	orrs	r2, r3
          hdma->Init.Mode                | hdma->Init.Priority;
 8001c84:	687b      	ldr	r3, [r7, #4]
 8001c86:	699b      	ldr	r3, [r3, #24]
          hdma->Init.PeriphDataAlignment | hdma->Init.MemDataAlignment |
 8001c88:	431a      	orrs	r2, r3
          hdma->Init.Mode                | hdma->Init.Priority;
 8001c8a:	687b      	ldr	r3, [r7, #4]
 8001c8c:	69db      	ldr	r3, [r3, #28]
 8001c8e:	4313      	orrs	r3, r2
  tmp |=  hdma->Init.Direction        |
 8001c90:	68fa      	ldr	r2, [r7, #12]
 8001c92:	4313      	orrs	r3, r2
 8001c94:	60fb      	str	r3, [r7, #12]

  /* Write to DMA Channel CR register */
  hdma->Instance->CCR = tmp;
 8001c96:	687b      	ldr	r3, [r7, #4]
 8001c98:	681b      	ldr	r3, [r3, #0]
 8001c9a:	68fa      	ldr	r2, [r7, #12]
 8001c9c:	601a      	str	r2, [r3, #0]

  /* Initialise the error code */
  hdma->ErrorCode = HAL_DMA_ERROR_NONE;
 8001c9e:	687b      	ldr	r3, [r7, #4]
 8001ca0:	2200      	movs	r2, #0
 8001ca2:	639a      	str	r2, [r3, #56]	; 0x38

  /* Initialize the DMA state*/
  hdma->State = HAL_DMA_STATE_READY;
 8001ca4:	687b      	ldr	r3, [r7, #4]
 8001ca6:	2201      	movs	r2, #1
 8001ca8:	f883 2021 	strb.w	r2, [r3, #33]	; 0x21
  /* Allocate lock resource and initialize it */
  hdma->Lock = HAL_UNLOCKED;
 8001cac:	687b      	ldr	r3, [r7, #4]
 8001cae:	2200      	movs	r2, #0
 8001cb0:	f883 2020 	strb.w	r2, [r3, #32]

  return HAL_OK;
 8001cb4:	2300      	movs	r3, #0
}
 8001cb6:	4618      	mov	r0, r3
 8001cb8:	3714      	adds	r7, #20
 8001cba:	46bd      	mov	sp, r7
 8001cbc:	bc80      	pop	{r7}
 8001cbe:	4770      	bx	lr
 8001cc0:	bffdfff8 	.word	0xbffdfff8
 8001cc4:	cccccccd 	.word	0xcccccccd
 8001cc8:	40020000 	.word	0x40020000

08001ccc <HAL_DMA_Start_IT>:
  * @param  DstAddress: The destination memory Buffer address
  * @param  DataLength: The length of data to be transferred from source to destination
  * @retval HAL status
  */
HAL_StatusTypeDef HAL_DMA_Start_IT(DMA_HandleTypeDef *hdma, uint32_t SrcAddress, uint32_t DstAddress, uint32_t DataLength)
{
 8001ccc:	b580      	push	{r7, lr}
 8001cce:	b086      	sub	sp, #24
 8001cd0:	af00      	add	r7, sp, #0
 8001cd2:	60f8      	str	r0, [r7, #12]
 8001cd4:	60b9      	str	r1, [r7, #8]
 8001cd6:	607a      	str	r2, [r7, #4]
 8001cd8:	603b      	str	r3, [r7, #0]
  HAL_StatusTypeDef status = HAL_OK;
 8001cda:	2300      	movs	r3, #0
 8001cdc:	75fb      	strb	r3, [r7, #23]

  /* Check the parameters */
  assert_param(IS_DMA_BUFFER_SIZE(DataLength));

  /* Process locked */
  __HAL_LOCK(hdma);
 8001cde:	68fb      	ldr	r3, [r7, #12]
 8001ce0:	f893 3020 	ldrb.w	r3, [r3, #32]
 8001ce4:	2b01      	cmp	r3, #1
 8001ce6:	d101      	bne.n	8001cec <HAL_DMA_Start_IT+0x20>
 8001ce8:	2302      	movs	r3, #2
 8001cea:	e04a      	b.n	8001d82 <HAL_DMA_Start_IT+0xb6>
 8001cec:	68fb      	ldr	r3, [r7, #12]
 8001cee:	2201      	movs	r2, #1
 8001cf0:	f883 2020 	strb.w	r2, [r3, #32]
  
  if(HAL_DMA_STATE_READY == hdma->State)
 8001cf4:	68fb      	ldr	r3, [r7, #12]
 8001cf6:	f893 3021 	ldrb.w	r3, [r3, #33]	; 0x21
 8001cfa:	2b01      	cmp	r3, #1
 8001cfc:	d13a      	bne.n	8001d74 <HAL_DMA_Start_IT+0xa8>
  {
    /* Change DMA peripheral state */
    hdma->State = HAL_DMA_STATE_BUSY;
 8001cfe:	68fb      	ldr	r3, [r7, #12]
 8001d00:	2202      	movs	r2, #2
 8001d02:	f883 2021 	strb.w	r2, [r3, #33]	; 0x21
    hdma->ErrorCode = HAL_DMA_ERROR_NONE;
 8001d06:	68fb      	ldr	r3, [r7, #12]
 8001d08:	2200      	movs	r2, #0
 8001d0a:	639a      	str	r2, [r3, #56]	; 0x38
    
    /* Disable the peripheral */
    __HAL_DMA_DISABLE(hdma);
 8001d0c:	68fb      	ldr	r3, [r7, #12]
 8001d0e:	681b      	ldr	r3, [r3, #0]
 8001d10:	681a      	ldr	r2, [r3, #0]
 8001d12:	68fb      	ldr	r3, [r7, #12]
 8001d14:	681b      	ldr	r3, [r3, #0]
 8001d16:	f022 0201 	bic.w	r2, r2, #1
 8001d1a:	601a      	str	r2, [r3, #0]
    
    /* Configure the source, destination address and the data length & clear flags*/
    DMA_SetConfig(hdma, SrcAddress, DstAddress, DataLength);
 8001d1c:	683b      	ldr	r3, [r7, #0]
 8001d1e:	687a      	ldr	r2, [r7, #4]
 8001d20:	68b9      	ldr	r1, [r7, #8]
 8001d22:	68f8      	ldr	r0, [r7, #12]
 8001d24:	f000 f9e8 	bl	80020f8 <DMA_SetConfig>
    
    /* Enable the transfer complete interrupt */
    /* Enable the transfer Error interrupt */
    if(NULL != hdma->XferHalfCpltCallback)
 8001d28:	68fb      	ldr	r3, [r7, #12]
 8001d2a:	6adb      	ldr	r3, [r3, #44]	; 0x2c
 8001d2c:	2b00      	cmp	r3, #0
 8001d2e:	d008      	beq.n	8001d42 <HAL_DMA_Start_IT+0x76>
    {
      /* Enable the Half transfer complete interrupt as well */
      __HAL_DMA_ENABLE_IT(hdma, (DMA_IT_TC | DMA_IT_HT | DMA_IT_TE));
 8001d30:	68fb      	ldr	r3, [r7, #12]
 8001d32:	681b      	ldr	r3, [r3, #0]
 8001d34:	681a      	ldr	r2, [r3, #0]
 8001d36:	68fb      	ldr	r3, [r7, #12]
 8001d38:	681b      	ldr	r3, [r3, #0]
 8001d3a:	f042 020e 	orr.w	r2, r2, #14
 8001d3e:	601a      	str	r2, [r3, #0]
 8001d40:	e00f      	b.n	8001d62 <HAL_DMA_Start_IT+0x96>
    }
    else
    {
      __HAL_DMA_DISABLE_IT(hdma, DMA_IT_HT);
 8001d42:	68fb      	ldr	r3, [r7, #12]
 8001d44:	681b      	ldr	r3, [r3, #0]
 8001d46:	681a      	ldr	r2, [r3, #0]
 8001d48:	68fb      	ldr	r3, [r7, #12]
 8001d4a:	681b      	ldr	r3, [r3, #0]
 8001d4c:	f022 0204 	bic.w	r2, r2, #4
 8001d50:	601a      	str	r2, [r3, #0]
      __HAL_DMA_ENABLE_IT(hdma, (DMA_IT_TC | DMA_IT_TE));
 8001d52:	68fb      	ldr	r3, [r7, #12]
 8001d54:	681b      	ldr	r3, [r3, #0]
 8001d56:	681a      	ldr	r2, [r3, #0]
 8001d58:	68fb      	ldr	r3, [r7, #12]
 8001d5a:	681b      	ldr	r3, [r3, #0]
 8001d5c:	f042 020a 	orr.w	r2, r2, #10
 8001d60:	601a      	str	r2, [r3, #0]
    }
    /* Enable the Peripheral */
    __HAL_DMA_ENABLE(hdma);
 8001d62:	68fb      	ldr	r3, [r7, #12]
 8001d64:	681b      	ldr	r3, [r3, #0]
 8001d66:	681a      	ldr	r2, [r3, #0]
 8001d68:	68fb      	ldr	r3, [r7, #12]
 8001d6a:	681b      	ldr	r3, [r3, #0]
 8001d6c:	f042 0201 	orr.w	r2, r2, #1
 8001d70:	601a      	str	r2, [r3, #0]
 8001d72:	e005      	b.n	8001d80 <HAL_DMA_Start_IT+0xb4>
  }
  else
  {      
    /* Process Unlocked */
    __HAL_UNLOCK(hdma); 
 8001d74:	68fb      	ldr	r3, [r7, #12]
 8001d76:	2200      	movs	r2, #0
 8001d78:	f883 2020 	strb.w	r2, [r3, #32]

    /* Remain BUSY */
    status = HAL_BUSY;
 8001d7c:	2302      	movs	r3, #2
 8001d7e:	75fb      	strb	r3, [r7, #23]
  }    
  return status;
 8001d80:	7dfb      	ldrb	r3, [r7, #23]
}
 8001d82:	4618      	mov	r0, r3
 8001d84:	3718      	adds	r7, #24
 8001d86:	46bd      	mov	sp, r7
 8001d88:	bd80      	pop	{r7, pc}

08001d8a <HAL_DMA_Abort>:
  * @param  hdma: pointer to a DMA_HandleTypeDef structure that contains
  *               the configuration information for the specified DMA Channel.
  * @retval HAL status
  */
HAL_StatusTypeDef HAL_DMA_Abort(DMA_HandleTypeDef *hdma)
{
 8001d8a:	b480      	push	{r7}
 8001d8c:	b085      	sub	sp, #20
 8001d8e:	af00      	add	r7, sp, #0
 8001d90:	6078      	str	r0, [r7, #4]
  HAL_StatusTypeDef status = HAL_OK;
 8001d92:	2300      	movs	r3, #0
 8001d94:	73fb      	strb	r3, [r7, #15]
  
  if(hdma->State != HAL_DMA_STATE_BUSY)
 8001d96:	687b      	ldr	r3, [r7, #4]
 8001d98:	f893 3021 	ldrb.w	r3, [r3, #33]	; 0x21
 8001d9c:	2b02      	cmp	r3, #2
 8001d9e:	d008      	beq.n	8001db2 <HAL_DMA_Abort+0x28>
  {
    /* no transfer ongoing */
    hdma->ErrorCode = HAL_DMA_ERROR_NO_XFER;
 8001da0:	687b      	ldr	r3, [r7, #4]
 8001da2:	2204      	movs	r2, #4
 8001da4:	639a      	str	r2, [r3, #56]	; 0x38
    
    /* Process Unlocked */
    __HAL_UNLOCK(hdma);
 8001da6:	687b      	ldr	r3, [r7, #4]
 8001da8:	2200      	movs	r2, #0
 8001daa:	f883 2020 	strb.w	r2, [r3, #32]
    
    return HAL_ERROR;
 8001dae:	2301      	movs	r3, #1
 8001db0:	e020      	b.n	8001df4 <HAL_DMA_Abort+0x6a>
  }
  else

  {
    /* Disable DMA IT */
    __HAL_DMA_DISABLE_IT(hdma, (DMA_IT_TC | DMA_IT_HT | DMA_IT_TE));
 8001db2:	687b      	ldr	r3, [r7, #4]
 8001db4:	681b      	ldr	r3, [r3, #0]
 8001db6:	681a      	ldr	r2, [r3, #0]
 8001db8:	687b      	ldr	r3, [r7, #4]
 8001dba:	681b      	ldr	r3, [r3, #0]
 8001dbc:	f022 020e 	bic.w	r2, r2, #14
 8001dc0:	601a      	str	r2, [r3, #0]
      
    /* Disable the channel */
    __HAL_DMA_DISABLE(hdma);
 8001dc2:	687b      	ldr	r3, [r7, #4]
 8001dc4:	681b      	ldr	r3, [r3, #0]
 8001dc6:	681a      	ldr	r2, [r3, #0]
 8001dc8:	687b      	ldr	r3, [r7, #4]
 8001dca:	681b      	ldr	r3, [r3, #0]
 8001dcc:	f022 0201 	bic.w	r2, r2, #1
 8001dd0:	601a      	str	r2, [r3, #0]
      
    /* Clear all flags */
    hdma->DmaBaseAddress->IFCR = (DMA_ISR_GIF1 << hdma->ChannelIndex);
 8001dd2:	687b      	ldr	r3, [r7, #4]
 8001dd4:	6c1a      	ldr	r2, [r3, #64]	; 0x40
 8001dd6:	687b      	ldr	r3, [r7, #4]
 8001dd8:	6bdb      	ldr	r3, [r3, #60]	; 0x3c
 8001dda:	2101      	movs	r1, #1
 8001ddc:	fa01 f202 	lsl.w	r2, r1, r2
 8001de0:	605a      	str	r2, [r3, #4]
  }
  /* Change the DMA state */
  hdma->State = HAL_DMA_STATE_READY;
 8001de2:	687b      	ldr	r3, [r7, #4]
 8001de4:	2201      	movs	r2, #1
 8001de6:	f883 2021 	strb.w	r2, [r3, #33]	; 0x21

  /* Process Unlocked */
  __HAL_UNLOCK(hdma);      
 8001dea:	687b      	ldr	r3, [r7, #4]
 8001dec:	2200      	movs	r2, #0
 8001dee:	f883 2020 	strb.w	r2, [r3, #32]
  
  return status; 
 8001df2:	7bfb      	ldrb	r3, [r7, #15]
}
 8001df4:	4618      	mov	r0, r3
 8001df6:	3714      	adds	r7, #20
 8001df8:	46bd      	mov	sp, r7
 8001dfa:	bc80      	pop	{r7}
 8001dfc:	4770      	bx	lr
	...

08001e00 <HAL_DMA_Abort_IT>:
  * @param  hdma  : pointer to a DMA_HandleTypeDef structure that contains
  *                 the configuration information for the specified DMA Channel.
  * @retval HAL status
  */
HAL_StatusTypeDef HAL_DMA_Abort_IT(DMA_HandleTypeDef *hdma)
{  
 8001e00:	b580      	push	{r7, lr}
 8001e02:	b084      	sub	sp, #16
 8001e04:	af00      	add	r7, sp, #0
 8001e06:	6078      	str	r0, [r7, #4]
  HAL_StatusTypeDef status = HAL_OK;
 8001e08:	2300      	movs	r3, #0
 8001e0a:	73fb      	strb	r3, [r7, #15]
  
  if(HAL_DMA_STATE_BUSY != hdma->State)
 8001e0c:	687b      	ldr	r3, [r7, #4]
 8001e0e:	f893 3021 	ldrb.w	r3, [r3, #33]	; 0x21
 8001e12:	2b02      	cmp	r3, #2
 8001e14:	d005      	beq.n	8001e22 <HAL_DMA_Abort_IT+0x22>
  {
    /* no transfer ongoing */
    hdma->ErrorCode = HAL_DMA_ERROR_NO_XFER;
 8001e16:	687b      	ldr	r3, [r7, #4]
 8001e18:	2204      	movs	r2, #4
 8001e1a:	639a      	str	r2, [r3, #56]	; 0x38
        
    status = HAL_ERROR;
 8001e1c:	2301      	movs	r3, #1
 8001e1e:	73fb      	strb	r3, [r7, #15]
 8001e20:	e051      	b.n	8001ec6 <HAL_DMA_Abort_IT+0xc6>
  }
  else
  { 
    /* Disable DMA IT */
    __HAL_DMA_DISABLE_IT(hdma, (DMA_IT_TC | DMA_IT_HT | DMA_IT_TE));
 8001e22:	687b      	ldr	r3, [r7, #4]
 8001e24:	681b      	ldr	r3, [r3, #0]
 8001e26:	681a      	ldr	r2, [r3, #0]
 8001e28:	687b      	ldr	r3, [r7, #4]
 8001e2a:	681b      	ldr	r3, [r3, #0]
 8001e2c:	f022 020e 	bic.w	r2, r2, #14
 8001e30:	601a      	str	r2, [r3, #0]

    /* Disable the channel */
    __HAL_DMA_DISABLE(hdma);
 8001e32:	687b      	ldr	r3, [r7, #4]
 8001e34:	681b      	ldr	r3, [r3, #0]
 8001e36:	681a      	ldr	r2, [r3, #0]
 8001e38:	687b      	ldr	r3, [r7, #4]
 8001e3a:	681b      	ldr	r3, [r3, #0]
 8001e3c:	f022 0201 	bic.w	r2, r2, #1
 8001e40:	601a      	str	r2, [r3, #0]

    /* Clear all flags */
    __HAL_DMA_CLEAR_FLAG(hdma, __HAL_DMA_GET_GI_FLAG_INDEX(hdma));
 8001e42:	687b      	ldr	r3, [r7, #4]
 8001e44:	681b      	ldr	r3, [r3, #0]
 8001e46:	4a22      	ldr	r2, [pc, #136]	; (8001ed0 <HAL_DMA_Abort_IT+0xd0>)
 8001e48:	4293      	cmp	r3, r2
 8001e4a:	d029      	beq.n	8001ea0 <HAL_DMA_Abort_IT+0xa0>
 8001e4c:	687b      	ldr	r3, [r7, #4]
 8001e4e:	681b      	ldr	r3, [r3, #0]
 8001e50:	4a20      	ldr	r2, [pc, #128]	; (8001ed4 <HAL_DMA_Abort_IT+0xd4>)
 8001e52:	4293      	cmp	r3, r2
 8001e54:	d022      	beq.n	8001e9c <HAL_DMA_Abort_IT+0x9c>
 8001e56:	687b      	ldr	r3, [r7, #4]
 8001e58:	681b      	ldr	r3, [r3, #0]
 8001e5a:	4a1f      	ldr	r2, [pc, #124]	; (8001ed8 <HAL_DMA_Abort_IT+0xd8>)
 8001e5c:	4293      	cmp	r3, r2
 8001e5e:	d01a      	beq.n	8001e96 <HAL_DMA_Abort_IT+0x96>
 8001e60:	687b      	ldr	r3, [r7, #4]
 8001e62:	681b      	ldr	r3, [r3, #0]
 8001e64:	4a1d      	ldr	r2, [pc, #116]	; (8001edc <HAL_DMA_Abort_IT+0xdc>)
 8001e66:	4293      	cmp	r3, r2
 8001e68:	d012      	beq.n	8001e90 <HAL_DMA_Abort_IT+0x90>
 8001e6a:	687b      	ldr	r3, [r7, #4]
 8001e6c:	681b      	ldr	r3, [r3, #0]
 8001e6e:	4a1c      	ldr	r2, [pc, #112]	; (8001ee0 <HAL_DMA_Abort_IT+0xe0>)
 8001e70:	4293      	cmp	r3, r2
 8001e72:	d00a      	beq.n	8001e8a <HAL_DMA_Abort_IT+0x8a>
 8001e74:	687b      	ldr	r3, [r7, #4]
 8001e76:	681b      	ldr	r3, [r3, #0]
 8001e78:	4a1a      	ldr	r2, [pc, #104]	; (8001ee4 <HAL_DMA_Abort_IT+0xe4>)
 8001e7a:	4293      	cmp	r3, r2
 8001e7c:	d102      	bne.n	8001e84 <HAL_DMA_Abort_IT+0x84>
 8001e7e:	f44f 1380 	mov.w	r3, #1048576	; 0x100000
 8001e82:	e00e      	b.n	8001ea2 <HAL_DMA_Abort_IT+0xa2>
 8001e84:	f04f 7380 	mov.w	r3, #16777216	; 0x1000000
 8001e88:	e00b      	b.n	8001ea2 <HAL_DMA_Abort_IT+0xa2>
 8001e8a:	f44f 3380 	mov.w	r3, #65536	; 0x10000
 8001e8e:	e008      	b.n	8001ea2 <HAL_DMA_Abort_IT+0xa2>
 8001e90:	f44f 5380 	mov.w	r3, #4096	; 0x1000
 8001e94:	e005      	b.n	8001ea2 <HAL_DMA_Abort_IT+0xa2>
 8001e96:	f44f 7380 	mov.w	r3, #256	; 0x100
 8001e9a:	e002      	b.n	8001ea2 <HAL_DMA_Abort_IT+0xa2>
 8001e9c:	2310      	movs	r3, #16
 8001e9e:	e000      	b.n	8001ea2 <HAL_DMA_Abort_IT+0xa2>
 8001ea0:	2301      	movs	r3, #1
 8001ea2:	4a11      	ldr	r2, [pc, #68]	; (8001ee8 <HAL_DMA_Abort_IT+0xe8>)
 8001ea4:	6053      	str	r3, [r2, #4]

    /* Change the DMA state */
    hdma->State = HAL_DMA_STATE_READY;
 8001ea6:	687b      	ldr	r3, [r7, #4]
 8001ea8:	2201      	movs	r2, #1
 8001eaa:	f883 2021 	strb.w	r2, [r3, #33]	; 0x21

    /* Process Unlocked */
    __HAL_UNLOCK(hdma);
 8001eae:	687b      	ldr	r3, [r7, #4]
 8001eb0:	2200      	movs	r2, #0
 8001eb2:	f883 2020 	strb.w	r2, [r3, #32]

    /* Call User Abort callback */
    if(hdma->XferAbortCallback != NULL)
 8001eb6:	687b      	ldr	r3, [r7, #4]
 8001eb8:	6b5b      	ldr	r3, [r3, #52]	; 0x34
 8001eba:	2b00      	cmp	r3, #0
 8001ebc:	d003      	beq.n	8001ec6 <HAL_DMA_Abort_IT+0xc6>
    {
      hdma->XferAbortCallback(hdma);
 8001ebe:	687b      	ldr	r3, [r7, #4]
 8001ec0:	6b5b      	ldr	r3, [r3, #52]	; 0x34
 8001ec2:	6878      	ldr	r0, [r7, #4]
 8001ec4:	4798      	blx	r3
    } 
  }
  return status;
 8001ec6:	7bfb      	ldrb	r3, [r7, #15]
}
 8001ec8:	4618      	mov	r0, r3
 8001eca:	3710      	adds	r7, #16
 8001ecc:	46bd      	mov	sp, r7
 8001ece:	bd80      	pop	{r7, pc}
 8001ed0:	40020008 	.word	0x40020008
 8001ed4:	4002001c 	.word	0x4002001c
 8001ed8:	40020030 	.word	0x40020030
 8001edc:	40020044 	.word	0x40020044
 8001ee0:	40020058 	.word	0x40020058
 8001ee4:	4002006c 	.word	0x4002006c
 8001ee8:	40020000 	.word	0x40020000

08001eec <HAL_DMA_IRQHandler>:
  * @param  hdma: pointer to a DMA_HandleTypeDef structure that contains
  *               the configuration information for the specified DMA Channel.  
  * @retval None
  */
void HAL_DMA_IRQHandler(DMA_HandleTypeDef *hdma)
{
 8001eec:	b580      	push	{r7, lr}
 8001eee:	b084      	sub	sp, #16
 8001ef0:	af00      	add	r7, sp, #0
 8001ef2:	6078      	str	r0, [r7, #4]
  uint32_t flag_it = hdma->DmaBaseAddress->ISR;
 8001ef4:	687b      	ldr	r3, [r7, #4]
 8001ef6:	6bdb      	ldr	r3, [r3, #60]	; 0x3c
 8001ef8:	681b      	ldr	r3, [r3, #0]
 8001efa:	60fb      	str	r3, [r7, #12]
  uint32_t source_it = hdma->Instance->CCR;
 8001efc:	687b      	ldr	r3, [r7, #4]
 8001efe:	681b      	ldr	r3, [r3, #0]
 8001f00:	681b      	ldr	r3, [r3, #0]
 8001f02:	60bb      	str	r3, [r7, #8]
  
  /* Half Transfer Complete Interrupt management ******************************/
  if (((flag_it & (DMA_FLAG_HT1 << hdma->ChannelIndex)) != RESET) && ((source_it & DMA_IT_HT) != RESET))
 8001f04:	687b      	ldr	r3, [r7, #4]
 8001f06:	6c1b      	ldr	r3, [r3, #64]	; 0x40
 8001f08:	2204      	movs	r2, #4
 8001f0a:	409a      	lsls	r2, r3
 8001f0c:	68fb      	ldr	r3, [r7, #12]
 8001f0e:	4013      	ands	r3, r2
 8001f10:	2b00      	cmp	r3, #0
 8001f12:	d04f      	beq.n	8001fb4 <HAL_DMA_IRQHandler+0xc8>
 8001f14:	68bb      	ldr	r3, [r7, #8]
 8001f16:	f003 0304 	and.w	r3, r3, #4
 8001f1a:	2b00      	cmp	r3, #0
 8001f1c:	d04a      	beq.n	8001fb4 <HAL_DMA_IRQHandler+0xc8>
  {
    /* Disable the half transfer interrupt if the DMA mode is not CIRCULAR */
    if((hdma->Instance->CCR & DMA_CCR_CIRC) == 0U)
 8001f1e:	687b      	ldr	r3, [r7, #4]
 8001f20:	681b      	ldr	r3, [r3, #0]
 8001f22:	681b      	ldr	r3, [r3, #0]
 8001f24:	f003 0320 	and.w	r3, r3, #32
 8001f28:	2b00      	cmp	r3, #0
 8001f2a:	d107      	bne.n	8001f3c <HAL_DMA_IRQHandler+0x50>
    {
      /* Disable the half transfer interrupt */
      __HAL_DMA_DISABLE_IT(hdma, DMA_IT_HT);
 8001f2c:	687b      	ldr	r3, [r7, #4]
 8001f2e:	681b      	ldr	r3, [r3, #0]
 8001f30:	681a      	ldr	r2, [r3, #0]
 8001f32:	687b      	ldr	r3, [r7, #4]
 8001f34:	681b      	ldr	r3, [r3, #0]
 8001f36:	f022 0204 	bic.w	r2, r2, #4
 8001f3a:	601a      	str	r2, [r3, #0]
    }
    /* Clear the half transfer complete flag */
    __HAL_DMA_CLEAR_FLAG(hdma, __HAL_DMA_GET_HT_FLAG_INDEX(hdma));
 8001f3c:	687b      	ldr	r3, [r7, #4]
 8001f3e:	681b      	ldr	r3, [r3, #0]
 8001f40:	4a66      	ldr	r2, [pc, #408]	; (80020dc <HAL_DMA_IRQHandler+0x1f0>)
 8001f42:	4293      	cmp	r3, r2
 8001f44:	d029      	beq.n	8001f9a <HAL_DMA_IRQHandler+0xae>
 8001f46:	687b      	ldr	r3, [r7, #4]
 8001f48:	681b      	ldr	r3, [r3, #0]
 8001f4a:	4a65      	ldr	r2, [pc, #404]	; (80020e0 <HAL_DMA_IRQHandler+0x1f4>)
 8001f4c:	4293      	cmp	r3, r2
 8001f4e:	d022      	beq.n	8001f96 <HAL_DMA_IRQHandler+0xaa>
 8001f50:	687b      	ldr	r3, [r7, #4]
 8001f52:	681b      	ldr	r3, [r3, #0]
 8001f54:	4a63      	ldr	r2, [pc, #396]	; (80020e4 <HAL_DMA_IRQHandler+0x1f8>)
 8001f56:	4293      	cmp	r3, r2
 8001f58:	d01a      	beq.n	8001f90 <HAL_DMA_IRQHandler+0xa4>
 8001f5a:	687b      	ldr	r3, [r7, #4]
 8001f5c:	681b      	ldr	r3, [r3, #0]
 8001f5e:	4a62      	ldr	r2, [pc, #392]	; (80020e8 <HAL_DMA_IRQHandler+0x1fc>)
 8001f60:	4293      	cmp	r3, r2
 8001f62:	d012      	beq.n	8001f8a <HAL_DMA_IRQHandler+0x9e>
 8001f64:	687b      	ldr	r3, [r7, #4]
 8001f66:	681b      	ldr	r3, [r3, #0]
 8001f68:	4a60      	ldr	r2, [pc, #384]	; (80020ec <HAL_DMA_IRQHandler+0x200>)
 8001f6a:	4293      	cmp	r3, r2
 8001f6c:	d00a      	beq.n	8001f84 <HAL_DMA_IRQHandler+0x98>
 8001f6e:	687b      	ldr	r3, [r7, #4]
 8001f70:	681b      	ldr	r3, [r3, #0]
 8001f72:	4a5f      	ldr	r2, [pc, #380]	; (80020f0 <HAL_DMA_IRQHandler+0x204>)
 8001f74:	4293      	cmp	r3, r2
 8001f76:	d102      	bne.n	8001f7e <HAL_DMA_IRQHandler+0x92>
 8001f78:	f44f 0380 	mov.w	r3, #4194304	; 0x400000
 8001f7c:	e00e      	b.n	8001f9c <HAL_DMA_IRQHandler+0xb0>
 8001f7e:	f04f 6380 	mov.w	r3, #67108864	; 0x4000000
 8001f82:	e00b      	b.n	8001f9c <HAL_DMA_IRQHandler+0xb0>
 8001f84:	f44f 2380 	mov.w	r3, #262144	; 0x40000
 8001f88:	e008      	b.n	8001f9c <HAL_DMA_IRQHandler+0xb0>
 8001f8a:	f44f 4380 	mov.w	r3, #16384	; 0x4000
 8001f8e:	e005      	b.n	8001f9c <HAL_DMA_IRQHandler+0xb0>
 8001f90:	f44f 6380 	mov.w	r3, #1024	; 0x400
 8001f94:	e002      	b.n	8001f9c <HAL_DMA_IRQHandler+0xb0>
 8001f96:	2340      	movs	r3, #64	; 0x40
 8001f98:	e000      	b.n	8001f9c <HAL_DMA_IRQHandler+0xb0>
 8001f9a:	2304      	movs	r3, #4
 8001f9c:	4a55      	ldr	r2, [pc, #340]	; (80020f4 <HAL_DMA_IRQHandler+0x208>)
 8001f9e:	6053      	str	r3, [r2, #4]

    /* DMA peripheral state is not updated in Half Transfer */
    /* but in Transfer Complete case */

    if(hdma->XferHalfCpltCallback != NULL)
 8001fa0:	687b      	ldr	r3, [r7, #4]
 8001fa2:	6adb      	ldr	r3, [r3, #44]	; 0x2c
 8001fa4:	2b00      	cmp	r3, #0
 8001fa6:	f000 8094 	beq.w	80020d2 <HAL_DMA_IRQHandler+0x1e6>
    {
      /* Half transfer callback */
      hdma->XferHalfCpltCallback(hdma);
 8001faa:	687b      	ldr	r3, [r7, #4]
 8001fac:	6adb      	ldr	r3, [r3, #44]	; 0x2c
 8001fae:	6878      	ldr	r0, [r7, #4]
 8001fb0:	4798      	blx	r3
    if(hdma->XferHalfCpltCallback != NULL)
 8001fb2:	e08e      	b.n	80020d2 <HAL_DMA_IRQHandler+0x1e6>
    }
  }

  /* Transfer Complete Interrupt management ***********************************/
  else if (((flag_it & (DMA_FLAG_TC1 << hdma->ChannelIndex)) != RESET) && ((source_it & DMA_IT_TC) != RESET))
 8001fb4:	687b      	ldr	r3, [r7, #4]
 8001fb6:	6c1b      	ldr	r3, [r3, #64]	; 0x40
 8001fb8:	2202      	movs	r2, #2
 8001fba:	409a      	lsls	r2, r3
 8001fbc:	68fb      	ldr	r3, [r7, #12]
 8001fbe:	4013      	ands	r3, r2
 8001fc0:	2b00      	cmp	r3, #0
 8001fc2:	d056      	beq.n	8002072 <HAL_DMA_IRQHandler+0x186>
 8001fc4:	68bb      	ldr	r3, [r7, #8]
 8001fc6:	f003 0302 	and.w	r3, r3, #2
 8001fca:	2b00      	cmp	r3, #0
 8001fcc:	d051      	beq.n	8002072 <HAL_DMA_IRQHandler+0x186>
  {
    if((hdma->Instance->CCR & DMA_CCR_CIRC) == 0U)
 8001fce:	687b      	ldr	r3, [r7, #4]
 8001fd0:	681b      	ldr	r3, [r3, #0]
 8001fd2:	681b      	ldr	r3, [r3, #0]
 8001fd4:	f003 0320 	and.w	r3, r3, #32
 8001fd8:	2b00      	cmp	r3, #0
 8001fda:	d10b      	bne.n	8001ff4 <HAL_DMA_IRQHandler+0x108>
    {
      /* Disable the transfer complete and error interrupt */
      __HAL_DMA_DISABLE_IT(hdma, DMA_IT_TE | DMA_IT_TC);  
 8001fdc:	687b      	ldr	r3, [r7, #4]
 8001fde:	681b      	ldr	r3, [r3, #0]
 8001fe0:	681a      	ldr	r2, [r3, #0]
 8001fe2:	687b      	ldr	r3, [r7, #4]
 8001fe4:	681b      	ldr	r3, [r3, #0]
 8001fe6:	f022 020a 	bic.w	r2, r2, #10
 8001fea:	601a      	str	r2, [r3, #0]

      /* Change the DMA state */
      hdma->State = HAL_DMA_STATE_READY;
 8001fec:	687b      	ldr	r3, [r7, #4]
 8001fee:	2201      	movs	r2, #1
 8001ff0:	f883 2021 	strb.w	r2, [r3, #33]	; 0x21
    }
    /* Clear the transfer complete flag */
      __HAL_DMA_CLEAR_FLAG(hdma, __HAL_DMA_GET_TC_FLAG_INDEX(hdma));
 8001ff4:	687b      	ldr	r3, [r7, #4]
 8001ff6:	681b      	ldr	r3, [r3, #0]
 8001ff8:	4a38      	ldr	r2, [pc, #224]	; (80020dc <HAL_DMA_IRQHandler+0x1f0>)
 8001ffa:	4293      	cmp	r3, r2
 8001ffc:	d029      	beq.n	8002052 <HAL_DMA_IRQHandler+0x166>
 8001ffe:	687b      	ldr	r3, [r7, #4]
 8002000:	681b      	ldr	r3, [r3, #0]
 8002002:	4a37      	ldr	r2, [pc, #220]	; (80020e0 <HAL_DMA_IRQHandler+0x1f4>)
 8002004:	4293      	cmp	r3, r2
 8002006:	d022      	beq.n	800204e <HAL_DMA_IRQHandler+0x162>
 8002008:	687b      	ldr	r3, [r7, #4]
 800200a:	681b      	ldr	r3, [r3, #0]
 800200c:	4a35      	ldr	r2, [pc, #212]	; (80020e4 <HAL_DMA_IRQHandler+0x1f8>)
 800200e:	4293      	cmp	r3, r2
 8002010:	d01a      	beq.n	8002048 <HAL_DMA_IRQHandler+0x15c>
 8002012:	687b      	ldr	r3, [r7, #4]
 8002014:	681b      	ldr	r3, [r3, #0]
 8002016:	4a34      	ldr	r2, [pc, #208]	; (80020e8 <HAL_DMA_IRQHandler+0x1fc>)
 8002018:	4293      	cmp	r3, r2
 800201a:	d012      	beq.n	8002042 <HAL_DMA_IRQHandler+0x156>
 800201c:	687b      	ldr	r3, [r7, #4]
 800201e:	681b      	ldr	r3, [r3, #0]
 8002020:	4a32      	ldr	r2, [pc, #200]	; (80020ec <HAL_DMA_IRQHandler+0x200>)
 8002022:	4293      	cmp	r3, r2
 8002024:	d00a      	beq.n	800203c <HAL_DMA_IRQHandler+0x150>
 8002026:	687b      	ldr	r3, [r7, #4]
 8002028:	681b      	ldr	r3, [r3, #0]
 800202a:	4a31      	ldr	r2, [pc, #196]	; (80020f0 <HAL_DMA_IRQHandler+0x204>)
 800202c:	4293      	cmp	r3, r2
 800202e:	d102      	bne.n	8002036 <HAL_DMA_IRQHandler+0x14a>
 8002030:	f44f 1300 	mov.w	r3, #2097152	; 0x200000
 8002034:	e00e      	b.n	8002054 <HAL_DMA_IRQHandler+0x168>
 8002036:	f04f 7300 	mov.w	r3, #33554432	; 0x2000000
 800203a:	e00b      	b.n	8002054 <HAL_DMA_IRQHandler+0x168>
 800203c:	f44f 3300 	mov.w	r3, #131072	; 0x20000
 8002040:	e008      	b.n	8002054 <HAL_DMA_IRQHandler+0x168>
 8002042:	f44f 5300 	mov.w	r3, #8192	; 0x2000
 8002046:	e005      	b.n	8002054 <HAL_DMA_IRQHandler+0x168>
 8002048:	f44f 7300 	mov.w	r3, #512	; 0x200
 800204c:	e002      	b.n	8002054 <HAL_DMA_IRQHandler+0x168>
 800204e:	2320      	movs	r3, #32
 8002050:	e000      	b.n	8002054 <HAL_DMA_IRQHandler+0x168>
 8002052:	2302      	movs	r3, #2
 8002054:	4a27      	ldr	r2, [pc, #156]	; (80020f4 <HAL_DMA_IRQHandler+0x208>)
 8002056:	6053      	str	r3, [r2, #4]

    /* Process Unlocked */
    __HAL_UNLOCK(hdma);
 8002058:	687b      	ldr	r3, [r7, #4]
 800205a:	2200      	movs	r2, #0
 800205c:	f883 2020 	strb.w	r2, [r3, #32]

    if(hdma->XferCpltCallback != NULL)
 8002060:	687b      	ldr	r3, [r7, #4]
 8002062:	6a9b      	ldr	r3, [r3, #40]	; 0x28
 8002064:	2b00      	cmp	r3, #0
 8002066:	d034      	beq.n	80020d2 <HAL_DMA_IRQHandler+0x1e6>
    {
      /* Transfer complete callback */
      hdma->XferCpltCallback(hdma);
 8002068:	687b      	ldr	r3, [r7, #4]
 800206a:	6a9b      	ldr	r3, [r3, #40]	; 0x28
 800206c:	6878      	ldr	r0, [r7, #4]
 800206e:	4798      	blx	r3
    if(hdma->XferCpltCallback != NULL)
 8002070:	e02f      	b.n	80020d2 <HAL_DMA_IRQHandler+0x1e6>
    }
  }

  /* Transfer Error Interrupt management **************************************/
  else if (( RESET != (flag_it & (DMA_FLAG_TE1 << hdma->ChannelIndex))) && (RESET != (source_it & DMA_IT_TE)))
 8002072:	687b      	ldr	r3, [r7, #4]
 8002074:	6c1b      	ldr	r3, [r3, #64]	; 0x40
 8002076:	2208      	movs	r2, #8
 8002078:	409a      	lsls	r2, r3
 800207a:	68fb      	ldr	r3, [r7, #12]
 800207c:	4013      	ands	r3, r2
 800207e:	2b00      	cmp	r3, #0
 8002080:	d028      	beq.n	80020d4 <HAL_DMA_IRQHandler+0x1e8>
 8002082:	68bb      	ldr	r3, [r7, #8]
 8002084:	f003 0308 	and.w	r3, r3, #8
 8002088:	2b00      	cmp	r3, #0
 800208a:	d023      	beq.n	80020d4 <HAL_DMA_IRQHandler+0x1e8>
  {
    /* When a DMA transfer error occurs */
    /* A hardware clear of its EN bits is performed */
    /* Disable ALL DMA IT */
    __HAL_DMA_DISABLE_IT(hdma, (DMA_IT_TC | DMA_IT_HT | DMA_IT_TE));
 800208c:	687b      	ldr	r3, [r7, #4]
 800208e:	681b      	ldr	r3, [r3, #0]
 8002090:	681a      	ldr	r2, [r3, #0]
 8002092:	687b      	ldr	r3, [r7, #4]
 8002094:	681b      	ldr	r3, [r3, #0]
 8002096:	f022 020e 	bic.w	r2, r2, #14
 800209a:	601a      	str	r2, [r3, #0]

    /* Clear all flags */
    hdma->DmaBaseAddress->IFCR = (DMA_ISR_GIF1 << hdma->ChannelIndex);
 800209c:	687b      	ldr	r3, [r7, #4]
 800209e:	6c1a      	ldr	r2, [r3, #64]	; 0x40
 80020a0:	687b      	ldr	r3, [r7, #4]
 80020a2:	6bdb      	ldr	r3, [r3, #60]	; 0x3c
 80020a4:	2101      	movs	r1, #1
 80020a6:	fa01 f202 	lsl.w	r2, r1, r2
 80020aa:	605a      	str	r2, [r3, #4]

    /* Update error code */
    hdma->ErrorCode = HAL_DMA_ERROR_TE;
 80020ac:	687b      	ldr	r3, [r7, #4]
 80020ae:	2201      	movs	r2, #1
 80020b0:	639a      	str	r2, [r3, #56]	; 0x38

    /* Change the DMA state */
    hdma->State = HAL_DMA_STATE_READY;
 80020b2:	687b      	ldr	r3, [r7, #4]
 80020b4:	2201      	movs	r2, #1
 80020b6:	f883 2021 	strb.w	r2, [r3, #33]	; 0x21

    /* Process Unlocked */
    __HAL_UNLOCK(hdma);
 80020ba:	687b      	ldr	r3, [r7, #4]
 80020bc:	2200      	movs	r2, #0
 80020be:	f883 2020 	strb.w	r2, [r3, #32]

    if (hdma->XferErrorCallback != NULL)
 80020c2:	687b      	ldr	r3, [r7, #4]
 80020c4:	6b1b      	ldr	r3, [r3, #48]	; 0x30
 80020c6:	2b00      	cmp	r3, #0
 80020c8:	d004      	beq.n	80020d4 <HAL_DMA_IRQHandler+0x1e8>
    {
      /* Transfer error callback */
      hdma->XferErrorCallback(hdma);
 80020ca:	687b      	ldr	r3, [r7, #4]
 80020cc:	6b1b      	ldr	r3, [r3, #48]	; 0x30
 80020ce:	6878      	ldr	r0, [r7, #4]
 80020d0:	4798      	blx	r3
    }
  }
  return;
 80020d2:	bf00      	nop
 80020d4:	bf00      	nop
}
 80020d6:	3710      	adds	r7, #16
 80020d8:	46bd      	mov	sp, r7
 80020da:	bd80      	pop	{r7, pc}
 80020dc:	40020008 	.word	0x40020008
 80020e0:	4002001c 	.word	0x4002001c
 80020e4:	40020030 	.word	0x40020030
 80020e8:	40020044 	.word	0x40020044
 80020ec:	40020058 	.word	0x40020058
 80020f0:	4002006c 	.word	0x4002006c
 80020f4:	40020000 	.word	0x40020000

080020f8 <DMA_SetConfig>:
  * @param  DstAddress: The destination memory Buffer address
  * @param  DataLength: The length of data to be transferred from source to destination
  * @retval HAL status
  */
static void DMA_SetConfig(DMA_HandleTypeDef *hdma, uint32_t SrcAddress, uint32_t DstAddress, uint32_t DataLength)
{
 80020f8:	b480      	push	{r7}
 80020fa:	b085      	sub	sp, #20
 80020fc:	af00      	add	r7, sp, #0
 80020fe:	60f8      	str	r0, [r7, #12]
 8002100:	60b9      	str	r1, [r7, #8]
 8002102:	607a      	str	r2, [r7, #4]
 8002104:	603b      	str	r3, [r7, #0]
  /* Clear all flags */
  hdma->DmaBaseAddress->IFCR = (DMA_ISR_GIF1 << hdma->ChannelIndex);
 8002106:	68fb      	ldr	r3, [r7, #12]
 8002108:	6c1a      	ldr	r2, [r3, #64]	; 0x40
 800210a:	68fb      	ldr	r3, [r7, #12]
 800210c:	6bdb      	ldr	r3, [r3, #60]	; 0x3c
 800210e:	2101      	movs	r1, #1
 8002110:	fa01 f202 	lsl.w	r2, r1, r2
 8002114:	605a      	str	r2, [r3, #4]

  /* Configure DMA Channel data length */
  hdma->Instance->CNDTR = DataLength;
 8002116:	68fb      	ldr	r3, [r7, #12]
 8002118:	681b      	ldr	r3, [r3, #0]
 800211a:	683a      	ldr	r2, [r7, #0]
 800211c:	605a      	str	r2, [r3, #4]

  /* Memory to Peripheral */
  if((hdma->Init.Direction) == DMA_MEMORY_TO_PERIPH)
 800211e:	68fb      	ldr	r3, [r7, #12]
 8002120:	685b      	ldr	r3, [r3, #4]
 8002122:	2b10      	cmp	r3, #16
 8002124:	d108      	bne.n	8002138 <DMA_SetConfig+0x40>
  {
    /* Configure DMA Channel destination address */
    hdma->Instance->CPAR = DstAddress;
 8002126:	68fb      	ldr	r3, [r7, #12]
 8002128:	681b      	ldr	r3, [r3, #0]
 800212a:	687a      	ldr	r2, [r7, #4]
 800212c:	609a      	str	r2, [r3, #8]

    /* Configure DMA Channel source address */
    hdma->Instance->CMAR = SrcAddress;
 800212e:	68fb      	ldr	r3, [r7, #12]
 8002130:	681b      	ldr	r3, [r3, #0]
 8002132:	68ba      	ldr	r2, [r7, #8]
 8002134:	60da      	str	r2, [r3, #12]
    hdma->Instance->CPAR = SrcAddress;

    /* Configure DMA Channel destination address */
    hdma->Instance->CMAR = DstAddress;
  }
}
 8002136:	e007      	b.n	8002148 <DMA_SetConfig+0x50>
    hdma->Instance->CPAR = SrcAddress;
 8002138:	68fb      	ldr	r3, [r7, #12]
 800213a:	681b      	ldr	r3, [r3, #0]
 800213c:	68ba      	ldr	r2, [r7, #8]
 800213e:	609a      	str	r2, [r3, #8]
    hdma->Instance->CMAR = DstAddress;
 8002140:	68fb      	ldr	r3, [r7, #12]
 8002142:	681b      	ldr	r3, [r3, #0]
 8002144:	687a      	ldr	r2, [r7, #4]
 8002146:	60da      	str	r2, [r3, #12]
}
 8002148:	bf00      	nop
 800214a:	3714      	adds	r7, #20
 800214c:	46bd      	mov	sp, r7
 800214e:	bc80      	pop	{r7}
 8002150:	4770      	bx	lr
	...

08002154 <HAL_GPIO_Init>:
  * @param  GPIO_Init: pointer to a GPIO_InitTypeDef structure that contains
  *         the configuration information for the specified GPIO peripheral.
  * @retval None
  */
void HAL_GPIO_Init(GPIO_TypeDef  *GPIOx, GPIO_InitTypeDef *GPIO_Init)
{
 8002154:	b480      	push	{r7}
 8002156:	b08b      	sub	sp, #44	; 0x2c
 8002158:	af00      	add	r7, sp, #0
 800215a:	6078      	str	r0, [r7, #4]
 800215c:	6039      	str	r1, [r7, #0]
  uint32_t position = 0x00u;
 800215e:	2300      	movs	r3, #0
 8002160:	627b      	str	r3, [r7, #36]	; 0x24
  uint32_t ioposition;
  uint32_t iocurrent;
  uint32_t temp;
  uint32_t config = 0x00u;
 8002162:	2300      	movs	r3, #0
 8002164:	623b      	str	r3, [r7, #32]
  assert_param(IS_GPIO_ALL_INSTANCE(GPIOx));
  assert_param(IS_GPIO_PIN(GPIO_Init->Pin));
  assert_param(IS_GPIO_MODE(GPIO_Init->Mode));

  /* Configure the port pins */
  while (((GPIO_Init->Pin) >> position) != 0x00u)
 8002166:	e169      	b.n	800243c <HAL_GPIO_Init+0x2e8>
  {
    /* Get the IO position */
    ioposition = (0x01uL << position);
 8002168:	2201      	movs	r2, #1
 800216a:	6a7b      	ldr	r3, [r7, #36]	; 0x24
 800216c:	fa02 f303 	lsl.w	r3, r2, r3
 8002170:	61fb      	str	r3, [r7, #28]

    /* Get the current IO position */
    iocurrent = (uint32_t)(GPIO_Init->Pin) & ioposition;
 8002172:	683b      	ldr	r3, [r7, #0]
 8002174:	681b      	ldr	r3, [r3, #0]
 8002176:	69fa      	ldr	r2, [r7, #28]
 8002178:	4013      	ands	r3, r2
 800217a:	61bb      	str	r3, [r7, #24]

    if (iocurrent == ioposition)
 800217c:	69ba      	ldr	r2, [r7, #24]
 800217e:	69fb      	ldr	r3, [r7, #28]
 8002180:	429a      	cmp	r2, r3
 8002182:	f040 8158 	bne.w	8002436 <HAL_GPIO_Init+0x2e2>
    {
      /* Check the Alternate function parameters */
      assert_param(IS_GPIO_AF_INSTANCE(GPIOx));

      /* Based on the required mode, filling config variable with MODEy[1:0] and CNFy[3:2] corresponding bits */
      switch (GPIO_Init->Mode)
 8002186:	683b      	ldr	r3, [r7, #0]
 8002188:	685b      	ldr	r3, [r3, #4]
 800218a:	4a9a      	ldr	r2, [pc, #616]	; (80023f4 <HAL_GPIO_Init+0x2a0>)
 800218c:	4293      	cmp	r3, r2
 800218e:	d05e      	beq.n	800224e <HAL_GPIO_Init+0xfa>
 8002190:	4a98      	ldr	r2, [pc, #608]	; (80023f4 <HAL_GPIO_Init+0x2a0>)
 8002192:	4293      	cmp	r3, r2
 8002194:	d875      	bhi.n	8002282 <HAL_GPIO_Init+0x12e>
 8002196:	4a98      	ldr	r2, [pc, #608]	; (80023f8 <HAL_GPIO_Init+0x2a4>)
 8002198:	4293      	cmp	r3, r2
 800219a:	d058      	beq.n	800224e <HAL_GPIO_Init+0xfa>
 800219c:	4a96      	ldr	r2, [pc, #600]	; (80023f8 <HAL_GPIO_Init+0x2a4>)
 800219e:	4293      	cmp	r3, r2
 80021a0:	d86f      	bhi.n	8002282 <HAL_GPIO_Init+0x12e>
 80021a2:	4a96      	ldr	r2, [pc, #600]	; (80023fc <HAL_GPIO_Init+0x2a8>)
 80021a4:	4293      	cmp	r3, r2
 80021a6:	d052      	beq.n	800224e <HAL_GPIO_Init+0xfa>
 80021a8:	4a94      	ldr	r2, [pc, #592]	; (80023fc <HAL_GPIO_Init+0x2a8>)
 80021aa:	4293      	cmp	r3, r2
 80021ac:	d869      	bhi.n	8002282 <HAL_GPIO_Init+0x12e>
 80021ae:	4a94      	ldr	r2, [pc, #592]	; (8002400 <HAL_GPIO_Init+0x2ac>)
 80021b0:	4293      	cmp	r3, r2
 80021b2:	d04c      	beq.n	800224e <HAL_GPIO_Init+0xfa>
 80021b4:	4a92      	ldr	r2, [pc, #584]	; (8002400 <HAL_GPIO_Init+0x2ac>)
 80021b6:	4293      	cmp	r3, r2
 80021b8:	d863      	bhi.n	8002282 <HAL_GPIO_Init+0x12e>
 80021ba:	4a92      	ldr	r2, [pc, #584]	; (8002404 <HAL_GPIO_Init+0x2b0>)
 80021bc:	4293      	cmp	r3, r2
 80021be:	d046      	beq.n	800224e <HAL_GPIO_Init+0xfa>
 80021c0:	4a90      	ldr	r2, [pc, #576]	; (8002404 <HAL_GPIO_Init+0x2b0>)
 80021c2:	4293      	cmp	r3, r2
 80021c4:	d85d      	bhi.n	8002282 <HAL_GPIO_Init+0x12e>
 80021c6:	2b12      	cmp	r3, #18
 80021c8:	d82a      	bhi.n	8002220 <HAL_GPIO_Init+0xcc>
 80021ca:	2b12      	cmp	r3, #18
 80021cc:	d859      	bhi.n	8002282 <HAL_GPIO_Init+0x12e>
 80021ce:	a201      	add	r2, pc, #4	; (adr r2, 80021d4 <HAL_GPIO_Init+0x80>)
 80021d0:	f852 f023 	ldr.w	pc, [r2, r3, lsl #2]
 80021d4:	0800224f 	.word	0x0800224f
 80021d8:	08002229 	.word	0x08002229
 80021dc:	0800223b 	.word	0x0800223b
 80021e0:	0800227d 	.word	0x0800227d
 80021e4:	08002283 	.word	0x08002283
 80021e8:	08002283 	.word	0x08002283
 80021ec:	08002283 	.word	0x08002283
 80021f0:	08002283 	.word	0x08002283
 80021f4:	08002283 	.word	0x08002283
 80021f8:	08002283 	.word	0x08002283
 80021fc:	08002283 	.word	0x08002283
 8002200:	08002283 	.word	0x08002283
 8002204:	08002283 	.word	0x08002283
 8002208:	08002283 	.word	0x08002283
 800220c:	08002283 	.word	0x08002283
 8002210:	08002283 	.word	0x08002283
 8002214:	08002283 	.word	0x08002283
 8002218:	08002231 	.word	0x08002231
 800221c:	08002245 	.word	0x08002245
 8002220:	4a79      	ldr	r2, [pc, #484]	; (8002408 <HAL_GPIO_Init+0x2b4>)
 8002222:	4293      	cmp	r3, r2
 8002224:	d013      	beq.n	800224e <HAL_GPIO_Init+0xfa>
          config = GPIO_CR_MODE_INPUT + GPIO_CR_CNF_ANALOG;
          break;

        /* Parameters are checked with assert_param */
        default:
          break;
 8002226:	e02c      	b.n	8002282 <HAL_GPIO_Init+0x12e>
          config = GPIO_Init->Speed + GPIO_CR_CNF_GP_OUTPUT_PP;
 8002228:	683b      	ldr	r3, [r7, #0]
 800222a:	68db      	ldr	r3, [r3, #12]
 800222c:	623b      	str	r3, [r7, #32]
          break;
 800222e:	e029      	b.n	8002284 <HAL_GPIO_Init+0x130>
          config = GPIO_Init->Speed + GPIO_CR_CNF_GP_OUTPUT_OD;
 8002230:	683b      	ldr	r3, [r7, #0]
 8002232:	68db      	ldr	r3, [r3, #12]
 8002234:	3304      	adds	r3, #4
 8002236:	623b      	str	r3, [r7, #32]
          break;
 8002238:	e024      	b.n	8002284 <HAL_GPIO_Init+0x130>
          config = GPIO_Init->Speed + GPIO_CR_CNF_AF_OUTPUT_PP;
 800223a:	683b      	ldr	r3, [r7, #0]
 800223c:	68db      	ldr	r3, [r3, #12]
 800223e:	3308      	adds	r3, #8
 8002240:	623b      	str	r3, [r7, #32]
          break;
 8002242:	e01f      	b.n	8002284 <HAL_GPIO_Init+0x130>
          config = GPIO_Init->Speed + GPIO_CR_CNF_AF_OUTPUT_OD;
 8002244:	683b      	ldr	r3, [r7, #0]
 8002246:	68db      	ldr	r3, [r3, #12]
 8002248:	330c      	adds	r3, #12
 800224a:	623b      	str	r3, [r7, #32]
          break;
 800224c:	e01a      	b.n	8002284 <HAL_GPIO_Init+0x130>
          if (GPIO_Init->Pull == GPIO_NOPULL)
 800224e:	683b      	ldr	r3, [r7, #0]
 8002250:	689b      	ldr	r3, [r3, #8]
 8002252:	2b00      	cmp	r3, #0
 8002254:	d102      	bne.n	800225c <HAL_GPIO_Init+0x108>
            config = GPIO_CR_MODE_INPUT + GPIO_CR_CNF_INPUT_FLOATING;
 8002256:	2304      	movs	r3, #4
 8002258:	623b      	str	r3, [r7, #32]
          break;
 800225a:	e013      	b.n	8002284 <HAL_GPIO_Init+0x130>
          else if (GPIO_Init->Pull == GPIO_PULLUP)
 800225c:	683b      	ldr	r3, [r7, #0]
 800225e:	689b      	ldr	r3, [r3, #8]
 8002260:	2b01      	cmp	r3, #1
 8002262:	d105      	bne.n	8002270 <HAL_GPIO_Init+0x11c>
            config = GPIO_CR_MODE_INPUT + GPIO_CR_CNF_INPUT_PU_PD;
 8002264:	2308      	movs	r3, #8
 8002266:	623b      	str	r3, [r7, #32]
            GPIOx->BSRR = ioposition;
 8002268:	687b      	ldr	r3, [r7, #4]
 800226a:	69fa      	ldr	r2, [r7, #28]
 800226c:	611a      	str	r2, [r3, #16]
          break;
 800226e:	e009      	b.n	8002284 <HAL_GPIO_Init+0x130>
            config = GPIO_CR_MODE_INPUT + GPIO_CR_CNF_INPUT_PU_PD;
 8002270:	2308      	movs	r3, #8
 8002272:	623b      	str	r3, [r7, #32]
            GPIOx->BRR = ioposition;
 8002274:	687b      	ldr	r3, [r7, #4]
 8002276:	69fa      	ldr	r2, [r7, #28]
 8002278:	615a      	str	r2, [r3, #20]
          break;
 800227a:	e003      	b.n	8002284 <HAL_GPIO_Init+0x130>
          config = GPIO_CR_MODE_INPUT + GPIO_CR_CNF_ANALOG;
 800227c:	2300      	movs	r3, #0
 800227e:	623b      	str	r3, [r7, #32]
          break;
 8002280:	e000      	b.n	8002284 <HAL_GPIO_Init+0x130>
          break;
 8002282:	bf00      	nop
      }

      /* Check if the current bit belongs to first half or last half of the pin count number
       in order to address CRH or CRL register*/
      configregister = (iocurrent < GPIO_PIN_8) ? &GPIOx->CRL     : &GPIOx->CRH;
 8002284:	69bb      	ldr	r3, [r7, #24]
 8002286:	2bff      	cmp	r3, #255	; 0xff
 8002288:	d801      	bhi.n	800228e <HAL_GPIO_Init+0x13a>
 800228a:	687b      	ldr	r3, [r7, #4]
 800228c:	e001      	b.n	8002292 <HAL_GPIO_Init+0x13e>
 800228e:	687b      	ldr	r3, [r7, #4]
 8002290:	3304      	adds	r3, #4
 8002292:	617b      	str	r3, [r7, #20]
      registeroffset = (iocurrent < GPIO_PIN_8) ? (position << 2u) : ((position - 8u) << 2u);
 8002294:	69bb      	ldr	r3, [r7, #24]
 8002296:	2bff      	cmp	r3, #255	; 0xff
 8002298:	d802      	bhi.n	80022a0 <HAL_GPIO_Init+0x14c>
 800229a:	6a7b      	ldr	r3, [r7, #36]	; 0x24
 800229c:	009b      	lsls	r3, r3, #2
 800229e:	e002      	b.n	80022a6 <HAL_GPIO_Init+0x152>
 80022a0:	6a7b      	ldr	r3, [r7, #36]	; 0x24
 80022a2:	3b08      	subs	r3, #8
 80022a4:	009b      	lsls	r3, r3, #2
 80022a6:	613b      	str	r3, [r7, #16]

      /* Apply the new configuration of the pin to the register */
      MODIFY_REG((*configregister), ((GPIO_CRL_MODE0 | GPIO_CRL_CNF0) << registeroffset), (config << registeroffset));
 80022a8:	697b      	ldr	r3, [r7, #20]
 80022aa:	681a      	ldr	r2, [r3, #0]
 80022ac:	210f      	movs	r1, #15
 80022ae:	693b      	ldr	r3, [r7, #16]
 80022b0:	fa01 f303 	lsl.w	r3, r1, r3
 80022b4:	43db      	mvns	r3, r3
 80022b6:	401a      	ands	r2, r3
 80022b8:	6a39      	ldr	r1, [r7, #32]
 80022ba:	693b      	ldr	r3, [r7, #16]
 80022bc:	fa01 f303 	lsl.w	r3, r1, r3
 80022c0:	431a      	orrs	r2, r3
 80022c2:	697b      	ldr	r3, [r7, #20]
 80022c4:	601a      	str	r2, [r3, #0]

      /*--------------------- EXTI Mode Configuration ------------------------*/
      /* Configure the External Interrupt or event for the current IO */
      if ((GPIO_Init->Mode & EXTI_MODE) == EXTI_MODE)
 80022c6:	683b      	ldr	r3, [r7, #0]
 80022c8:	685b      	ldr	r3, [r3, #4]
 80022ca:	f003 5380 	and.w	r3, r3, #268435456	; 0x10000000
 80022ce:	2b00      	cmp	r3, #0
 80022d0:	f000 80b1 	beq.w	8002436 <HAL_GPIO_Init+0x2e2>
      {
        /* Enable AFIO Clock */
        __HAL_RCC_AFIO_CLK_ENABLE();
 80022d4:	4b4d      	ldr	r3, [pc, #308]	; (800240c <HAL_GPIO_Init+0x2b8>)
 80022d6:	699b      	ldr	r3, [r3, #24]
 80022d8:	4a4c      	ldr	r2, [pc, #304]	; (800240c <HAL_GPIO_Init+0x2b8>)
 80022da:	f043 0301 	orr.w	r3, r3, #1
 80022de:	6193      	str	r3, [r2, #24]
 80022e0:	4b4a      	ldr	r3, [pc, #296]	; (800240c <HAL_GPIO_Init+0x2b8>)
 80022e2:	699b      	ldr	r3, [r3, #24]
 80022e4:	f003 0301 	and.w	r3, r3, #1
 80022e8:	60bb      	str	r3, [r7, #8]
 80022ea:	68bb      	ldr	r3, [r7, #8]
        temp = AFIO->EXTICR[position >> 2u];
 80022ec:	4a48      	ldr	r2, [pc, #288]	; (8002410 <HAL_GPIO_Init+0x2bc>)
 80022ee:	6a7b      	ldr	r3, [r7, #36]	; 0x24
 80022f0:	089b      	lsrs	r3, r3, #2
 80022f2:	3302      	adds	r3, #2
 80022f4:	f852 3023 	ldr.w	r3, [r2, r3, lsl #2]
 80022f8:	60fb      	str	r3, [r7, #12]
        CLEAR_BIT(temp, (0x0Fu) << (4u * (position & 0x03u)));
 80022fa:	6a7b      	ldr	r3, [r7, #36]	; 0x24
 80022fc:	f003 0303 	and.w	r3, r3, #3
 8002300:	009b      	lsls	r3, r3, #2
 8002302:	220f      	movs	r2, #15
 8002304:	fa02 f303 	lsl.w	r3, r2, r3
 8002308:	43db      	mvns	r3, r3
 800230a:	68fa      	ldr	r2, [r7, #12]
 800230c:	4013      	ands	r3, r2
 800230e:	60fb      	str	r3, [r7, #12]
        SET_BIT(temp, (GPIO_GET_INDEX(GPIOx)) << (4u * (position & 0x03u)));
 8002310:	687b      	ldr	r3, [r7, #4]
 8002312:	4a40      	ldr	r2, [pc, #256]	; (8002414 <HAL_GPIO_Init+0x2c0>)
 8002314:	4293      	cmp	r3, r2
 8002316:	d013      	beq.n	8002340 <HAL_GPIO_Init+0x1ec>
 8002318:	687b      	ldr	r3, [r7, #4]
 800231a:	4a3f      	ldr	r2, [pc, #252]	; (8002418 <HAL_GPIO_Init+0x2c4>)
 800231c:	4293      	cmp	r3, r2
 800231e:	d00d      	beq.n	800233c <HAL_GPIO_Init+0x1e8>
 8002320:	687b      	ldr	r3, [r7, #4]
 8002322:	4a3e      	ldr	r2, [pc, #248]	; (800241c <HAL_GPIO_Init+0x2c8>)
 8002324:	4293      	cmp	r3, r2
 8002326:	d007      	beq.n	8002338 <HAL_GPIO_Init+0x1e4>
 8002328:	687b      	ldr	r3, [r7, #4]
 800232a:	4a3d      	ldr	r2, [pc, #244]	; (8002420 <HAL_GPIO_Init+0x2cc>)
 800232c:	4293      	cmp	r3, r2
 800232e:	d101      	bne.n	8002334 <HAL_GPIO_Init+0x1e0>
 8002330:	2303      	movs	r3, #3
 8002332:	e006      	b.n	8002342 <HAL_GPIO_Init+0x1ee>
 8002334:	2304      	movs	r3, #4
 8002336:	e004      	b.n	8002342 <HAL_GPIO_Init+0x1ee>
 8002338:	2302      	movs	r3, #2
 800233a:	e002      	b.n	8002342 <HAL_GPIO_Init+0x1ee>
 800233c:	2301      	movs	r3, #1
 800233e:	e000      	b.n	8002342 <HAL_GPIO_Init+0x1ee>
 8002340:	2300      	movs	r3, #0
 8002342:	6a7a      	ldr	r2, [r7, #36]	; 0x24
 8002344:	f002 0203 	and.w	r2, r2, #3
 8002348:	0092      	lsls	r2, r2, #2
 800234a:	4093      	lsls	r3, r2
 800234c:	68fa      	ldr	r2, [r7, #12]
 800234e:	4313      	orrs	r3, r2
 8002350:	60fb      	str	r3, [r7, #12]
        AFIO->EXTICR[position >> 2u] = temp;
 8002352:	492f      	ldr	r1, [pc, #188]	; (8002410 <HAL_GPIO_Init+0x2bc>)
 8002354:	6a7b      	ldr	r3, [r7, #36]	; 0x24
 8002356:	089b      	lsrs	r3, r3, #2
 8002358:	3302      	adds	r3, #2
 800235a:	68fa      	ldr	r2, [r7, #12]
 800235c:	f841 2023 	str.w	r2, [r1, r3, lsl #2]


        /* Configure the interrupt mask */
        if ((GPIO_Init->Mode & GPIO_MODE_IT) == GPIO_MODE_IT)
 8002360:	683b      	ldr	r3, [r7, #0]
 8002362:	685b      	ldr	r3, [r3, #4]
 8002364:	f403 3380 	and.w	r3, r3, #65536	; 0x10000
 8002368:	2b00      	cmp	r3, #0
 800236a:	d006      	beq.n	800237a <HAL_GPIO_Init+0x226>
        {
          SET_BIT(EXTI->IMR, iocurrent);
 800236c:	4b2d      	ldr	r3, [pc, #180]	; (8002424 <HAL_GPIO_Init+0x2d0>)
 800236e:	681a      	ldr	r2, [r3, #0]
 8002370:	492c      	ldr	r1, [pc, #176]	; (8002424 <HAL_GPIO_Init+0x2d0>)
 8002372:	69bb      	ldr	r3, [r7, #24]
 8002374:	4313      	orrs	r3, r2
 8002376:	600b      	str	r3, [r1, #0]
 8002378:	e006      	b.n	8002388 <HAL_GPIO_Init+0x234>
        }
        else
        {
          CLEAR_BIT(EXTI->IMR, iocurrent);
 800237a:	4b2a      	ldr	r3, [pc, #168]	; (8002424 <HAL_GPIO_Init+0x2d0>)
 800237c:	681a      	ldr	r2, [r3, #0]
 800237e:	69bb      	ldr	r3, [r7, #24]
 8002380:	43db      	mvns	r3, r3
 8002382:	4928      	ldr	r1, [pc, #160]	; (8002424 <HAL_GPIO_Init+0x2d0>)
 8002384:	4013      	ands	r3, r2
 8002386:	600b      	str	r3, [r1, #0]
        }

        /* Configure the event mask */
        if ((GPIO_Init->Mode & GPIO_MODE_EVT) == GPIO_MODE_EVT)
 8002388:	683b      	ldr	r3, [r7, #0]
 800238a:	685b      	ldr	r3, [r3, #4]
 800238c:	f403 3300 	and.w	r3, r3, #131072	; 0x20000
 8002390:	2b00      	cmp	r3, #0
 8002392:	d006      	beq.n	80023a2 <HAL_GPIO_Init+0x24e>
        {
          SET_BIT(EXTI->EMR, iocurrent);
 8002394:	4b23      	ldr	r3, [pc, #140]	; (8002424 <HAL_GPIO_Init+0x2d0>)
 8002396:	685a      	ldr	r2, [r3, #4]
 8002398:	4922      	ldr	r1, [pc, #136]	; (8002424 <HAL_GPIO_Init+0x2d0>)
 800239a:	69bb      	ldr	r3, [r7, #24]
 800239c:	4313      	orrs	r3, r2
 800239e:	604b      	str	r3, [r1, #4]
 80023a0:	e006      	b.n	80023b0 <HAL_GPIO_Init+0x25c>
        }
        else
        {
          CLEAR_BIT(EXTI->EMR, iocurrent);
 80023a2:	4b20      	ldr	r3, [pc, #128]	; (8002424 <HAL_GPIO_Init+0x2d0>)
 80023a4:	685a      	ldr	r2, [r3, #4]
 80023a6:	69bb      	ldr	r3, [r7, #24]
 80023a8:	43db      	mvns	r3, r3
 80023aa:	491e      	ldr	r1, [pc, #120]	; (8002424 <HAL_GPIO_Init+0x2d0>)
 80023ac:	4013      	ands	r3, r2
 80023ae:	604b      	str	r3, [r1, #4]
        }

        /* Enable or disable the rising trigger */
        if ((GPIO_Init->Mode & RISING_EDGE) == RISING_EDGE)
 80023b0:	683b      	ldr	r3, [r7, #0]
 80023b2:	685b      	ldr	r3, [r3, #4]
 80023b4:	f403 1380 	and.w	r3, r3, #1048576	; 0x100000
 80023b8:	2b00      	cmp	r3, #0
 80023ba:	d006      	beq.n	80023ca <HAL_GPIO_Init+0x276>
        {
          SET_BIT(EXTI->RTSR, iocurrent);
 80023bc:	4b19      	ldr	r3, [pc, #100]	; (8002424 <HAL_GPIO_Init+0x2d0>)
 80023be:	689a      	ldr	r2, [r3, #8]
 80023c0:	4918      	ldr	r1, [pc, #96]	; (8002424 <HAL_GPIO_Init+0x2d0>)
 80023c2:	69bb      	ldr	r3, [r7, #24]
 80023c4:	4313      	orrs	r3, r2
 80023c6:	608b      	str	r3, [r1, #8]
 80023c8:	e006      	b.n	80023d8 <HAL_GPIO_Init+0x284>
        }
        else
        {
          CLEAR_BIT(EXTI->RTSR, iocurrent);
 80023ca:	4b16      	ldr	r3, [pc, #88]	; (8002424 <HAL_GPIO_Init+0x2d0>)
 80023cc:	689a      	ldr	r2, [r3, #8]
 80023ce:	69bb      	ldr	r3, [r7, #24]
 80023d0:	43db      	mvns	r3, r3
 80023d2:	4914      	ldr	r1, [pc, #80]	; (8002424 <HAL_GPIO_Init+0x2d0>)
 80023d4:	4013      	ands	r3, r2
 80023d6:	608b      	str	r3, [r1, #8]
        }

        /* Enable or disable the falling trigger */
        if ((GPIO_Init->Mode & FALLING_EDGE) == FALLING_EDGE)
 80023d8:	683b      	ldr	r3, [r7, #0]
 80023da:	685b      	ldr	r3, [r3, #4]
 80023dc:	f403 1300 	and.w	r3, r3, #2097152	; 0x200000
 80023e0:	2b00      	cmp	r3, #0
 80023e2:	d021      	beq.n	8002428 <HAL_GPIO_Init+0x2d4>
        {
          SET_BIT(EXTI->FTSR, iocurrent);
 80023e4:	4b0f      	ldr	r3, [pc, #60]	; (8002424 <HAL_GPIO_Init+0x2d0>)
 80023e6:	68da      	ldr	r2, [r3, #12]
 80023e8:	490e      	ldr	r1, [pc, #56]	; (8002424 <HAL_GPIO_Init+0x2d0>)
 80023ea:	69bb      	ldr	r3, [r7, #24]
 80023ec:	4313      	orrs	r3, r2
 80023ee:	60cb      	str	r3, [r1, #12]
 80023f0:	e021      	b.n	8002436 <HAL_GPIO_Init+0x2e2>
 80023f2:	bf00      	nop
 80023f4:	10320000 	.word	0x10320000
 80023f8:	10310000 	.word	0x10310000
 80023fc:	10220000 	.word	0x10220000
 8002400:	10210000 	.word	0x10210000
 8002404:	10120000 	.word	0x10120000
 8002408:	10110000 	.word	0x10110000
 800240c:	40021000 	.word	0x40021000
 8002410:	40010000 	.word	0x40010000
 8002414:	40010800 	.word	0x40010800
 8002418:	40010c00 	.word	0x40010c00
 800241c:	40011000 	.word	0x40011000
 8002420:	40011400 	.word	0x40011400
 8002424:	40010400 	.word	0x40010400
        }
        else
        {
          CLEAR_BIT(EXTI->FTSR, iocurrent);
 8002428:	4b0b      	ldr	r3, [pc, #44]	; (8002458 <HAL_GPIO_Init+0x304>)
 800242a:	68da      	ldr	r2, [r3, #12]
 800242c:	69bb      	ldr	r3, [r7, #24]
 800242e:	43db      	mvns	r3, r3
 8002430:	4909      	ldr	r1, [pc, #36]	; (8002458 <HAL_GPIO_Init+0x304>)
 8002432:	4013      	ands	r3, r2
 8002434:	60cb      	str	r3, [r1, #12]
        }
      }
    }

	position++;
 8002436:	6a7b      	ldr	r3, [r7, #36]	; 0x24
 8002438:	3301      	adds	r3, #1
 800243a:	627b      	str	r3, [r7, #36]	; 0x24
  while (((GPIO_Init->Pin) >> position) != 0x00u)
 800243c:	683b      	ldr	r3, [r7, #0]
 800243e:	681a      	ldr	r2, [r3, #0]
 8002440:	6a7b      	ldr	r3, [r7, #36]	; 0x24
 8002442:	fa22 f303 	lsr.w	r3, r2, r3
 8002446:	2b00      	cmp	r3, #0
 8002448:	f47f ae8e 	bne.w	8002168 <HAL_GPIO_Init+0x14>
  }
}
 800244c:	bf00      	nop
 800244e:	bf00      	nop
 8002450:	372c      	adds	r7, #44	; 0x2c
 8002452:	46bd      	mov	sp, r7
 8002454:	bc80      	pop	{r7}
 8002456:	4770      	bx	lr
 8002458:	40010400 	.word	0x40010400

0800245c <HAL_GPIO_WritePin>:
  *            @arg GPIO_PIN_RESET: to clear the port pin
  *            @arg GPIO_PIN_SET: to set the port pin
  * @retval None
  */
void HAL_GPIO_WritePin(GPIO_TypeDef *GPIOx, uint16_t GPIO_Pin, GPIO_PinState PinState)
{
 800245c:	b480      	push	{r7}
 800245e:	b083      	sub	sp, #12
 8002460:	af00      	add	r7, sp, #0
 8002462:	6078      	str	r0, [r7, #4]
 8002464:	460b      	mov	r3, r1
 8002466:	807b      	strh	r3, [r7, #2]
 8002468:	4613      	mov	r3, r2
 800246a:	707b      	strb	r3, [r7, #1]
  /* Check the parameters */
  assert_param(IS_GPIO_PIN(GPIO_Pin));
  assert_param(IS_GPIO_PIN_ACTION(PinState));

  if (PinState != GPIO_PIN_RESET)
 800246c:	787b      	ldrb	r3, [r7, #1]
 800246e:	2b00      	cmp	r3, #0
 8002470:	d003      	beq.n	800247a <HAL_GPIO_WritePin+0x1e>
  {
    GPIOx->BSRR = GPIO_Pin;
 8002472:	887a      	ldrh	r2, [r7, #2]
 8002474:	687b      	ldr	r3, [r7, #4]
 8002476:	611a      	str	r2, [r3, #16]
  }
  else
  {
    GPIOx->BSRR = (uint32_t)GPIO_Pin << 16u;
  }
}
 8002478:	e003      	b.n	8002482 <HAL_GPIO_WritePin+0x26>
    GPIOx->BSRR = (uint32_t)GPIO_Pin << 16u;
 800247a:	887b      	ldrh	r3, [r7, #2]
 800247c:	041a      	lsls	r2, r3, #16
 800247e:	687b      	ldr	r3, [r7, #4]
 8002480:	611a      	str	r2, [r3, #16]
}
 8002482:	bf00      	nop
 8002484:	370c      	adds	r7, #12
 8002486:	46bd      	mov	sp, r7
 8002488:	bc80      	pop	{r7}
 800248a:	4770      	bx	lr

0800248c <HAL_GPIO_TogglePin>:
  * @param  GPIOx: where x can be (A..G depending on device used) to select the GPIO peripheral
  * @param  GPIO_Pin: Specifies the pins to be toggled.
  * @retval None
  */
void HAL_GPIO_TogglePin(GPIO_TypeDef *GPIOx, uint16_t GPIO_Pin)
{
 800248c:	b480      	push	{r7}
 800248e:	b085      	sub	sp, #20
 8002490:	af00      	add	r7, sp, #0
 8002492:	6078      	str	r0, [r7, #4]
 8002494:	460b      	mov	r3, r1
 8002496:	807b      	strh	r3, [r7, #2]

  /* Check the parameters */
  assert_param(IS_GPIO_PIN(GPIO_Pin));

  /* get current Ouput Data Register value */
  odr = GPIOx->ODR;
 8002498:	687b      	ldr	r3, [r7, #4]
 800249a:	68db      	ldr	r3, [r3, #12]
 800249c:	60fb      	str	r3, [r7, #12]

  /* Set selected pins that were at low level, and reset ones that were high */
  GPIOx->BSRR = ((odr & GPIO_Pin) << GPIO_NUMBER) | (~odr & GPIO_Pin);
 800249e:	887a      	ldrh	r2, [r7, #2]
 80024a0:	68fb      	ldr	r3, [r7, #12]
 80024a2:	4013      	ands	r3, r2
 80024a4:	041a      	lsls	r2, r3, #16
 80024a6:	68fb      	ldr	r3, [r7, #12]
 80024a8:	43d9      	mvns	r1, r3
 80024aa:	887b      	ldrh	r3, [r7, #2]
 80024ac:	400b      	ands	r3, r1
 80024ae:	431a      	orrs	r2, r3
 80024b0:	687b      	ldr	r3, [r7, #4]
 80024b2:	611a      	str	r2, [r3, #16]
}
 80024b4:	bf00      	nop
 80024b6:	3714      	adds	r7, #20
 80024b8:	46bd      	mov	sp, r7
 80024ba:	bc80      	pop	{r7}
 80024bc:	4770      	bx	lr
	...

080024c0 <HAL_GPIO_EXTI_IRQHandler>:
  * @brief  This function handles EXTI interrupt request.
  * @param  GPIO_Pin: Specifies the pins connected EXTI line
  * @retval None
  */
void HAL_GPIO_EXTI_IRQHandler(uint16_t GPIO_Pin)
{
 80024c0:	b580      	push	{r7, lr}
 80024c2:	b082      	sub	sp, #8
 80024c4:	af00      	add	r7, sp, #0
 80024c6:	4603      	mov	r3, r0
 80024c8:	80fb      	strh	r3, [r7, #6]
  /* EXTI line interrupt detected */
  if (__HAL_GPIO_EXTI_GET_IT(GPIO_Pin) != 0x00u)
 80024ca:	4b08      	ldr	r3, [pc, #32]	; (80024ec <HAL_GPIO_EXTI_IRQHandler+0x2c>)
 80024cc:	695a      	ldr	r2, [r3, #20]
 80024ce:	88fb      	ldrh	r3, [r7, #6]
 80024d0:	4013      	ands	r3, r2
 80024d2:	2b00      	cmp	r3, #0
 80024d4:	d006      	beq.n	80024e4 <HAL_GPIO_EXTI_IRQHandler+0x24>
  {
    __HAL_GPIO_EXTI_CLEAR_IT(GPIO_Pin);
 80024d6:	4a05      	ldr	r2, [pc, #20]	; (80024ec <HAL_GPIO_EXTI_IRQHandler+0x2c>)
 80024d8:	88fb      	ldrh	r3, [r7, #6]
 80024da:	6153      	str	r3, [r2, #20]
    HAL_GPIO_EXTI_Callback(GPIO_Pin);
 80024dc:	88fb      	ldrh	r3, [r7, #6]
 80024de:	4618      	mov	r0, r3
 80024e0:	f000 f806 	bl	80024f0 <HAL_GPIO_EXTI_Callback>
  }
}
 80024e4:	bf00      	nop
 80024e6:	3708      	adds	r7, #8
 80024e8:	46bd      	mov	sp, r7
 80024ea:	bd80      	pop	{r7, pc}
 80024ec:	40010400 	.word	0x40010400

080024f0 <HAL_GPIO_EXTI_Callback>:
  * @brief  EXTI line detection callbacks.
  * @param  GPIO_Pin: Specifies the pins connected EXTI line
  * @retval None
  */
__weak void HAL_GPIO_EXTI_Callback(uint16_t GPIO_Pin)
{
 80024f0:	b480      	push	{r7}
 80024f2:	b083      	sub	sp, #12
 80024f4:	af00      	add	r7, sp, #0
 80024f6:	4603      	mov	r3, r0
 80024f8:	80fb      	strh	r3, [r7, #6]
  /* Prevent unused argument(s) compilation warning */
  UNUSED(GPIO_Pin);
  /* NOTE: This function Should not be modified, when the callback is needed,
           the HAL_GPIO_EXTI_Callback could be implemented in the user file
   */
}
 80024fa:	bf00      	nop
 80024fc:	370c      	adds	r7, #12
 80024fe:	46bd      	mov	sp, r7
 8002500:	bc80      	pop	{r7}
 8002502:	4770      	bx	lr

08002504 <HAL_RCC_OscConfig>:
  *         supported by this macro. User should request a transition to HSE Off
  *         first and then HSE On or HSE Bypass.
  * @retval HAL status
  */
HAL_StatusTypeDef HAL_RCC_OscConfig(RCC_OscInitTypeDef  *RCC_OscInitStruct)
{
 8002504:	b580      	push	{r7, lr}
 8002506:	b086      	sub	sp, #24
 8002508:	af00      	add	r7, sp, #0
 800250a:	6078      	str	r0, [r7, #4]
  uint32_t tickstart;
  uint32_t pll_config;

  /* Check Null pointer */
  if (RCC_OscInitStruct == NULL)
 800250c:	687b      	ldr	r3, [r7, #4]
 800250e:	2b00      	cmp	r3, #0
 8002510:	d101      	bne.n	8002516 <HAL_RCC_OscConfig+0x12>
  {
    return HAL_ERROR;
 8002512:	2301      	movs	r3, #1
 8002514:	e272      	b.n	80029fc <HAL_RCC_OscConfig+0x4f8>

  /* Check the parameters */
  assert_param(IS_RCC_OSCILLATORTYPE(RCC_OscInitStruct->OscillatorType));

  /*------------------------------- HSE Configuration ------------------------*/
  if (((RCC_OscInitStruct->OscillatorType) & RCC_OSCILLATORTYPE_HSE) == RCC_OSCILLATORTYPE_HSE)
 8002516:	687b      	ldr	r3, [r7, #4]
 8002518:	681b      	ldr	r3, [r3, #0]
 800251a:	f003 0301 	and.w	r3, r3, #1
 800251e:	2b00      	cmp	r3, #0
 8002520:	f000 8087 	beq.w	8002632 <HAL_RCC_OscConfig+0x12e>
  {
    /* Check the parameters */
    assert_param(IS_RCC_HSE(RCC_OscInitStruct->HSEState));

    /* When the HSE is used as system clock or clock source for PLL in these cases it is not allowed to be disabled */
    if ((__HAL_RCC_GET_SYSCLK_SOURCE() == RCC_SYSCLKSOURCE_STATUS_HSE)
 8002524:	4b92      	ldr	r3, [pc, #584]	; (8002770 <HAL_RCC_OscConfig+0x26c>)
 8002526:	685b      	ldr	r3, [r3, #4]
 8002528:	f003 030c 	and.w	r3, r3, #12
 800252c:	2b04      	cmp	r3, #4
 800252e:	d00c      	beq.n	800254a <HAL_RCC_OscConfig+0x46>
        || ((__HAL_RCC_GET_SYSCLK_SOURCE() == RCC_SYSCLKSOURCE_STATUS_PLLCLK) && (__HAL_RCC_GET_PLL_OSCSOURCE() == RCC_PLLSOURCE_HSE)))
 8002530:	4b8f      	ldr	r3, [pc, #572]	; (8002770 <HAL_RCC_OscConfig+0x26c>)
 8002532:	685b      	ldr	r3, [r3, #4]
 8002534:	f003 030c 	and.w	r3, r3, #12
 8002538:	2b08      	cmp	r3, #8
 800253a:	d112      	bne.n	8002562 <HAL_RCC_OscConfig+0x5e>
 800253c:	4b8c      	ldr	r3, [pc, #560]	; (8002770 <HAL_RCC_OscConfig+0x26c>)
 800253e:	685b      	ldr	r3, [r3, #4]
 8002540:	f403 3380 	and.w	r3, r3, #65536	; 0x10000
 8002544:	f5b3 3f80 	cmp.w	r3, #65536	; 0x10000
 8002548:	d10b      	bne.n	8002562 <HAL_RCC_OscConfig+0x5e>
    {
      if ((__HAL_RCC_GET_FLAG(RCC_FLAG_HSERDY) != RESET) && (RCC_OscInitStruct->HSEState == RCC_HSE_OFF))
 800254a:	4b89      	ldr	r3, [pc, #548]	; (8002770 <HAL_RCC_OscConfig+0x26c>)
 800254c:	681b      	ldr	r3, [r3, #0]
 800254e:	f403 3300 	and.w	r3, r3, #131072	; 0x20000
 8002552:	2b00      	cmp	r3, #0
 8002554:	d06c      	beq.n	8002630 <HAL_RCC_OscConfig+0x12c>
 8002556:	687b      	ldr	r3, [r7, #4]
 8002558:	685b      	ldr	r3, [r3, #4]
 800255a:	2b00      	cmp	r3, #0
 800255c:	d168      	bne.n	8002630 <HAL_RCC_OscConfig+0x12c>
      {
        return HAL_ERROR;
 800255e:	2301      	movs	r3, #1
 8002560:	e24c      	b.n	80029fc <HAL_RCC_OscConfig+0x4f8>
      }
    }
    else
    {
      /* Set the new HSE configuration ---------------------------------------*/
      __HAL_RCC_HSE_CONFIG(RCC_OscInitStruct->HSEState);
 8002562:	687b      	ldr	r3, [r7, #4]
 8002564:	685b      	ldr	r3, [r3, #4]
 8002566:	f5b3 3f80 	cmp.w	r3, #65536	; 0x10000
 800256a:	d106      	bne.n	800257a <HAL_RCC_OscConfig+0x76>
 800256c:	4b80      	ldr	r3, [pc, #512]	; (8002770 <HAL_RCC_OscConfig+0x26c>)
 800256e:	681b      	ldr	r3, [r3, #0]
 8002570:	4a7f      	ldr	r2, [pc, #508]	; (8002770 <HAL_RCC_OscConfig+0x26c>)
 8002572:	f443 3380 	orr.w	r3, r3, #65536	; 0x10000
 8002576:	6013      	str	r3, [r2, #0]
 8002578:	e02e      	b.n	80025d8 <HAL_RCC_OscConfig+0xd4>
 800257a:	687b      	ldr	r3, [r7, #4]
 800257c:	685b      	ldr	r3, [r3, #4]
 800257e:	2b00      	cmp	r3, #0
 8002580:	d10c      	bne.n	800259c <HAL_RCC_OscConfig+0x98>
 8002582:	4b7b      	ldr	r3, [pc, #492]	; (8002770 <HAL_RCC_OscConfig+0x26c>)
 8002584:	681b      	ldr	r3, [r3, #0]
 8002586:	4a7a      	ldr	r2, [pc, #488]	; (8002770 <HAL_RCC_OscConfig+0x26c>)
 8002588:	f423 3380 	bic.w	r3, r3, #65536	; 0x10000
 800258c:	6013      	str	r3, [r2, #0]
 800258e:	4b78      	ldr	r3, [pc, #480]	; (8002770 <HAL_RCC_OscConfig+0x26c>)
 8002590:	681b      	ldr	r3, [r3, #0]
 8002592:	4a77      	ldr	r2, [pc, #476]	; (8002770 <HAL_RCC_OscConfig+0x26c>)
 8002594:	f423 2380 	bic.w	r3, r3, #262144	; 0x40000
 8002598:	6013      	str	r3, [r2, #0]
 800259a:	e01d      	b.n	80025d8 <HAL_RCC_OscConfig+0xd4>
 800259c:	687b      	ldr	r3, [r7, #4]
 800259e:	685b      	ldr	r3, [r3, #4]
 80025a0:	f5b3 2fa0 	cmp.w	r3, #327680	; 0x50000
 80025a4:	d10c      	bne.n	80025c0 <HAL_RCC_OscConfig+0xbc>
 80025a6:	4b72      	ldr	r3, [pc, #456]	; (8002770 <HAL_RCC_OscConfig+0x26c>)
 80025a8:	681b      	ldr	r3, [r3, #0]
 80025aa:	4a71      	ldr	r2, [pc, #452]	; (8002770 <HAL_RCC_OscConfig+0x26c>)
 80025ac:	f443 2380 	orr.w	r3, r3, #262144	; 0x40000
 80025b0:	6013      	str	r3, [r2, #0]
 80025b2:	4b6f      	ldr	r3, [pc, #444]	; (8002770 <HAL_RCC_OscConfig+0x26c>)
 80025b4:	681b      	ldr	r3, [r3, #0]
 80025b6:	4a6e      	ldr	r2, [pc, #440]	; (8002770 <HAL_RCC_OscConfig+0x26c>)
 80025b8:	f443 3380 	orr.w	r3, r3, #65536	; 0x10000
 80025bc:	6013      	str	r3, [r2, #0]
 80025be:	e00b      	b.n	80025d8 <HAL_RCC_OscConfig+0xd4>
 80025c0:	4b6b      	ldr	r3, [pc, #428]	; (8002770 <HAL_RCC_OscConfig+0x26c>)
 80025c2:	681b      	ldr	r3, [r3, #0]
 80025c4:	4a6a      	ldr	r2, [pc, #424]	; (8002770 <HAL_RCC_OscConfig+0x26c>)
 80025c6:	f423 3380 	bic.w	r3, r3, #65536	; 0x10000
